:100000000C9455090C9486090C9486090C94860965
:100010000C9486090C9486090C9486090C94860924
:100020000C9486090C9486090C9486090C94860914
:100030000C9486090C94C00E0C9486090C948609C5
:100040000C9486090C9486090C9486090C948609F4
:100050000C9486090C9486090C9486090C94C20DA4
:100060000C9486090C9475860C944B860C94860926
:100070000C9486090C9486090C9486090C948609C4
:100080000C9486090C9486090C9486090C948609B4
:100090000C9486090C9486090C9486090C94E30F41
:1000A0000C9486090C9486090C9486090C94860994
:1000B0000C9486090C9486090C9486090C94860984
:1000C0000C9486090C9486090C9486090C94860974
:1000D0000C9486090C9486090C9415860C94EB8577
:1000E0000C9486090C94010B0C94A90A0C9490248E
:1000F0000C94040C0C94FD210C9414770C94D10CEA
:100100000C94A1270C9442240C94BA0A0C94F50B7D
:100110000C94D00B0C94F1760C94300B0C947F372C
:100120000C94FF220C94040D0C94E80C0C94EC0C31
:100130000C94AB0A0C9422770C94D1270C94F10BFD
:100140000C94D40C0C94031A0C94E2960C94FC2797
:100150000C94ED2D0C940C0C0C94BF0C0C94F1250C
:100160000C94A80A0C94FF0B0C9421850C94D325B5
:100170000C9483220C94000D0C9416230C942722CB
:100180000C94240C0C9406210C94390E0C94272802
:100190000C94D51F0C94C9230C94D4750C94C50CE5
:1001A0000C94100C0C94982D0C949D220C94BA0B6A
:1001B0000C94E40C0C94BE220C94010C0C9400776B
:1001C0000C94CD0A0C94F60C0C9450200C94F779F6
:1001D0000C94D6190C94C3760C94C5170C94D21BAE
:1001E0000C94DA0C0C94CF170C9435200C942B0C37
:1001F0000C94FA0C0C945C260C94FF0C0C947A2052
:100200000C94B1770C94BF200C94F20C0C94A58C38
:100210000C942E0C0C942B260C9464770C942B6F5E
:100220000C9420240C94500B0C94B60B0C94A00B43
:100230000C947B240C94140C0C94CD0C0C94AA0AF2
:100240000C942E180C94C90C0C94CE200C94DE2126
:100250000C94DE0C0C94E31B0C94D40A0C94DB0B72
:100260000C94C4764E414E494E495459494E46CDA0
:10027000CCCC3D0AD7233C17B7D13877CC2B32955D
:1002800095E6241FB14F0A000020410000C842003B
:10029000401C4620BCBE4CCA1B0E5AAEC59D740005
:1002A000407A10F35A00A0724E18090010A5D4E845
:1002B0000000E87648170000E40B54020000CA9AD8
:1002C0003B000000E1F5050000809698000000402A
:1002D000420F000000A0860100000010270000006F
:1002E00000E803000000006400000000000A0000B5
:1002F0000000000100000000002C76D888DC674F69
:100300000823DFC1DFAE59E1B1B796E5E3E453C698
:100310003AE651997696E8E6C28426EB898C9B6290
:10032000ED407C6FFCEFBC9C9F40F2BAA56FA5F43A
:1003300090055A2AF75C936B6CF9676DC11BFCE062
:10034000E40D47FEF520E6B500D0ED902E030094B5
:100350003577050080841E080000204E0A0000004A
:10036000C80C333333330F986E12831141EF8D2154
:1003700014893BE65516CFFEE6DB18D1844B381BBB
:10038000F77C1D901DA4BBE424203284725E228180
:1003900000C9F124ECA1E53D27436F6E74656E74CE
:1003A0002D547970653A20746578742F68746D6C7B
:1003B0000D0A0D0A3C68313E4550494320464149EB
:1003C0004C3C2F68313E00485454502F312E302081
:1003D0003430302042616420526571756573740D4C
:1003E0000A004163636573732D436F6E74726F6CA3
:1003F0002D416C6C6F772D4F726967696E3A202AB8
:100400000D0A436F6E74656E742D547970653A20D1
:10041000005365727665723A205765626475696E3D
:100420006F2F312E370D0A00485454502F312E3083
:1004300020323030204F4B0D0A00506F737420660D
:1004400061696C656400436F6E6E656374696F6E9D
:100450003A20636C6F73650D0A00436F6E6E6563BF
:1004600074696F6E3A20636C6F73650D0A436F6E2B
:1004700074656E742D547970653A206170706C6982
:10048000636174696F6E2F782D7777772D666F7241
:100490006D2D75726C656E636F646564002D2D2D16
:1004A0002D2D2D5765624B6974466F726D426F75C5
:1004B0006E646172796A6732715649555338746552
:1004C0004F41624E332D2D00436F6E74656E742D57
:1004D000547970653A206170706C69636174696FFA
:1004E0006E2F6F637465742D73747265616D004354
:1004F0006F6E74656E742D446973706F736974697F
:100500006F6E3A20666F726D2D646174613B206E70
:10051000616D653D2266696C65223B2066696C658C
:100520006E616D653D22002D2D2D2D2D2D5765629F
:100530004B6974466F726D426F756E646172796A51
:10054000673271564955533874654F41624E3300D6
:10055000436F6E74656E742D4C656E6774683A20D7
:1005600000436F6E74656E742D547970653A206D1A
:10057000756C7469706172742F666F726D2D646131
:1005800074613B20626F756E646172793D2D2D2D13
:100590002D5765624B6974466F726D426F756E645C
:1005A0006172796A673271564955533874654F41A3
:1005B000624E3300436F6E6E656374696F6E3A20EE
:1005C000636C6F736500504F53542055706C6F61AE
:1005D00064204661696C65643A2000234E6F207385
:1005E000656E736F7220666F722074656D70202661
:1005F0002068756D696469747921004E6F205365B8
:100600006E736F72210020666F722074656D7020AA
:10061000262068756D696469747921002353656EBD
:10062000736F72204572726F72200053656E736F24
:1006300072204572726F7221002357726F6E6720AD
:1006400073656E736F7220666F722074656D7020B3
:10065000262068756D6964697479210057726F6E20
:10066000672053656E736F7221004320483D00542C
:100670003D0020202020202020202020202020207D
:10068000202000202020202020202020202020208A
:10069000202020002020202020202020202020207A
:1006A000202020200020202020202020202020206A
:1006B000202020200020202020202020202020205A
:1006C000202020200054696D657374616D70207561
:1006D000706C6F6164206661696C65640053657459
:1006E00074696E6720636C6F636B2074696D65005D
:1006F000236572726F72202D20004950206164645E
:10070000726573733A2000496E76616C6964205398
:100710004D2073746570732070657220616E676C14
:10072000653D00534D2073746570732070657220B1
:10073000616E676C653D003C703E54696D653A20A2
:10074000003C2F68333E0A003C62723E4254206EE9
:10075000616D653D003C62723E506174683D003CD5
:1007600068333E53797374656D3A205665727369C8
:100770006F6E3D00506172616D65746572732072B9
:100780006573657420646F6E6521002F6F652F732C
:100790006D6C69676874706F2F73332F00234C6121
:1007A0006D7020766F6C746167652070617269741A
:1007B000793A2000235461626C6520616E676C6534
:1007C00020646972656374696F6E3A200023437513
:1007D0007272656E7420534D206973202300235379
:1007E0004D3A5461626C6520737465707320706556
:1007F0007220616E676C653D0023534D3A506F6CFB
:100800006172697A657220737465707320706572A5
:1008100020616E676C653D002344485450494E3D4D
:1008200000234448543D00236E65743D424C45000E
:10083000236E65743D5769466900236E65743D42B9
:1008400054002366747020757365726E616D653A2D
:10085000003A0023486F73742073657276657220C6
:10086000495020616E6420506F72743A00235469BD
:100870006D65207365727665722049503A00235287
:10088000656C617920646576696365733A0023520B
:10089000656C617920737461747573206C61626535
:1008A0006C733A20002352656C6179207374617413
:1008B00065733A002352656C61792070696E733AF2
:1008C00000234E6F2E206F6620636F6E74726F6C04
:1008D0002072656C6179733D00234E6F2E206F6628
:1008E0002072656C6179733D000A00446576696326
:1008F0006520737461747573206174200046696E9D
:1009000064696E672057694669204950004E455416
:100910003D426C7565746F6F7468204C45004E45A0
:10092000543D426C7565746F6F7468004E45543D5C
:1009300057694669005344206F70656E206661698F
:100940006C004E6577206461746120636F6C6C6528
:100950006374696F6E2073746172746564005348C8
:100960004F57533D0048494748004C4F57004E45AC
:1009700057002343757272656E74207365747469D1
:100980006E67733A005345540053797374656D2054
:10099000726573657420617420005245534554009C
:1009A0005052494E54504152005245414453440024
:1009B0005341564553443D002344532054686572C7
:1009C0006D6F6D657465722063616C6962726174CC
:1009D000656420666F7220230044535400496E768C
:1009E000616C696420616E676C6520666F722000BF
:1009F0004D323D004E3D004D323D004E3D002073D6
:100A0000746570732070657220616E676C653D005F
:100A10005350413D00545350413D00505350413DCF
:100A2000005350413D0020737465707320706572EF
:100A300020616E676C653D004631303030004635D0
:100A4000303000463130303000414E474D00544187
:100A50004E47430050414E474300414E47430054E8
:100A600061626C654000506F6C6172697A657240BA
:100A700000414E474D3D0054414E474D3D005041D1
:100A80004E474D3D00414E474D3D00414E47533D81
:100A9000005233300054414E47533D0050414E47C1
:100AA000533D00414E47533D005200414E474C4597
:100AB0003D0054413D0050413D00413D00414E4705
:100AC0004C453D005461626C6520536574203000D4
:100AD000235475726E7461626C65205365742030A6
:100AE000005233300046333000506F6C6172697AC7
:100AF00065722053657420300023506F6C617269F9
:100B00007A657220536574203000505A45524F3D2B
:100B100000540050005A45524F005461626C6520E9
:100B2000536574203000235475726E7461626C6575
:100B300020536574203000506F6C6172697A657261
:100B40002053657420300023506F6C6172697A65A0
:100B5000722053657420300053455400505A45525A
:100B60004F3D005A45524F0053504545443D0050BB
:100B700053504545443D005453504545443D005372
:100B8000504545443D004D3D004D4F544F523D00B2
:100B90004D3D004D4F544F523D00534D3D00535479
:100BA00045503D004453544E3D0052564849474835
:100BB0003D0052564C4F573D004C4F5746414E5406
:100BC000494D453D00484947484D4F544F523D001F
:100BD0004C4F574D4F544F523D004849474854459C
:100BE0004D503D004C4F5754454D503D0054454DE0
:100BF00050433D007361766553443D004E45543D7E
:100C000000576946692049503A0049504144440020
:100C100041542B0050494E3D0042543D004C43444A
:100C20003D00534554434C4F434B00234C6F676783
:100C30006572204E616D653A20004C4F4747455222
:100C40000056455253494F4E00234465766963650B
:100C5000207374617475732075706C6F6164656462
:100C6000210055535441545553005265626F6F74BF
:100C7000696E672E2E2E005245424F4F5400536529
:100C80007276657220506F7274207570646174653D
:100C9000640053504F52543D0049502075706461B8
:100CA000746564005349503D002354696D652053B9
:100CB0006572766572204950207570646174656450
:100CC00000545349503D0052454C41593F00524554
:100CD0004C415920004352454C415900444854501E
:100CE000494E3D00524E414D453D004E523D005053
:100CF00052494E54004E554E4348554B3D004155C8
:100D0000544F53544152543D0074696D6520696ECF
:100D100074657276616C3D0054494D453D005449FF
:100D20004D455354414D503D0054494D4553544158
:100D30004D500053484F5749500054455354524565
:100D40004C415900434845434B433D0043484543CC
:100D50004B543D004453543D004C5041524954596A
:100D60003D0046414E3D004F56454E3D00444854DF
:100D70003D0050573D00555345523D0050415448A9
:100D80003D007C3C3E5E2B3D3F2F5B5D3B2C2A2291
:100D90005C003C703E4C616D7020616E64204D6F54
:100DA000746F722044726976657273205374617433
:100DB0007573EFBC9A3C2F703E003C21646F6374E6
:100DC0007970652068746D6C3E3C68746D6C3E3C57
:100DD000686561643E3C6D6574612063686172732F
:100DE00065743D227574662D38223E3C7469746CBE
:100DF000653E4F6E6C696E65206578706572696DD1
:100E0000656E74202D20506F6C6172697A6174690F
:100E10006F6E2065666665637473206F66206C690B
:100E20006768743C2F7469746C653E3C2F6865611B
:100E3000643E3C626F64793E3C68313E4F6E6C6943
:100E40006E65206578706572696D656E74202D2001
:100E5000506F6C6172697A6174696F6E2065666645
:100E600065637473206F66206C696768743C2F68D3
:100E7000313E003C68343E436F7079726967687434
:100E8000284329323032302D323032322E50726FB8
:100E9000662E205945554E47205961752059756574
:100EA0006E3C2F68343E3C2F626F64793E3C2F6865
:100EB000746D6C3E003C68313E43616E6E6F742011
:100EC0006765742073656E736F7220726561646903
:100ED0006E6773213C2F68313E0000002000230024
:100EE000260029002C002F00320000010000030121
:100EF0000601090100000A0B02090C0D0E08070388
:100F000004010000000000000000000000000000DC
:100F100000000000000000000000000000000000D1
:100F2000121110000000000000000000000000008E
:100F30000000000000000000000023776562736578
:100F40007276657220626567696E730053657474AA
:100F5000696E672049500053657474696E67204458
:100F60006576696365204950202E2E2E00546573E6
:100F700074204C616D70732F46616E7300657272E0
:100F80006F72206F70656E696E672066696C653A76
:100F900020004C616D70204D6F746F720023546996
:100FA0006D652020202020204461746520202020B1
:100FB000205365636F6E647320506F6C6172697A41
:100FC0006572205461626C652054286F4329204863
:100FD000282529202000696E69742E20646F6E65B3
:100FE0002E00534420696E69742E206661696C6519
:100FF000642100696E69742E206661696C656421E4
:101000000053657474696E672049502063616D00F8
:101010002323204F452057656C636F6D6520232384
:1010200000496E697469616C697A696E672053441E
:1010300020636172642E2E2E0053797374656D20C7
:101040007374617274696E672E2E2E00202D2075C8
:10105000706C6F616420627920504F535420666138
:10106000696C65642100202D2075706C6F616420AF
:10107000627920504F5354204F4B210053797374A1
:10108000656D20726573746172746564210020530C
:10109000797374656D20726573746172746564210F
:1010A00000234E6574776F726B206D61696E746199
:1010B000696E656420617420002323436F6D6D6148
:1010C0006E64400000002200250028002B002E0046
:1010D0003100340002010000050108010B0100008D
:1010E0002100240027002A002D00300033000101D8
:1010F0000000040107010A01010210202008081065
:101100002040102040800201020108040201010277
:101110000408102040808040201008040201800450
:1011200002018040201008040201080402010102AB
:1011300004081020408001020408102040800505AA
:101140000505070508080808020202020A0A08083D
:10115000040404040101010101010101030303036B
:1011600003030303040707070C0C0C0C0C0C0C0CFA
:101170000202020206060606060606060B0B0B0B0B
:101180000B0B0B0B417070656E64206D6561732EE7
:10119000200053696E676C65206D6561732E2000B9
:1011A00053617665206D65617375726520746F3A61
:1011B000002020202020202020202020202020204F
:1011C00020000000010001001010020001000100D9
:1011D000B000000016000000280000001000000011
:1011E00020000000010001000000000000000000DD
:1011F00000000000000000000000000000000000EF
:1012000000000000FF000000FFFF0000FFFF0000E3
:10121000FFFF0000CFBF0000C7BF0000C3BF00003A
:10122000C1BF0000C0BF000000000000C0BF000040
:10123000C1BF0000C3BF0000C7BF0000CFBF000098
:10124000FFFF0000FFFF00000000000000000000A2
:10125000000000000000000000000000000000008E
:10126000000000000000000000000000000000007E
:10127000000000000000000000000000000000006E
:101280000000000000000000557365722D61676565
:101290006E743A202A0D0A446973616C6C6F773A58
:1012A000202F0D0A0000E296A58C11241FBECFEF5F
:1012B000D1E2DEBFCDBF00E00CBF18E0A0E0B2E09D
:1012C000E0E8F2E701E00BBF02C007900D92A439FD
:1012D000B107D9F724E1A4E9B8E001C01D92A0321A
:1012E000B207E1F719E0C4E5D9E000E006C02197B4
:1012F0000109802FFE010E9447B6C335D10780E067
:101300000807A9F70E949F990C942EB90C9400002D
:101310004F925F926F927F928F929F92AF92BF9205
:10132000CF92DF92EF92FF920F931F93CF93DF93B1
:101330004B015C018091A90B9091AA0BA091AB0B82
:10134000B091AC0B88159905AA05BB0509F4C6C078
:101350008CE3C82ED12CE12CF12CC501A7019601FC
:101360000E94B1B46093AD0BCA01B901A701960107
:101370000E94B1B46093AE0BC501B40120E13EE020
:1013800040E050E00E94B1B4CA01B90128E130E068
:1013900040E050E00E94B1B46093AF0BC501B401CE
:1013A00020E831E541E050E00E94B1B469017A01E2
:1013B000CA01B9016C5F7F4F8F4F9F4F27E030E02C
:1013C00040E050E00E94B1B46F5F6093B00B412CDD
:1013D000512C320140E004E610E0C0E9D1E0242FB6
:1013E00030E02E54384FF901E370FF273097F9F4BD
:1013F000C901B8010E9433B6892B31F4C901BE017D
:101400000E9433B6892B99F48EE691E0A0E0B0E01B
:10141000480E591E6A1E7B1ED301C201AA27BB2794
:10142000C816D906EA06FB0638F04F5FD8CF8DE61E
:1014300091E0A0E0B0E0ECCF4093B30BC90164E6CB
:1014400070E00E9433B6EC01C90160E971E00E94CE
:1014500033B6309721F42097D9F40097C9F04DE6C0
:1014600051E060E070E0441A550A660A770AC41831
:10147000D508E608F708A5E2B3E020E0213069F4DA
:101480003097E9F5209711F40097C9F54DE106C0B2
:101490004EE651E060E070E0E6CF4C9150E070E045
:1014A00060E031E0320FC416D506E606F70640F0DC
:1014B000C41AD50AE60AF70A1196232F3C30F1F632
:1014C0002F5F2093B20BC394C092B10B8092A90BF3
:1014D0009092AA0BA092AB0BB092AC0BDF91CF9184
:1014E0001F910F91FF90EF90DF90CF90BF90AF9042
:1014F0009F908F907F906F905F904F9008954CE1F8
:10150000CDCF2091B50A260F3327331F2132310565
:10151000ECF420917F0EFC0190E080E0243069F033
:1015200082E00895A091B50A2191AC014B56554F28
:10153000A40FB52FB11D2C930196861798F38091B7
:10154000B50A680F6093B50A80E0089581E00895B8
:10155000089508950895E0913A0C8091390CE817A8
:1015600030F4F0E0EC58F54F808190E008958FEF73
:101570009FEF089590913A0C8091390C2FEF3FEF37
:10158000981748F4E92FF0E0EC58F54F208130E04F
:101590009F5F90933A0CC90108958091390C909106
:1015A0003A0C891B990B0895CF92DF92EF92FF922C
:1015B0000F931F93CF93DF937C01CB018A0120917E
:1015C000850E222389F0EB016B01C40ED51ECC15CC
:1015D000DD0569F06991D701ED91FC910190F081F1
:1015E000E02DC7011995F3CF642F0E94810AC8012D
:1015F000DF91CF911F910F91FF90EF90DF90CF90EF
:101600000895CF93DF931F92CDB7DEB76983209102
:10161000850E2223F9F02091A80E203258F021E007
:1016200030E0FC013383228390E080E00F90DF9173
:10163000CF9108958091860EE82FF0E0E957F14FA1
:10164000998190838F5F8093860E8093A80E81E0AE
:1016500090E0ECCF61E0CE0101960E94810AF7CFC5
:10166000DC015996ED91FC913097B9F0838994890A
:10167000A589B6894285538564857585841B950B3C
:10168000A60BB70B811520E89207A105B10538F02C
:101690008FEF9FE7A0E0B0E0089590E080E008952C
:1016A000CF93DF931F92CDB7DEB76983DC01ED9155
:1016B000FC910280F381E02D41E050E0BE016F5FBC
:1016C0007F4F19950F90DF91CF910895FC012081F4
:1016D0002EBD9B012150310941F051810DB407FE0F
:1016E000FDCF4EB55EBD4193F5CF61507109860FB8
:1016F000971F0DB407FEFDCF2EB5FC012083089582
:10170000E0913E0CF0913F0C908180913D0C8095D2
:101710008923808308958EBD00000DB407FEFDCFA0
:101720008EB5089590E02091400C233339F40C9647
:10173000982F990F990F990F80E008954896F8CF48
:10174000CF93DF931F92CDB7DEB76983DC01ED91B4
:10175000FC910280F381E02D41E050E0BE016F5F1B
:101760007F4F19950F90DF91CF910895FC01818DE6
:10177000928D0895CF93DF931F92CDB7DEB7698323
:10178000DC01ED91FC910280F381E02D41E050E01D
:10179000BE016F5F7F4F19950F90DF91CF91089534
:1017A000FC019485FB018485981303C081E0983087
:1017B00008F080E00895CF93DF931F92CDB7DEB796
:1017C0006983DC01ED91FC910280F381E02D41E021
:1017D00050E0BE016F5F7F4F19950F90DF91CF9161
:1017E0000895FC01768765870895DC01ED91FC91F1
:1017F000068CF78DE02D199591E089270895862FA5
:10180000089581E08627089521E0FC0184858830D1
:1018100008F020E0822F0895FC01848595850895C5
:10182000FC0184899589089520E334E0FC0131832B
:101830002083FB014089518962897389FC014283BD
:101840005383648375830895DC01ED91FC91048CCE
:10185000F58DE02D199490E080E00895CF92DF920D
:10186000EF92FF920F931F93CF93DF93CDB7DEB725
:10187000AF970FB6F894DEBF0FBECDBF7C016A01F3
:1018800000E314E01A8309831C861B8688EE93E02C
:10189000A0E0B0E08D879E87AF87B88B8AEB93E09E
:1018A0009A878987188F0F8B198E1A8E1B8E1C8E24
:1018B00088E089A31BA70AA71CA61DA61EA61FA613
:1018C00080913B1090913C10A0913D10B0913E1042
:1018D0008EA39FA3A8A7B9A78B839C83AD83BE8348
:1018E00018861F82AE01465D5F4FCE0101960E94B1
:1018F000937D81309105B1F4D701ED91FC9104887D
:10190000F589E02D1DA30CA38CA59DA5AEA5BFA5B3
:101910008EA39FA3A8A7B9A7A601BE016C5D7F4FA8
:10192000C7011995AF960FB6F894DEBF0FBECDBFB5
:10193000DF91CF911F910F91FF90EF90DF90CF90AB
:1019400008958150823108F05AC0E82FF0E08827CE
:10195000E355F34F8F4F0C9447B6CD0CD10CBF0C11
:10196000C50CC90CFF0CD40CDA0CDE0CE40CE80C32
:10197000EC0CF20CF60CFF0CFA0C000D040D80912F
:1019800080008F77809380000895809180008F7D04
:10199000F9CF80918000877FF5CF84B58F7784BDA4
:1019A000089584B58F7DFBCF8091B0008F778093B1
:1019B000B00008958091B0008F7DF9CF80919000A4
:1019C0008F77809390000895809190008F7DF9CF5C
:1019D00080919000877FF5CF8091A0008F778093D2
:1019E000A00008958091A0008F7DF9CF8091A00084
:1019F000877FF5CF809120018F7780932001089514
:101A0000809120018F7DF9CF80912001877FF5CFD4
:101A1000CF93DF9390E0FC01E850FF4E2491825C6D
:101A20009E4EFC0184918823D1F090E0880F991F8D
:101A3000FC01E252FF4EA591B491FC01EC53FF4E24
:101A4000C591D49161110EC09FB7F8948C91E22F8B
:101A5000E0958E238C932881E223E8839FBFDF915A
:101A6000CF9108958FB7F894EC91E22BEC938FBF50
:101A7000F6CF3FB7F8948091C70B9091C80BA09117
:101A8000C90BB091CA0B26B5A89B05C02F3F19F012
:101A90000196A11DB11D3FBFBA2FA92F982F8827EE
:101AA000BC01CD01620F711D811D911D42E0660FC9
:101AB000771F881F991F4A95D1F708958F929F929B
:101AC000AF92BF92CF92DF92EF92FF926B017C01B7
:101AD0000E94390D4B015C01C114D104E104F104F1
:101AE000B9F00E94390D681979098A099B09683E85
:101AF00073408105910580F321E0C21AD108E10805
:101B0000F10888EE880E83E0981EA11CB11CE4CF7A
:101B1000FF90EF90DF90CF90BF90AF909F908F900D
:101B200008952FB7F8946091C30B7091C40B809106
:101B3000C50B9091C60B2FBF08956093BE0B709399
:101B4000BF0B8093C00B9093C10B645D7E4F8F4F92
:101B50009F4F6093BA0B7093BB0B8093BC0B909319
:101B6000BD0B82E090E09093B90B8093B80B0E947C
:101B7000910D6093B40B7093B50B8093B60B90935B
:101B8000B70B08951F920F920FB60F9211242F9347
:101B90003F938F939F93AF93BF938091C30B90918B
:101BA000C40BA091C50BB091C60B3091C20B23E0C2
:101BB000230F2D3758F50196A11DB11D2093C20B9F
:101BC0008093C30B9093C40BA093C50BB093C60B2B
:101BD0008091C70B9091C80BA091C90BB091CA0B13
:101BE0000196A11DB11D8093C70B9093C80BA093C4
:101BF000C90BB093CA0BBF91AF919F918F913F9149
:101C00002F910F900FBE0F901F90189526E8230F6D
:101C10000296A11DB11DD2CFFC01248131E0309389
:101C2000850E2093A70E1092860E1092A80E838523
:101C3000682B84EE9FE00E94010B81E00C94837A74
:101C40000F931F93CF938C01C62F0E940C0E6C2F05
:101C50006460C8010E940C0E6C2F6B7FC8010E944B
:101C60000C0E83EC90E00197F1F7CF911F910F914B
:101C700008950F931F93CF938C01C62F607F6160EF
:101C80000E94200E80E1C89FB00111246160C8014C
:101C90000E94200E81E090E0CF911F910F91089556
:101CA000CF92DF92EF92FF920F931F930E94910DBC
:101CB0008B019C01C090B40BD090B50BE090B60B9B
:101CC000F090B70B6091BE0B7091BF0B8091C00B71
:101CD0009091C10B0C191D092E093F09083E1340B4
:101CE00021053105E0F0DC01CB010196A11DB11DFC
:101CF0008093BE0B9093BF0BA093C00BB093C10B0E
:101D0000B701A60148515C4F6F4F7F4F4093B40B12
:101D10005093B50B6093B60B7093B70BC7CF1F9161
:101D20000F91FF90EF90DF90CF9008950E94500E9A
:101D30000E9488098091B30B90E08E54984F0895CB
:101D40000E94500E0E9488098091B20B90E0089585
:101D50000E94500E0E9488098091B10B90E0089576
:101D60000E94500E0E9488098091AE0B90E0089569
:101D70000E94500E0E9488098091AF0B90E0089558
:101D80001F920F920FB60F9211240BB60F922F9342
:101D90003F934F935F936F937F938F939F93AF93F3
:101DA000BF93EF93FF938091D90A0E94AB86209155
:101DB000DC0A3091DD0A2F5F3F4F3093DD0A20931C
:101DC000DC0A9091DB0A953618F096E09093D80AD9
:101DD0009091D80A943009F46EC0F8F4923031F141
:101DE000933009F44CC09091DA0A992319F08111CB
:101DF00071C02F9AFF91EF91BF91AF919F918F91F9
:101E00007F916F915F914F913F912F910F900BBEFA
:101E10000F900FBE0F901F901895953009F457C082
:101E2000963009F791E09093A80B4FC08111DBCF5A
:101E30002091DC0A3091DD0A2436310528F4109215
:101E4000DD0A1092DC0ACFCF1092A80B1092DB0AA9
:101E5000E091DB0A91E09E0F9093DB0AF0E0209185
:101E6000DC0A3091DD0AEE0FFF1FE252F54F31839D
:101E700020831092DD0A1092DC0A93E019C08130B1
:101E800009F0B1CFE091DB0A91E09E0F9093DB0A5D
:101E9000F0E02091DC0A3091DD0AEE0FFF1FE252E4
:101EA000F54F318320831092DD0A1092DC0A94E012
:101EB0009093D80A98CF882359F22091DC0A309168
:101EC000DD0A2536310508F48ECF95E0F1CF81117A
:101ED0008ACFB5CF2F988ECF10927F0E81E080935E
:101EE0007E0E1092590E61E084E10E94D48661E07A
:101EF00085E10E94D486E9EBF0E080818E7F8083CB
:101F000080818D7F808388E48093B80085E480930E
:101F1000BC000895CF93DF9391E09093940A8823B7
:101F2000B9F0C091B800D091BA008091BC008A7B12
:101F30008093BC0060E084E10E94D48660E085E18B
:101F40000E94D4860E946C0FD093BA00C093B80050
:101F5000DF91CF91089585ED8093BC008091810E33
:101F60009091820EA091830EB091840E0796A11DD0
:101F7000B11D23E0B695A795979587952A95D1F73A
:101F80002091BC0024FD03C010927F0E0895409163
:101F9000810E5091820E6091830E7091840E452BBC
:101FA000462B472B69F30097A105B10541F025E3C6
:101FB0002A95F1F700000197A109B109E1CF8091BD
:101FC000800E0C948A0F1F920F920FB60F9211245D
:101FD0000BB60F922F933F934F935F936F937F9323
:101FE0008F939F93AF93BF93EF93FF938091B9002B
:101FF000887F803609F44DC008F040C0883209F46B
:10200000A9C028F5803109F49DC0C8F4882309F4DB
:10201000FBC0883009F496C0FF91EF91BF91AF915A
:102020009F918F917F916F915F914F913F912F91F0
:102030000F900BBE0F900FBE0F901F901895883118
:1020400009F488C0803241F780937D0E14C080343B
:1020500009F49DC040F48033B9F38833E9F68093E6
:102060007D0E85ECB0C0803509F485C0883509F453
:1020700096C0883489F60E94AB0FCECF883909F418
:102080008CC038F5883729F050F4883611F0803745
:1020900019F683E080937F0E1092D70A57C08838D4
:1020A00009F47BC0803919F0803809F0B5CF8091F0
:1020B000D70A803208F071C0E091D70A81E08E0F14
:1020C0008093D70A8091BB00F0E0E954F54F8083FC
:1020D0003DC0803B39F0E0F4803A09F479C0883A99
:1020E00009F09ACF84E080937F0E1092B60A109286
:1020F000B50AE091370CF091380C19958091B50A2A
:1021000081110FC081E08093B50A1092950A09C031
:10211000803C09F4A6CF883C09F4A3CF883B09F0A2
:102120007BCFE091B60A81E08E0F8093B60AF0E093
:10213000EB56F54F80818093BB009091B60A809159
:10214000B50A29C080915A0E8093BB0085EC80931C
:10215000BC0062CF90917C0E80917B0E981758F551
:10216000E0917C0E81E08E0F80937C0EF0E0E55ACA
:10217000F14F8081E9CFE0917C0E81E08E0F80935A
:102180007C0E8091BB00F0E0E55AF14F8083909186
:102190007C0E80917B0E9817C8F285E8D8CFE0912D
:1021A0007C0E81E08E0F80937C0E8091BB00F0E06E
:1021B000E55AF14F808380917E0E81115CCF81E0E2
:1021C0008093590E84EA8093BC0010927F0E24CF36
:1021D00085EC8093BC0010927F0E8091D70A8032EC
:1021E00030F4E091D70AF0E0E954F54F10826091A5
:1021F000D70A70E0E091350CF091360C87EB9AE04D
:1022000019951092D70A08CF10927D0E34CF61E055
:10221000FC0184810C94D486CF93DF93EC018FEF83
:102220008EBD2FEF8F819885AC014F5F5F4F588730
:102230004F838130924028F40DB407FEFDCF2EBDB0
:10224000F1CF0DB407FEFDCFCE010E9407111E8213
:10225000DF91CF9108958EBD0DB407FEFDCF089597
:102260008FEF0E942B118EB508958F929F92AF929F
:10227000BF92FF920F931F93CF93DF93EC01F62E43
:1022800049015A018E81882319F0CE010E940C1158
:1022900060E08C810E94D4868CE291E00E94CD7C2B
:1022A0008F2D80640E942B1108E110E0D501C4013C
:1022B000002E04C0B695A795979587950A94D2F7F6
:1022C0000E942B1108501109083F8FEF180771F772
:1022D00085E9FF2021F088E0F8120DC087E80E9410
:1022E0002B1110E00E9430118A8787FF06C01F3F24
:1022F00021F01F5FF7CF8FEFF2CFDF91CF911F91CA
:102300000F91FF90BF90AF909F908F900895AF92E4
:10231000BF92CF92DF92EF92FF920F931F93CF93D2
:10232000DF93EC016901C801820F931F8130924055
:1023300050F58E81882379F088819981AA81BB81AB
:1023400084179507A607B70731F48F819885C816BB
:10235000D90608F042C0488359836A837B838B8502
:10236000833039F089E0440F551F661F771F8A9527
:10237000D1F79A01AB0161E1CE010E9435118823AA
:1023800089F083E08D83CE010E94071180E0DF9108
:10239000CF911F910F91FF90EF90DF90CF90BF9062
:1023A000AF9008950E94910D5B010E9430118A87C1
:1023B0008F3F69F40E94910D6A197B096D3271405B
:1023C000A0F38FE08D83CE010E940711DCCF8E3FFA
:1023D000B1F418861F8281E08E838FEF8EBD2FEFC0
:1023E0008F8198858C159D0560F40DB407FEFDCF97
:1023F0002EBD8F819885019698878F83F1CF8DE0D0
:10240000E1CFC8010197F7012FEFAF014E195F0926
:102410004817590738F40DB407FEFDCF3EB5319388
:102420002EBDF3CF0DB407FEFDCF2EB5E80EF91E7D
:10243000F70120838F819885080F191F18870F8354
:102440008985882319F00115124030F08E81882388
:1024500019F0CE010E940C1181E099CF0F931F93C8
:10246000CF93DF93EC01890182E1411551056105AC
:10247000710599F08B85833039F089E0440F551F41
:10248000661F771F8A95D1F79A01AB0168E1CE01EB
:102490000E943511882319F084E08D8338C08EEFB7
:1024A0008EBDF801C8019E5F0DB407FEFDCF2081EF
:1024B0002EBD0DB407FEFDCF21812EBD3296E8174B
:1024C000F90791F70DB407FEFDCF8FEF0E942B1196
:1024D0008FEF0E942B110E9430118A878F718530F7
:1024E00089F488E592E00E94CD7C8823A9F020E061
:1024F00030E0A9016DE0CE010E943511882371F012
:1025000084E1CBCF81E18D83CE010E940711CE0102
:102510000E94071180E00AC085E1BFCF0E94301100
:102520008111EECFCE010E94071181E0DF91CF91A2
:102530001F910F91089580916F0A8823A9F140910E
:10254000460250914702609148027091490225E588
:102550003CE080913B0C90913C0C0E942E1281112A
:1025600002C080E008954091700A5091710A609114
:10257000720A7091730A411551056105710591F058
:1025800025E53CE080913B0C90913C0C0E942E1282
:10259000882339F31092700A1092710A1092720A0D
:1025A0001092730A10926F0A81E008958F929F92A1
:1025B000AF92BF92EF92FF920F931F93CF934B0175
:1025C0005C01C42F8091460290914702A09148027D
:1025D000B091490288159905AA05BB0549F10E94E9
:1025E0009B1281110BC080E0CF911F910F91FF9042
:1025F000EF90BF90AF909F908F90089585E5E82E63
:102600008CE0F82E00E012E030E020E0B501A401FB
:1026100080913B0C90913C0C0E948711882319F308
:102620008092460290924702A0924802B0924902DC
:1026300040916F0A4C2B40936F0A81E0D5CF4F92A7
:102640005F926F927F928F929F92AF92BF92CF9242
:10265000DF92EF92FF920F931F93CF93DF93EC01E2
:10266000423051056105710590F480E0DF91CF9112
:102670001F910F91FF90EF90DF90CF90BF90AF90A0
:102680009F908F907F906F905F904F900895898575
:102690009A85AB85BC850196A11DB11D8417950750
:1026A000A607B70710F3CB88DC88ED88FE888F89F2
:1026B000803109F042C0BB27A72F962F852F4801F4
:1026C00059012A013B01C80ED91EEA1EFB1E80914A
:1026D000460290914702A0914802B0914902C81663
:1026E000D906EA06FB0699F58F898031C1F5B30159
:1026F000A201552766277727440F551F4B5A534F82
:10270000FA019182808280916F0A816080936F0AC2
:102710008A89823080F08D819E81AF81B8858C0D51
:102720009D1DAE1DBF1D8093700A9093710AA093EA
:10273000720AB093730A81E099CFDB01CA01E7E026
:10274000B695A79597958795EA95D1F7B8CF40E0CC
:10275000C701B6010E94D6128111C6CF86CFB30140
:10276000A2014F77552766277727440F551F440F3F
:10277000551F4B5A534FFA0180829182A282B38235
:10278000C2CF8F929F92AF92BF92CF92DF92EF9281
:10279000FF920F931F93CF93DF93FC018185928566
:1027A000A385B4850196A11DB11D84179507A607C1
:1027B000B70770F480E0DF91CF911F910F91FF90E8
:1027C000EF90DF90CF90BF90AF909F908F90089543
:1027D00083889488A588B6888789803189F5BB2746
:1027E000A72F962F852FE9016A017B018F01BC017C
:1027F000CD01680D791D8A1D9B1D80904602909029
:102800004702A0904802B090490286169706A80693
:10281000B90601F5F8018789803111F5DD24EE2430
:10282000FF24F601EE0FFF1FEB5AF34F80819181D9
:10283000B0E0A0E088839983AA83BB8381E0BBCF0B
:10284000DB01CA01C7E0B695A79597958795CA950C
:10285000D1F7C9CF40E00E94D6128111DBCFAACFB9
:10286000E894C7F8DD24EE24FF24F601EE0FFF1FE5
:10287000EE0FFF1FEB5AF34F80819181A281B3814C
:10288000BF70D8CF4F925F926F927F92AF92BF92FC
:10289000CF92DF92EF92FF920F931F93CF93DF932C
:1028A00000D01F92CDB7DEB78C0149835A836B836A
:1028B0007C835901C12CD12C7601412C82E0582E09
:1028C000612C712C49815A816B817C819E012F5F23
:1028D0003F4FC8010E94C113882339F1F801858553
:1028E000A301920104C0220F331F441F551F8A9574
:1028F000D2F7DA01C901C80ED91EEA1EFB1E4981B2
:102900005A816B817C818789803111F188EF9FEF3B
:10291000AFEFBFE0481759076A077B0798F2F50148
:10292000C082D182E282F38281E00F900F900F90FB
:102930000F90DF91CF911F910F91FF90EF90DF905B
:10294000CF90BF90AF907F906F905F904F90089521
:1029500088EF9FEFA0E0B0E0DDCFCF92DF92EF9263
:10296000FF921F93CF93DF93EC0180E2689FF00109
:102970001124EB5AF34F9385917161F0842F827487
:1029800049F080E0DF91CF911F91FF90EF90DF90B1
:10299000CF900895142F6A8B809146029091470240
:1029A000A0914802B09149028E879F87A88BB98B6E
:1029B000C488D588F12CE12C7601DD24CC24CF8A83
:1029C000D88EE98EFA8E828D938DB0E0A0E0AC01B6
:1029D000BD014C295D296E297F294F8B588F698F46
:1029E0007A8F83858871B1F4848D958DA68DB78D8E
:1029F0008B8B9C8BAD8BBE8B81E08D831F701C837A
:102A00001E821F82188619861A861B861C861D86C2
:102A100081E0B8CF803109F0B4CF9E012D5E3F4FE9
:102A20008B8D9C8D0E944214882309F4AACF84E0E8
:102A3000E4CF8F929F92AF92BF92CF92DF92EF92AC
:102A4000FF920F931F93CF93DF93EC018D81811140
:102A50000EC080E0DF91CF911F910F91FF90EF901A
:102A6000DF90CF90BF90AF909F908F9008950B898B
:102A70001C892D893E89041715072607370748F357
:102A80004A015B01823031F48A869B86AC86BD8622
:102A900081E0E0CF81149104A104B10449F41E82C5
:102AA0001F82188619861A861B861C861D86F0CF03
:102AB0000A851B852C853D85EB8DFC8D858590E0F9
:102AC0000996B901A8014150510961097109082EFF
:102AD00004C076956795579547950A94D2F7750186
:102AE0006401E1E0CE1AD108E108F10804C0F694CF
:102AF000E794D794C7948A95D2F7C416D506E6060C
:102B0000F70620F0012B022B032B11F58F89988DEE
:102B1000A98DBA8D8E839F83A887B9878E010A5F9E
:102B20001F4FC114D104E104F10409F4ADCF4E816B
:102B30005F816885798598018B8D9C8D0E94C1137A
:102B400091E0C91AD108E108F1088111EACF81CFDB
:102B5000C41AD50AE60AF70AE1CF3F924F925F9274
:102B60006F927F928F929F92AF92BF92CF92DF929D
:102B7000EF92FF920F931F93CF93DF93CDB7DEB702
:102B80002C970FB6F894DEBF0FBECDBF5C01DC0101
:102B90005B968D909C905C9716964D905D906D9095
:102BA0007C901997411451046104710409F468C0C0
:102BB000BFEF4B1A5B0A6B0A7B0A312CF40181854B
:102BC0009285A385B4859C01AD012F5F3F4F4F4F88
:102BD0005F4F29873A874B875C87730162011D82AB
:102BE0001E821F821886F40181859285A385B48593
:102BF0002D813E814F815885281739074A075B0789
:102C000008F056C089859A85AB85BC858C159D05D5
:102C1000AE05BF0550F482E0C82ED12CE12CF12C7A
:102C200092E0492E512C612C712C9E012F5F3F4F59
:102C3000B701A601C4010E94C1138823C9F189818B
:102C40009A81AB81BC81892B8A2B8B2B09F12601C0
:102C500037019FEF491A590A690A790A2D813E8185
:102C60004F8158852F5F3F4F4F4F5F4F2D833E83DE
:102C70004F8358873FEFC31AD30AE30AF30AB3CF4F
:102C8000F40140805180628073803324339496CF66
:102C9000C414D504E604F70409F70FEF1FEF2FEF74
:102CA0003FE0B701A601C4010E941F13811119C0A2
:102CB00080E02C960FB6F894DEBF0FBECDBFDF913B
:102CC000CF911F910F91FF90EF90DF90CF90BF9029
:102CD000AF909F908F907F906F905F904F903F90BC
:102CE0000895F5014681578160857185411551052B
:102CF0006105710539F097018601C4010E941F1317
:102D00008823B1F2D5011696CD92DD92ED92FC9218
:102D10001997332051F0D701C6010196A11DB11DAD
:102D2000F40180839183A283B383F5018789908D19
:102D3000A18DB28D892B8A2B8B2B39F4C78AD08E2B
:102D4000E18EF28E84818068848381E0B2CF2F92FD
:102D50003F924F925F926F927F928F929F92AF922B
:102D6000BF92CF92DF92EF92FF920F931F93CF9378
:102D7000DF93EC015B012A018D81811115C08FEF7A
:102D80009FEFDF91CF911F910F91FF90EF90DF9018
:102D9000CF90BF90AF909F908F907F906F905F90FB
:102DA0004F903F902F9008958C8180FFE8CF0B8942
:102DB0001C892D893E894A855B856C857D85C2018C
:102DC000B0E0A0E068017901C41AD50AE60AF70A62
:102DD000C816D906EA06FB0618F42801441A550A53
:102DE00042011E0126E0220E311C8114910409F4D7
:102DF000B3C04A855B856C857D856A0181E0D822F8
:102E00008B8D9C8D8A019B01E9E03695279517955E
:102E10000795EA95D1F7ED81E230E1F5FC01628D8D
:102E2000738D848D958D600F711F821F931F612C90
:102E300022E0722E6C187D088614970408F4340181
:102E40002C8126FD04C06114F2E07F0671F400912C
:102E5000460210914702209148023091490206171C
:102E600017072807390709F053C040E00E94D6121F
:102E7000882309F484CFC6018B5A934FD5019C0156
:102E8000260D371DFC012E173F0709F460C0419144
:102E90004D93F9CFFC0174807A947022C114D1044F
:102EA00071F471100CC0452B462B472B39F58F89D7
:102EB000988DA98DBA8D8E839F83A887B987EB8D56
:102EC000FC8D6E817F8188859985625071098109A9
:102ED0009109258504C0660F771F881F991F2A95C1
:102EE000D2F70685178520893189600F711F821FEF
:102EF000931F670D711D811D911D99CF4E815F81BB
:102F00006885798591010E94C1138111D8CF37CF8F
:102F1000750183019601AB01BC0180913B0C90913E
:102F20003C0C0E948711882309F429CFA60CB71CFA
:102F30008A859B85AC85BD85860D971DA11DB11D1C
:102F40008A879B87AC87BD87861897084ECF281B3A
:102F5000390BA20EB31EECCFC20113CFCF93DF9378
:102F60001F92CDB7DEB741E050E0BE016F5F7F4FEB
:102F70000E94A716019731F4898190E00F90DF91AC
:102F8000CF9108958FEF9FEFF9CFFC01818D928D46
:102F9000009711F00C94AE178FEF9FEF08950F93E9
:102FA0001F93CF93DF93EC01898D9A8D10E000E0A1
:102FB000009799F00E94AE178C010F3F100769F03F
:102FC000898D9A8DFC0142855385648575854150B4
:102FD0005109610971090E941915C801DF91CF914A
:102FE0001F910F910895CF93DF93EC018D8188237A
:102FF00029F18C8187FF1EC0CE010E94E87CFC0174
:10300000892BE1F08D81823040F48B899C89AD89D8
:10301000BE89848F958FA68FB78F8F89988D938F58
:10302000828F8F89988DA98DBA8DB58BA48B8C8159
:103030008F778C83DF91CF910C949B1280E0DF918E
:10304000CF910895CF93DF93EC010E94F31788236B
:1030500011F01D8281E0DF91CF910895FC01818DF7
:10306000928D009711F00C94F31708953F924F92B0
:103070005F926F927F928F929F92AF92BF92CF9208
:10308000DF92EF92FF920F931F93CF93DF9300D0C5
:1030900000D000D01F921F92CDB7DEB77C01DC01BB
:1030A00015968C91811115C0FE013196CE010C96BA
:1030B0006F0130E23193E817F907E1F7DA0130E008
:1030C00087E09D91B92E992329F19E3239F48A30F7
:1030D00011F480E0D9C038E08AE0F3CFE2E8FDE007
:1030E0004491442321F031969413FACFF2CF831701
:1030F00080F34FED490F4E3560F74FE9490F4A31E4
:1031000018F440EEB42EB90EF601E30FF11DB082B3
:103110003F5FD7CF89818032E1F2322E8B01FB01F4
:10312000838D948DD7015C969C938E935B971682CA
:103130001782108611861286138614861586F8016A
:1031400082859385A485B585438954896589768967
:1031500084179507A607B70708F04DC025E0B69578
:10316000A795979587952A95D1F7F82FFF70AF2EE1
:10317000D80115968C91823008F4ABCFC8010E941B
:10318000AE1797FDA6CFF80182859385A485B585F6
:103190004F96A11DB11D82879387A487B587F0E262
:1031A000AF9EB00111246B5A734F6115710509F47C
:1031B00090CFDB018C91882341F0853E09F057C008
:1031C000BB2029F0BB24B394BACFB1100EC0F701D5
:1031D000A28A8091460290914702A0914802B09144
:1031E000490286879787A08BB18BDB018C91811177
:1031F000E9CFBB24B394832D8271823109F069CF6A
:10320000BB2009F459C0C7010E94E87C009709F46B
:1032100060CF20E2FC0111922A95E9F72BE0F6013C
:10322000DC0101900D922A95E1F721E238E2DC0100
:1032300051963C932E93509740E058E01F965C9334
:103240004E931E9753963C932E93529759963C93C8
:103250002E93589757965C934E9356970E949B12C5
:10326000882309F436CF432DF70162890AC04BE069
:1032700050E0C6010E947DB8892B09F060CF432D34
:103280006A2DC7010E94AD142B960FB6F894DEBFCD
:103290000FBECDBFDF91CF911F910F91FF90EF90A7
:1032A000DF90CF90BF90AF909F908F907F906F9066
:1032B0005F904F903F900895F8018581823009F426
:1032C00008CFC8010E94AD15882309F402CFD801A8
:1032D0005B96ED91FC915C9716968D909D90AD90CC
:1032E000BC901997B2E08B1A9108A108B1088585A6
:1032F00004C0880C991CAA1CBB1C8A95D2F7868531
:103300009785A089B189880E991EAA1EBB1E84814B
:1033100024013501480E511C611C711C8414950454
:10332000A604B70401F1E1E04E1A510861087108E2
:103330000E949B12882309F4CCCEE5E5FCE01192B3
:1033400085E59EE08E179F07D1F740924602509286
:103350004702609248027092490280916F0A816030
:1033600080936F0ADBCFD8015B96ED91FC912585A8
:1033700080E092E0A0E0B0E004C0880F991FAA1F8F
:10338000BB1F2A95D2F7F80143895489658976894C
:10339000840F951FA61FB71F838B948BA58BB68BAD
:1033A000D70152961C9285E59CE033CF1F93CF93B3
:1033B000DF93CDB7DEB76D970FB6F894DEBF0FBEC3
:1033C000CDBFAB011C821B8222E933E03A83298303
:1033D0001E8221E0BC01CE0101960E94361811E048
:1033E00081110CC010E0812F6D960FB6F894DEBFEE
:1033F0000FBECDBFDF91CF911F910895CE010196F1
:103400000E942218F0CFCF93DF93CDB7DEB76D9730
:103410000FB6F894DEBF0FBECDBF442391F1AB01D0
:10342000BC011C821B8282E993E09A8389831E82FD
:1034300022E0CE0101960E94361881110EC090E064
:1034400081E0911101C080E06D960FB6F894DEBF67
:103450000FBECDBFDF91CF910895CE0101960E949E
:10346000017D882361F3CE0101960E94E87C0097DC
:1034700031F325EEFC0120831E820E949B12982FBF
:10348000DFCF81E0E1CF2F923F924F925F926F9218
:103490007F928F929F92AF92BF92CF92DF92EF92E4
:1034A000FF920F931F93CF93DF9300D01F92CDB75E
:1034B000DEB78C015B011A01DC0115968C91159722
:1034C000813009F0C8C014968C9181FFC4C082FD80
:1034D000AEC06101D8011A964D915D916D917C91BC
:1034E0001D97C114D10409F429C15B968D919C915B
:1034F0005C97FC0174802FEF270D2A013B0139E016
:1035000076946794579447943A95D1F7722E742025
:103510007A01F1E0FF22711020C0E114F104E9F416
:1035200016964D915D916D917C91199741155105BC
:103530006105710509F098C057968D919D910D9088
:10354000BC91A02D0097A105B10509F0AFC0C8013D
:103550000E94AD15882309F47EC080E092E08E19A8
:103560009F0946018C159D0508F44C01D8015B9616
:103570004D915C915C9716968D919D910D90BC91AB
:10358000A02D0297A109B109FA01258504C0880F71
:10359000991FAA1FBB1F2A95D2F7468557856089B8
:1035A0007189840F951FA61FB71F9C01AD01270DC0
:1035B000311D411D511D29013A01811432E093064C
:1035C00009F07AC08091460290914702A09148028A
:1035D000B091490284159505A605B70559F48FEFFA
:1035E0009FEFDC018093460290934702A09348022C
:1035F000B09349029501B301A20180913B0C9091D7
:103600003C0C0E942E12882331F19EEFB91AC81883
:10361000D908F80182859385A485B585880D991D03
:10362000A11DB11D82879387A487B58753CFF80169
:10363000438954896589768982859385A485B58572
:10364000481759076A077B0709F443CFC8010E944E
:10365000191581113ECF81E090E0D80113969C931B
:103660008E93129780E007C09E012F5F3F4F0E940C
:10367000C113811102C090E077C089819A81AB812A
:10368000BC81F801238D348DF901278948EF5FEF64
:1036900060E070E0203121F048EF5FEF6FEF7FE0F6
:1036A00084179507A607B70708F051CFF80186835E
:1036B0009783A087B18751CFE114F10491F5D80128
:1036C0001A964D915D916D917C911D9753968D91B8
:1036D0009D910D90BC91A02D481759076A077B0753
:1036E00000F10E949B12882309F4B5CF4092460254
:1036F00050924702609248027092490280916F0A8C
:10370000816080936F0A97012B5A334FD501C9010D
:10371000880D991DF9018E179F0759F04D9141931E
:10372000FACF41E0C301B2010E94D6128111EBCF62
:1037300092CF821B930BA80EB91E69CFF801838923
:103740009489A589B68984179507A607B70738F421
:103750008481438B548B658B768B80688483F801DE
:10376000848183FD18C0C1010F900F900F900F90BE
:10377000DF91CF911F910F91FF90EF90DF90CF904D
:10378000BF90AF909F908F907F906F905F904F9081
:103790003F902F900895C8010E94F317882309F4E1
:1037A0005ACFE1CFCF93DF931F92CDB7DEB76983B6
:1037B00041E050E0BE016F5F7F4F0E94431A0F90BF
:1037C000DF91CF910895CF93DF93EC01E98DFA8DCE
:1037D000309749F481E090E09B838A8390E080E019
:1037E000DF91CF91089513821282898D9A8D0E9464
:1037F000431AE98DFA8D22813381232B59F7F0CFBB
:10380000FC01DB0112968D919C9113979383828327
:1038100082E993E09183808314968C91149784833A
:1038200015968C911597858316964D915D916D91A6
:103830007C91199746835783608771871A964D91BB
:103840005D916D917C911D97428753876487758741
:103850001E964D915D916D917C915197468757874A
:10386000608B718B52968C915297828B53964D91AF
:103870005D916D917C915697438B548B658B768BC4
:1038800057964D915D916D917C915A97478B508FD2
:10389000618F728F5B968D919C91948F838F089529
:1038A000DC015996ED91FC91309721F081E09581F2
:1038B000911101C080E00895CF93DF93EC01898DD1
:1038C0009A8D009741F00E942218898D9A8D0E944E
:1038D00006B71A8E198EDF91CF910895EF92FF925D
:1038E0000F931F93CF93DF93EC017B018A011B821F
:1038F0001A8288EE93E0A0E0B0E08C839D83AE83D3
:10390000BF8382E194E0998388838DE190E00E94F7
:103910006AB69A8F898F009779F02DE1F701DC0163
:1039200001900D922A95E1F74CE050E0B801CE01EC
:103930000C960E94D5B8188EDF91CF911F910F91F0
:10394000FF90EF900895E0913E0CF0913F0C808144
:1039500090913D0C892B80830895AF92BF92CF92B6
:10396000DF92EF92FF920F931F93CF93DF9300D0DC
:103970001F92CDB7DEB78C016B017A018091400CAC
:103980008333E9F45B016801C40ED51EC016D1066D
:10399000A9F10E94800B8FE00E948B0B812F0E9467
:1039A0008B0B802F0E948B0B0F5F1F4F80E00E94BC
:1039B0008B0BF50181935F010E94A31CE7CF843339
:1039C00069F50E94800B19830A838F2D8F778B8373
:1039D000EC8264E070E0CE0101960E94660BA701C4
:1039E00070E060E0C6010E94A5B8E114F10421F086
:1039F000B701C6010E94660B0E94A31CC7010F906D
:103A00000F900F900F90DF91CF911F910F91FF902A
:103A1000EF90DF90CF90BF90AF9008950E94800B01
:103A20000F3F110509F030F419820A831B8263E00D
:103A300070E0D1CF17FD0BC019820A8333E01695D1
:103A400007953A95E1F7007E08600B83F0CFC80137
:103A500026E0969587952A95E1F7807E19830A835B
:103A60000115104C18F480618B83E1CF8861FCCF85
:103A7000CF93DF931F92CDB7DEB72091410C30E09A
:103A8000322F2227260F371F90E0982F882741E0FA
:103A900050E0BE016F5F7F4F820F931F0E94AD1CED
:103AA00089810F90DF91CF910895AF92BF92CF920D
:103AB000DF92EF92FF920F931F93CF93DF9300D08B
:103AC00000D01F921F92CDB7DEB78C017B016A0137
:103AD0008091400C8333E1F45801A40EB51EA0166A
:103AE000B10609F46FC00E94800B80EF0E948B0B1F
:103AF000812F0E948B0B802F0E948B0B0F5F1F4F1B
:103B0000F70181917F010E948B0B0E94A31CE7CFDC
:103B10005B01A40EB51E8433C1F40E94800B19838F
:103B20000A838D2D80688B83CC8264E070E0CE01A7
:103B300001960E94660BAE14BF0409F441C0F70160
:103B400081917F010E948B0BF6CF0E94800B0F3F6B
:103B5000110509F028F419820A8384E08B830CC0D4
:103B600017FD17C019820A8333E0169507953A9519
:103B7000E1F7007E0C600B8386E0C816D104A0F547
:103B8000F701DE011496EA15FB0599F081918D93FA
:103B9000FACFC80126E0969587952A95E1F7807EB1
:103BA00019830A830115104C10F48461D7CF8C61FE
:103BB000D5CFB6016D5F7F4FCE0101960E94660B97
:103BC0000E94A31CC60128960FB6F894DEBF0FBE54
:103BD000CDBFDF91CF911F910F91FF90EF90DF90BC
:103BE000CF90BF90AF90089563E070E0CE01019652
:103BF0000E94660BF70181917F010E948B0BAE142E
:103C0000BF04C1F7DDCFCF93DF931F92CDB7DEB7EF
:103C100041E050E0BE016F5F7F4F90E080E00E9486
:103C2000AD1C89810F90DF91CF910895CF93DF93E1
:103C3000C4E1D0E00E94031E882361F061E070E0DF
:103C400080E090E00E945E0D2197A1F780E0DF9177
:103C5000CF91089581E0FBCFCF93DF931F92CDB733
:103C6000DEB7898341E050E0BE016F5F7F4F90E097
:103C700080E00E94551D0F90DF91CF91089563E081
:103C800070E00C94381DDA01E091410CF0E0FE2F59
:103C9000EE27E60FF71F90E0982F8827A901BD01B6
:103CA0008E0F9F1F0C94551DCF93DF931F921F9271
:103CB000CDB7DEB779836A8322E030E0AE014F5F93
:103CC0005F4F60E170E00E94431E0F900F90DF9104
:103CD000CF910895CF93DF931F921F92CDB7DEB798
:103CE00079836A8322E030E0AE014F5F5F4F64E08A
:103CF00070E00E94431E0F900F90DF91CF910895C6
:103D0000CF93DF931F92CDB7DEB72091410C30E007
:103D1000322F2227260F371F90E0982F88274983BC
:103D200041E050E0BE016F5F7F4F820F931F0E9402
:103D3000551D0F90DF91CF910895CF93C82F462F37
:103D400061E070E00E94801E61E070E08C2F0E94B4
:103D5000381D8111F9CFCF910895DA01E091410C1E
:103D6000F0E0FE2FEE27E60FF71F90E0982F882750
:103D7000A901BD018E0F9F1F0C94AD1C6F927F9205
:103D80009F92AF92BF92CF92DF92EF92FF920F93EA
:103D90001F93CF93DF931F921F92CDB7DEB7982E5C
:103DA0008B013A01690122E030E0AE014F5F5F4FC5
:103DB00064E270E00E94AD1EE980FA80FE24EF24E8
:103DC000FE24E00EF11E970137704091400C092D42
:103DD00010E0C801433309F04CC00896982F88279B
:103DE000990F990F990F820F931F473309F446C01B
:103DF000A9014C0D5D1D4130584008F43FC060E002
:103E000078E05B01A21AB30AA501B3010E94551D17
:103E1000A6014A195B09B3016A0D7B1D8091400C14
:103E2000833349F5085F1F4F000F000F000F80E03C
:103E3000902F0E94551DEC0CFD1CF982EA8222E0B5
:103E400030E0AE014F5F5F4F64E270E0892D0E9469
:103E5000431E0F900F90DF91CF911F910F91FF9014
:103E6000EF90DF90CF90BF90AF909F907F906F903A
:103E700008954096B3CF005F1F4FD6CFA601B30180
:103E8000D8CFEF92FF921F93CF93DF931F921F9291
:103E9000CDB7DEB7182F22E030E0AE014F5F5F4FA5
:103EA00060E270E00E94AD1EE980FA80FE24EF24FB
:103EB000FE2422E030E0AE014F5F5F4F60E270E031
:103EC000812F0E94AD1E89819A8198278927982782
:103ED000E816F90689F487E0189FF0011124E351F0
:103EE000F44FF582E482C7010F900F90DF91CF91DC
:103EF0001F91FF90EF9008957C01DBCFFF920F930D
:103F00001F93CF93DF931F921F92CDB7DEB7F82E8A
:103F100022E030E0AE014F5F5F4F66E270E00E944A
:103F2000AD1E09811A8110270127102722E030E0F9
:103F3000AE014F5F5F4F66E270E08F2D0E94AD1EB5
:103F400089819A819827892798270817190749F4A2
:103F5000C8010F900F90DF91CF911F910F91FF90AB
:103F600008958C01E3CF44E050E0BC018FE090E085
:103F70000C94551D08951F93CF93DF93182F80E560
:103F800091E00E94807A812F0E94411FEC01812FD5
:103F90000E943F1E873121F08C3111F0D0E0C0E04B
:103FA000CE01DF91CF911F910895FC018485883067
:103FB00010F40C94BB1F90E080E00895CF92DF9244
:103FC000EF92FF921F93CF93DF93182F7B01EA01AB
:103FD0004130584010F0C0E0D8E080E591E00E9408
:103FE000807A812F0E94411F6C01812F0E943F1E09
:103FF000873111F08C3121F5CC16DD0670F380E5A8
:1040000091E00E94807A9E01A70170E060E0812F1C
:104010000E94BE1E60E270E0812F0E949D1E62E041
:1040200070E0812F0E94381D84FD0DC0812F0E94F9
:104030003F1E8823B9F080E591E00E94807AEFCF9F
:10404000D0E0C0E0DCCF40E162E070E0812F0E9470
:10405000801ECE01DF91CF911F91FF90EF90DF90F6
:10406000CF900895D0E0C0E0F4CF0F931F93CF938B
:10407000DF938C01EA01FC018485883048F40E94BA
:10408000DE1F892B39F481E090E0F801938382836D
:10409000D0E0C0E0CE01DF91CF911F910F91089544
:1040A000CF92DF92EF92FF920F931F93CF93DF9304
:1040B0008B017A016C0129EBC20ED11CF601408103
:1040C000EC012A96442349F050E0BC0167567F4F2B
:1040D000CE010E943520F6011082A701B801CE0161
:1040E000DF91CF911F910F91FF90EF90DF90CF90D4
:1040F0000C943520CF93DF93EC01C754DF4FE88158
:1041000021E02E0F2883E80FF92FF11DE756FF4F0E
:104110006083203249F4BC0167567F4F40E250E093
:104120000A960E943520188281E090E0DF91CF91BD
:1041300008951F93CF93DF931F92CDB7DEB7182F4B
:1041400080E591E00E94807A812F0E94920B27E007
:10415000129FF0011124E351F44F22813381377013
:1041600041E050E0BE016F5F7F4F820F931F0E94BE
:10417000AD1C89810F90DF91CF911F910895FC01B3
:10418000808D883040F4218D328D232B21F00E94C8
:10419000992090E008958FEF9FEF0895CF93DF93DC
:1041A000FC012485283028F08FEF9FEFDF91CF911D
:1041B0000895EC010190F081E02D0084F185E02D5F
:1041C0001995892B89F38C850E94992090E0EECF78
:1041D0001F93CF93DF93182F87E0189FE0011124DE
:1041E000C351D44F88819981009761F480E591E0B3
:1041F0000E94807A812F0E947E1F2E81821B91094E
:1042000099838883DF91CF911F910895FC01848564
:10421000883010F40C94E82090E080E008954F92EC
:104220005F927F928F929F92AF92BF92CF92DF92D6
:10423000EF92FF920F931F93CF93DF931F921F92E2
:10424000CDB7DEB7782E6B014A01A82EB12C27E03E
:10425000829FC0011124FC01E351F44F7F010081D2
:10426000118180E591E00E94807A0815190554F4C7
:10427000872D0E947E1FF70126818C01021B1109E8
:10428000118300830115110519F5872D0E943F1E2A
:10429000843159F0882349F001E010E08C3111F4A9
:1042A00010E000E0119501951109C8010F900F90E1
:1042B000DF91CF911F910F91FF90EF90DF90CF9002
:1042C000BF90AF909F908F907F905F904F90089598
:1042D000801691060CF4840187E08A9DF0018B9D85
:1042E000F00D1124E351F44FE280F380C114D104A6
:1042F00051F12701F7E05F22872D0E94920B840D78
:10430000951D2091400C273309F453C09801240DCA
:10431000351D2130384008F44CC020E038E0490118
:1043200084189508A401B6010E94AD1C2601480C12
:10433000591C6801C818D908872D0E94920BA60144
:10434000B2010E94AD1CE00EF11E87E08A9DF001D3
:104350008B9DF00D1124E351F44FF382E282208112
:104360003181201B310B318320838681800F912F77
:10437000911D8A3F910510F4232BF1F487E08A9D6B
:10438000F0018B9DF00D1124E351F44F1682F98258
:10439000EA8222E030E0AE014F5F5F4F68E270E0FA
:1043A000872D0E94431E60E470E0872D0E949D1EB1
:1043B0007CCFA801B601C5CF868377CFCF93DF939B
:1043C000FC01218D328D2115310529F48FEF9FEFEE
:1043D000DF91CF910895EC01808D4217530708F0CB
:1043E000A9010E940F211816190684F7298D3A8D0C
:1043F000281B390B3A8F298FEBCF0F931F93CF9345
:10440000DF931F92CDB7DEB7FC01218D328D232BB8
:1044100041F48FEF9FEF0F90DF91CF911F910F919C
:1044200008958C0141E050E0BE016F5F7F4FFC01B9
:10443000808D0E940F21181619065CF7F801818DF6
:10444000928D0197928F818F898190E0E4CF0F93B5
:104450001F93CF93DF9300D000D01F921F92CDB750
:10446000DEB78C01D80159964D915C915A97411550
:10447000510551F0ED91FC91048CF58DE02D70E02B
:1044800060E0C8011995EECFF801808D0E94E82008
:10449000892BB1F148E050E0BE016F5F7F4FD8013A
:1044A00058968C910E940F2118161906F4F4D80121
:1044B000509684E0FE01319601900D928A95E1F7C5
:1044C0008D8190E0982F88272E81820F911DF80111
:1044D000958B848B8F81282F30E0322F222788857F
:1044E000820F932F911D928F818F28960FB6F8948B
:1044F000DEBF0FBECDBFDF91CF911F910F91089509
:1045000090E080E0F2CFCF93DF931F92CDB7DEB77C
:1045100041E050E0BE016F5F7F4FFC0184850E9447
:104520000F211816190634F4898190E00F90DF915D
:10453000CF9108958FEF9FEFF9CFFC0184858830EC
:1045400010F40C940F2190E080E00895CF93C82FD1
:1045500080E591E00E94807A68E070E08C2FCF9136
:104560000C949D1ECF93C82F80E591E00E94807A25
:1045700060E170E08C2FCF910C949D1ECF92DF9262
:10458000EF92FF920F931F93CF93DF9300D000D051
:10459000CDB7DEB78C016B017A01FC01808D8830CC
:1045A00010F40E94B22280E394E09A838983F6019A
:1045B00082819381A481B5818B839C83AD83BE83EB
:1045C000B701CE0101960E94DC80F801808F88300F
:1045D000A0F4F586E486128E118E81E026960FB641
:1045E000F894DEBF0FBECDBFDF91CF911F910F9129
:1045F000FF90EF90DF90CF90089580E0EFCFCF93C2
:10460000DF93EC01888D883020F40E94B22288E08C
:10461000888FDF91CF910895CF93C82F80E591E0E7
:104620000E94807A8C2FCF910C943F1EEF92FF92C4
:104630000F931F93CF93DF937C018091400CD4E0C4
:10464000833309F0D8E005E21CE0C0E0F8012191D5
:1046500031918F01F701848195812817390729F05D
:10466000CF5FDC13F3CF80E006C08C2F0E940C23B9
:104670008431B1F781E0DF91CF911F910F91FF90CD
:10468000EF9008959F92AF92BF92CF92DF92EF92F8
:10469000FF920F931F93CF93DF93EC017B018091E7
:1046A000400C811121C01B821A8288EE93E0A0E0A9
:1046B000B0E08C839D83AE83BF8384EE93E09983C7
:1046C000888388E08C8788EE93E09E878D87CE0173
:1046D000DF91CF911F910F91FF90EF90DF90CF90DE
:1046E000BF90AF909F90089534E0932E833311F0E4
:1046F00028E0922E85E2C82E8CE0D82E10E098E0BB
:10470000B92EA12CD6012D913D916D01F701848127
:1047100095812817390791F4812F0E940C23082FC7
:10472000873111F08C3139F5812F0E94E820892BD7
:1047300059F50C3119F4812F0E94A6221F5F9112A6
:10474000E1CFA11008C0D701ED91FC910084F18563
:10475000E02DC70119951B821A8288EE93E0A0E034
:10476000B0E08C839D83AE83BF8384EE93E0998316
:104770008883BC86A8CF843149F08111DFCFF60150
:10478000329711821082DACFB12ED8CFAA24A39407
:10479000D5CF8F929F92AF92BF92CF92DF92EF923E
:1047A000FF920F931F93CF93DF93CDB7DEB72F9771
:1047B0000FB6F894DEBF0FBECDBF5C014B017A018E
:1047C0008091400C8823C9F104E0833309F008E0AC
:1047D000B501CE0101960E94422385E2C82E8CE0ED
:1047E000D82E10E0F601219131916F01F5018481FD
:1047F00095812817390751F4812F0E940C238731A6
:1048000029F4A701B401812F0E94DE1F1F5F01134D
:10481000E9CFC7012F960FB6F894DEBF0FBECDBF0C
:10482000DF91CF911F910F91FF90EF90DF90CF908C
:10483000BF90AF909F908F900895F12CE12CE9CF1D
:10484000CF93DF93EC018C858830D0F40E940C2349
:10485000843189F0882379F0883169F021E08C3146
:1048600059F4E881F9810084F185E02DCE01199594
:1048700021E0892B09F420E0822FDF91CF91089568
:1048800080E0FBCFCF92DF92EF92FF92CF93DF9346
:10489000EC018C85883068F40E94A6220E94910D5C
:1048A0006B017C018C850E940C23811109C088E07A
:1048B0008C87DF91CF91FF90EF90DF90CF9008959C
:1048C00061E070E080E090E00E945E0D0E94910D3A
:1048D000AB01BC014C195D096E097F098D859E8570
:1048E000B0E0A0E0481759076A077B07D8F28C852B
:1048F0000E94B222DCCFCF93DF93EC018C8588300D
:1049000060F40E940C23873111F08C3131F48C85D6
:104910000E94BB1F8115984088F3DF91CF910895C5
:10492000CF92DF92EF92FF920F931F93CF93DF937B
:10493000CDB7DEB7AF970FB6F894DEBF0FBECDBFD1
:104940008C016B017A0180E394E09A8389831B8256
:104950001C821D821E821C861B8648EE53E060E08E
:1049600070E04D875E876F87788B2AEB33E03A875C
:104970002987988F8F8B198E1A8E1B8E1C8E28E09C
:1049800029A39BA78AA71CA61DA61EA61FA6D80101
:104990001C968C91883060F40E940C23882321F0AF
:1049A000F80184850E94A62288E0D8011C968C9389
:1049B00080913B1090913C10A0913D10B0913E1021
:1049C0008EA39FA3A8A7B9A78B839C83AD83BE8327
:1049D00018861F82AE01465D5F4FB601CE0101967B
:1049E0000E94937D0097C1F0D801ED91FC9106845F
:1049F000F785E02D80E394E09DA38CA38CA59DA575
:104A0000AEA5BFA58EA39FA3A8A7B9A7A701BE0166
:104A10006C5D7F4FC8011995AF960FB6F894DEBF55
:104A20000FBECDBFDF91CF911F910F91FF90EF90FF
:104A3000DF90CF9008958F929F92AF92BF92CF92C6
:104A4000DF92EF92FF920F931F93CF93DF9300D0EB
:104A500000D000D01F92CDB7DEB79091400C9111DD
:104A600015C018E0812F2A960FB6F894DEBF0FBE4E
:104A7000CDBFDF91CF911F910F91FF90EF90DF900D
:104A8000CF90BF90AF909F908F90089528E0F22E26
:104A9000933311F494E0F92E6B01082F80E591E037
:104AA0000E94807A9E012F5F3F4F5901490110E01B
:104AB000812F0E943F1EF40181934F018823C1F092
:104AC0001F5FF112F5CFF12CF50191915F019D313E
:104AD00049F0983139F09A51923020F0F3941F1137
:104AE000F3CFBFCF60E170E08F2D0E949D1E1F2D80
:104AF000E12EF12CF701EE0FFF1FEB5DF34F11825A
:104B0000108283EE93E00197F1F7402F70E060E0B0
:104B1000812F0E94801E4FEF62E070E0812F0E9483
:104B2000801EB601CD2889F4809190029091910267
:104B300001968115F0EC9F0798F190939102809374
:104B400090026091900270919102812F0E946A1EE2
:104B500061E070E0812F0E949D1E27E02E9DC00124
:104B60002F9D900D11249C012351344F7901F9019F
:104B70001182108222E030E0AE01475F5F4F68E2B1
:104B800070E0812F0E94AD1E89859A85982789271C
:104B90009827F7019383828316821582148262CF4D
:104BA00080E090ECCACF0F931F93CF93DF93EC017B
:104BB0008B01888D883010F40E94B222B80182E007
:104BC0000E941B25888F883050F41D870C871A8E11
:104BD000198E81E0DF91CF911F910F91089580E0B0
:104BE000F9CF9F92AF92BF92CF92DF92EF92FF9256
:104BF0000F931F93CF93DF938C015B01942EE52ECF
:104C0000FC01C688D788F08C80E591E00E94807A0C
:104C10008F2D0E94411FC92DDE2D8C179D0708F492
:104C2000EC019E01A501B6018F2D0E94BE1EF80168
:104C3000868997898C0F9D1F978B868BCE01DF917C
:104C4000CF911F910F91FF90EF90DF90CF90BF9089
:104C5000AF909F900895CF93FC01C08D80E591E0C7
:104C60000E94807A60E270E08C2F0E949D1E62E0BC
:104C700070E08C2F0E94381D84FD16C062E070E049
:104C80008C2F0E94381D83FF0AC048E162E070E06B
:104C90008C2F0E94801E80E090E0CF91089580E5E7
:104CA00091E00E94807AE3CF40E162E070E08C2FD7
:104CB0000E94801E81E0F0CFFF920F931F93CF934D
:104CC000DF93EB01FC01178A168A2A81211109C0A2
:104CD0002B81211106C02C81211103C02D8122239B
:104CE00001F141155105E9F08A01FC01F08C80E5E4
:104CF00091E00E94807AAE014E5F5F4F24E030E089
:104D00006CE070E08F2D0E94431EB8018F2D0E9431
:104D1000541E81E090E0DF91CF911F910F91FF90A1
:104D2000089580E0F7CF7F928F929F92AF92BF92CB
:104D3000CF92DF92EF92FF920F931F93CF93DF9367
:104D4000CDB7DEB7A6970FB6F894DEBF0FBECDBFC6
:104D50008C01762E942E852E20E2A22ECE01019675
:104D60007C01DC01EA2D1D92EA95E9F76801F3E484
:104D7000CF0ED11C80E394E09AA389A38FEF8BA37D
:104D80008CA38DA38EA343E450E0BE016F5D7F4FE3
:104D9000C6010E945C26019609F4BFC081E08983A8
:104DA0008A8386E0B82EBB821C82D80114966D914E
:104DB0007D918D919C9117970E944FB66D837E8354
:104DC0008F83988789869A8680E890E09C878B8776
:104DD0004CE150E0B701C6010E94F125FE01379673
:104DE0008AE1DF011D928A95E9F74801B8E08B0E50
:104DF000911CF401D70101900D92BA94E1F740E1C2
:104E000050E0B701C6010E94F125F7011192AA9462
:104E1000E9F796E0A92EB12C40E250E0B701C601B7
:104E20000E94F125F1E0AF1AB108B1F783E689835A
:104E300092E89A8393E59B838C8385E38D8381E05D
:104E40008E837F829DE3988797E099878A8786E0A3
:104E5000F401DE011B9601900D928A95E1F78CE03A
:104E6000898B8A8B62E374E0CE0143960E94C0B8BE
:104E7000D8011B966C91CE0149960E941980F801C9
:104E80006485CE014B960E941980D8011D966C91C5
:104E9000CE014D960E9419804EE150E0B701C60147
:104EA0000E94F125B3E07B121EC082E3898384E077
:104EB0008A83F80196859B8397859C8390899D833F
:104EC00091899E8396E39F838887828D8987838DCE
:104ED0008A87848D8B87858D8C874CE050E0B70165
:104EE000C6010E94F12587E3898386E08A8391E0E9
:104EF0009B8393E09C838D838FE08E838AE38F83F3
:104F00008BE388878FEF898749E050E0B701C601BE
:104F10000E94F125C6010E942B26A6960FB6F89492
:104F2000DEBF0FBECDBFDF91CF911F910F91FF90DC
:104F3000EF90DF90CF90BF90AF909F908F907F9039
:104F400008950F931F93CF938C01FC0164817581A9
:104F500081E20E941B25C82F8830F8F480E591E09B
:104F60000E94807A8C2F0E943F1E833131F08C2F5B
:104F7000CF911F910F910C94A62262E070E08C2FCC
:104F80000E949D1EF80184819581EC2FF0E0EE0FC8
:104F9000FF1FEB5DF34F91838083CF911F910F91A2
:104FA00008950F931F93CF93DF931F921F92CDB756
:104FB000DEB7FC0124852830E0F48C0180E591E027
:104FC0000E94807A22E030E0AE014F5F5F4F60E1E7
:104FD00070E0F80184850E94AD1E89819A8198272E
:104FE000892798270F900F90DF91CF911F910F91F4
:104FF000089590E080E0F6CF0F931F93CF93DF9357
:105000001F921F92CDB7DEB7FC0124852830E0F453
:105010008C0180E591E00E94807A22E030E0AE01D0
:105020004F5F5F4F64E070E0F80184850E94AD1E21
:1050300089819A819827892798270F900F90DF916F
:10504000CF911F910F91089590E080E0F6CFCF921D
:10505000DF92EF92FF921F93CF93DF93EC017B01DE
:105060006A018C85883048F40E940C23882319F04B
:105070008C850E94A62288E08C87F701828193812B
:10508000A481B5810097A105B10551F490E080E0BD
:10509000DF91CF911F91FF90EF90DF90CF90089517
:1050A0008F3F9F4FAF4FBF4F89F370E060E081E2C9
:1050B0000E941B25182F8C87883040F780E591E0EF
:1050C0000E94807AA7014E5F5F4F24E030E06CE0E1
:1050D00070E0812F0E94431EB601812F0E94541E52
:1050E00064E070E0812F0E949D1E0E94910D6B0173
:1050F0007C018C850E940C23873111F18C3101F1E8
:10510000882321F20E94910DAB01BC014C195D096D
:105110006E097F098D859E85B0E0A0E08417950714
:10512000A607B70738F061E070E080E090E00E94E9
:105130005E0DDFCF8C850E94B22288E08C87A6CFDF
:1051400081E090E0A5CFCF93DF93EC0180E394E082
:10515000998388831A821B821C821D8280E591E0DC
:105160000E94807ABE016E5F7F4F44E050E08FE086
:1051700090E00E94AD1CCE01DF91CF9108959F92E7
:10518000AF92BF92CF92DF92EF92FF920F931F9355
:10519000CF93DF935C017B018B01D0E0C0E0F8018D
:1051A00091908F016501CC0EDD1EC6010E948BB46B
:1051B000981621F0692DC6010E9493B42196C5333B
:1051C000F1E0DF0761F7C701DF91CF911F910F91E8
:1051D000FF90EF90DF90CF90BF90AF909F90089599
:1051E00081E08093EF028091F002882341F088E013
:1051F00080936E1360E083E693E10C940C0E0895A7
:105200008091F0028823F9F08091EF028823D9F091
:1052100081E00E94737B8BE39FE10197F1F760E0EF
:1052200080E00E94847B65EB76E083E693E10E9458
:10523000A98561E080E00E94847B65EA76E083E6F0
:1052400093E10C94A98508950F931F93CF93DF9357
:105250002091F002222309F45CC02091EF02222366
:1052600009F457C0EA018C016F3F7F4FF1F461E010
:1052700080E00E94847BB80183E693E10E948985E7
:1052800064E976E083E693E10E94A98561E0F80194
:1052900084810E94847BBE01DD0F880B990BDF9116
:1052A000CF911F910F910C945E0D0E94910DAB0157
:1052B000BC018091610990916209A0916309B0914C
:1052C00064098C599F4FAF4FBF4F84179507A607AE
:1052D000B707F8F461E080E00E94847BB80183E6C0
:1052E00093E10E94898563E876E083E693E10E947A
:1052F000A98561E0F80184810E94847B0E94910D60
:1053000060936109709362098093630990936409C3
:10531000C2CFDF91CF911F910F9108958F929F92ED
:10532000AF92BF92CF92DF92EF92FF920F931F93B3
:10533000CF93DF938C01862F0B30110509F09FC0AE
:105340009091EC12992309F0F89462E10E9402878F
:10535000EC018091EC12882309F07894209701F1F8
:1053600080E090ECA9E7B4EC8093DF129093E01218
:10537000A093E112B093E2128093E3129093E412AF
:10538000A093E512B093E612CE3F8FEFD80709F451
:10539000A9C0CF3FDC0709F462C0CCEFDFEF30C11A
:1053A000C091E712E090E8126E2D70E090E080E08E
:1053B0000E946EB32DEC3CEC4CEC5DE30E94CDB34F
:1053C0004B015C016C2F70E090E080E00E946EB3B6
:1053D0009B01AC01C501B4010E9415B56093DF12B9
:1053E0007093E0128093E1129093E212D091E9124F
:1053F000F090EA126D2F6F7770E090E080E00E94ED
:105400006EB34B015C016F2D70E090E080E00E9474
:105410006EB32DEC3CEC4CEC5DE30E94CDB39B01F4
:10542000AC01C501B4010E9415B5D7FD26C060933B
:10543000E3127093E4128093E5129093E612CE0D7E
:10544000CD0FCF0D81E090E02091EB12C21302C08E
:1054500090E080E0892B09F493C0CFEFDFEFCE011D
:10546000DF91CF911F910F91FF90EF90DF90CF9040
:10547000BF90AF909F908F9008959058D8CFCFEF66
:10548000DFEF0631110509F0BBC09091EC129923B2
:1054900009F0F89461E00E940287EC018091EC121F
:1054A000882309F07894209701F180E090ECA9E737
:1054B000B4EC8093DF129093E012A093E112B093CA
:1054C000E2128093E3129093E412A093E512B0935A
:1054D000E612CF3FDC0719F2209709F451C022965B
:1054E00009F05BCFCEEFDFEF8BC0C091E812D09117
:1054F000E7126091E7127091E81276276727762706
:1055000090E080E00E946CB32DEC3CEC4CEC5DE351
:105510000E94CDB36093DF127093E0128093E1128A
:105520009093E212E090EA12F090E9126F2D6F77FB
:10553000762F6E2D90E080E00E946CB32DEC3CEC59
:105540004CEC5DE30E94CDB3F7FC18C06093E3120E
:105550007093E4128093E5129093E6128C2F8D0FD6
:105560008E0D8F0DC1E0D0E09091EB12891302C037
:10557000D0E0C0E0D195C195D109ABCF9058E6CF2E
:10558000C090DF12D090E012E090E112F090E212B1
:1055900020E030E048EC52E4C701B6010E9429B691
:1055A000D0E0C0E0181614F4CBEFDFEF20E030E0DD
:1055B000A901C701B6010E9467B387FF02C0CAEF05
:1055C000DFEFC090E312D090E412E090E512F0908B
:1055D000E61220E030E048EC52ECC701B6010E9430
:1055E00067B387FF02C0C9EFDFEF20E030E040EF94
:1055F00052E4C701B6010E9429B618160CF483C004
:105600000C30110509F02BCF81E08093850E8CE5DD
:105610008093A70E1092860E1092A80E60E084EE82
:105620009FE00E94010B81E00E94837A0E94390D65
:105630006B017C0180917F0E811168C081E08093B5
:105640007F0E80937E0E9FEF90937D0E10927C0EC6
:1056500094E090937B0E80935A0E80915A0E886B43
:1056600080935A0E8091590E813009F028C1109212
:10567000590E0E94390D6B017C0180915A0E809366
:10568000BB008091810E9091820EA091830EB0910B
:10569000840E892B8A2B8B2BA1F00E94390D00914F
:1056A000810E1091820E2091830E3091840E6C1920
:1056B0007D098E099F09061717072807390708F47F
:1056C00046C08091BC0083FDD8CF85EC8093BC00A0
:1056D0000E94390D6B017C0180917F0E813009F4AD
:1056E000F0C080917C0E853008F00DC180917C0E59
:1056F000ABE5BEE0E4E7FAE090E0981769F12D91A0
:1057000021939F5FFACFC8EFDFEF7ACF8091810EB0
:105710009091820EA091830EB091840E892B8A2BDA
:105720008B2B09F487CF0E94390D0091810E1091C7
:10573000820E2091830E3091840E6C197D098E09A2
:105740009F09061717072807390708F073CF8091BC
:10575000800E0E948A0F80E010923A0C8093390CE0
:10576000082F10E0CEEFDFEF882309F478CECDEFDD
:10577000DFEF053011050CF472CEC4E5D9E084EEFC
:105780009FE00E94BA0A88872196CE0184559940ED
:1057900080179107A4F3C0915C0900915D09602F07
:1057A00070E090E080E00E946EB32DEC3CEC4CEC9D
:1057B0005DE30E94CDB36B017C016C2F70E090E043
:1057C00080E00E946EB39B01AC01C701B6010E944C
:1057D00015B56B017C01C0925409D0925509E09235
:1057E0005609F0925709D0915E0910915F096D2F0B
:1057F0006F7770E090E080E00E946EB34B015C0137
:10580000612F70E090E080E00E946EB32DEC3CECE4
:105810004CEC5DE30E94CDB39B01AC01C501B4012A
:105820000E9415B5D7FD71C060935809709359094E
:1058300080935A0990935B09C00FCD0FC10F8091DF
:105840006009C8130ACE20E030E048EC52E4C701FA
:10585000B6010E9429B6D0E0C0E0181614F4CBEFD0
:10586000DFEF20E030E040EA50E4C701B6010E94DB
:1058700067B387FF02C0CAEFDFEFC0905809D0902E
:105880005909E0905A09F0905B0920E030E040EFC0
:1058900051ECC701B6010E9467B387FF02C0C9EF90
:1058A000DFEF20E030E040EF52E4C701B6010E9494
:1058B00029B618160CF0D3CDC8EFDFEFD0CD85EEAA
:1058C00005CF8091810E9091820EA091830EB091B0
:1058D000840E892B8A2B8B2B09F4FECE0E94390D66
:1058E0000091810E1091820E2091830E3091840ED2
:1058F0006C197D098E099F090617170728073907B4
:1059000008F0EACE24CF85E0F3CE90588DCFCF9328
:10591000DF93FB0122813381DC0113963C932E93AC
:105920001297448155816681778114964D935D93DA
:105930006D937C9317974085518562857385189682
:105940004D935D936D937C931B971C96EF012C9662
:105950009C01275E3F4F49914D93A217B307D9F79A
:10596000218D328DFC01328F218FDF91CF910895EF
:10597000DF92EF92FF920F931F93CF93DF93D82E76
:10598000CBE4DCE07E0101E010E0F7018081F2E091
:10599000EF0EF11C61E00E94080D90E080E0013004
:1059A000110531F48091DE12881F8827881F90E04E
:1059B000880F991FFC01EF5AF34F6081F70132976E
:1059C00080810E94D48664EF71E080E090E00E94C4
:1059D0005E0D0F5F1F4F04301105B9F6DD2009F48D
:1059E00054C0EE24E394F12C81E0E816F10409F0B0
:1059F00046C08091DE128095881F8827881F90E01E
:105A00008E01880F991FFC01EF5AF34F6081888146
:105A10000E94D48668EE73E080E090E00E945E0D04
:105A200091E0E916F10471F58091DE12881F882754
:105A3000881F90E02296880F991FFC01EF5AF34FC0
:105A40006081F80180810E94D48668EE73E080E076
:105A500090E00E945E0DFFEFEF1AFF0A84E0E81667
:105A6000F10411F668EE73E080E090E0DF91CF91F1
:105A70001F910F91FF90EF90DF900C945E0D81E0ED
:105A800090E0BECF90E080E0D5CFDF91CF911F9125
:105A90000F91FF90EF90DF9008950F931F93CF9396
:105AA000DF938C01EB01FE0164912196662349F09E
:105AB000D801ED91FC910190F081E02DC80119957C
:105AC000F2CFDF91CF911F910F910895EF92FF9246
:105AD0000F931F93CF93DF93EC017B018A0168E260
:105AE00074E00E944D2D61E174E0CE010E944D2DC5
:105AF00062EE73E0CE010E944D2DB701CE010E94EF
:105B000081856DE378E0CE010E9481850115110544
:105B100021F0B801CE010E9481856DE378E0CE01CD
:105B2000DF91CF911F910F91FF90EF900C948185A1
:105B3000CF93DF93EC0167EC73E00E944D2D61E1A0
:105B400074E0CE010E944D2D69E973E0CE01DF9132
:105B5000CF910C944D2DCF93DF93EC01FB01248169
:105B600035810E948984CE01DF91CF910895EF9213
:105B7000FF920F931F93CF93DF9300D000D0CDB748
:105B8000DEB78C017B016DE574E00E9474848AE0CD
:105B9000E816F1042CF466E276E0C8010E944F8317
:105BA000B701CE0101960E94CC81BE016F5F7F4F8D
:105BB000C8010E945983CE0101960E94D583C80175
:105BC00026960FB6F894DEBF0FBECDBFDF91CF9102
:105BD0001F910F91FF90EF900895CF92DF92EF9277
:105BE000FF920F931F93CF93DF93CDB7DEB7C455CA
:105BF000D1090FB6F894DEBF0FBECDBF65965FAF7B
:105C00004EAF65972091D00B3091D10B2F5F3F4F56
:105C10003093D10B2093D00B2091EC0B2111C1C0FC
:105C20008B016C0181E08093EC0B1092D10B1092F0
:105C3000D00B6DE574E0CE01895B9F4F0E947484A8
:105C40006DE574E0CE01835B9F4F0E94748450E049
:105C500040E069E374E0C6010E94662D0130110541
:105C600009F08EC06DE574E084E791E10E94C28185
:105C70006DE574E080E591E10E94C2816596EEAD2C
:105C8000FFAD65978081882309F474C000E210E0BD
:105C90009E012F5F3F4F40E250E0BE016F5D7F4F9E
:105CA000CE018D5A9F4F0E94F57B049739F3BE01B8
:105CB0006F5D7F4FCE018F5B9F4F0E947484BE014A
:105CC0006F5B7F4FCE01895B9F4F0E949C83CE010B
:105CD0008F5B9F4F0E94D583BE016F5F7F4FCE01C8
:105CE0008F5B9F4F0E947484BE016F5B7F4FCE011C
:105CF000835B9F4F0E949C83CE018F5B9F4F0E94CE
:105D0000D5832D968EAD9FAD2D970297029730F4D7
:105D100062E574E080E591E10E94C281BE01695BA9
:105D20007F4F84E791E10E94598363968EAD9FADCA
:105D30006397892B09F4A2CF6DEB75E0CE018F5BE1
:105D40009F4F0E947484BE01635B7F4FCE018F5BC7
:105D50009F4F0E94EF826AEB75E00E94D982BC01DE
:105D600084E791E10E945983CE018F5B9F4F0E948F
:105D7000D58384CF64E771E180E591E10E94598386
:105D80001092EC0BCE01835B9F4F0E94D583CE0116
:105D9000895B9F4F0E94D5830FB6F894DEBF0FBE7C
:105DA000CDBFCC5ADF4F0FB6F894DEBF0FBECDBFCC
:105DB000DF91CF911F910F91FF90EF90DF90CF90E7
:105DC00008950F931F93CF93DF9300D000D0CDB7EA
:105DD000DEB72091CD0B2223A9F08C0165E876E097
:105DE000CE0101960E947484B801CE0101960E94F2
:105DF000EF82BC0187E49FE00E949785CE01019667
:105E00000E94D58326960FB6F894DEBF0FBECDBF95
:105E1000DF91CF911F910F9108950F931F93CF930F
:105E2000DF93CDB7DEB72C970FB6F894DEBF0FBE69
:105E3000CDBF8C010E94B80EBC01C8010E94B72DD5
:105E40000E94B00EBC01CE0107960E94B72D6FE4F0
:105E500076E0CE0101960E947484BE01695F7F4F97
:105E6000CE0101960E94EF82BC01C8010E945983B5
:105E7000CE0101960E94D583CE0107960E94D5835C
:105E80006AEB75E0C8010E944F830E94A80EBC0116
:105E9000CE0101960E94B72DBE016F5F7F4FC801F2
:105EA0000E945983CE0101960E94D58369E574E072
:105EB000C8010E944F830E94A00EBC01CE01019632
:105EC0000E94B72DBE016F5F7F4FC8010E945983AA
:105ED000CE0101960E94D58369E574E0C8010E9455
:105EE0004F830E94960EBC01CE0101960E94B72DF1
:105EF000BE016F5F7F4FC8010E945983CE0101969A
:105F00000E94D583C8012C960FB6F894DEBF0FBE51
:105F1000CDBFDF91CF911F910F9108950F931F93E4
:105F2000CF93DF93CDB7DEB72C970FB6F894DEBFD3
:105F30000FBECDBF8C010E94B80EBC01C8010E94EB
:105F4000B72D0E94B00EBC01CE0107960E94B72D5E
:105F50006FE476E0CE0101960E947484BE01695F11
:105F60007F4FCE0101960E94EF82BC01C8010E94C2
:105F70005983CE0101960E94D583CE0107960E94D7
:105F8000D5830E94500E0E9488096091AD0B70E08D
:105F9000CE0107960E94B72D6FE476E0CE01019600
:105FA0000E947484BE01695F7F4FCE0101960E94FA
:105FB000EF82BC01C8010E945983CE0101960E9464
:105FC000D583CE0107960E94D5836AEB75E0C801A0
:105FD0000E944F830E94A80EBC01CE0101960E9430
:105FE000B72DBE016F5F7F4FC8010E945983CE015C
:105FF00001960E94D58369E574E0C8010E944F8331
:106000000E94A00EBC01CE0101960E94B72DBE01D8
:106010006F5F7F4FC8010E945983CE0101960E9495
:10602000D58369E574E0C8010E944F830E94960EF3
:10603000BC01CE0101960E94B72DBE016F5F7F4F5C
:10604000C8010E945983CE0101960E94D583C801E0
:106050002C960FB6F894DEBF0FBECDBFDF91CF9167
:106060001F910F910895CF92DF92EF92FF920F93BD
:106070001F93CF93DF9300D000D0CDB7DEB77C0164
:10608000FB01848195818A01081B190B10161106EA
:106090009CF0C7010E945984C70126960FB6F89458
:1060A000DEBF0FBECDBFDF91CF911F910F91FF904B
:1060B000EF90DF90CF900895CE0101960E946B84FF
:1060C000CC24C394D12C6AEB75E0CE0101960E94DA
:1060D0004F83FFEFCF1ADF0A0C151D05A4F7BE0191
:1060E0006F5F7F4FC7010E945984CE0101960E94C5
:1060F000D583D2CF0F931F93CF93DF9300D000D0DF
:10610000CDB7DEB78C0180915E0A882329F0B801F3
:106110008AEA9EE00E9497856EE170E080E090E060
:106120000E945E0DB80187E49FE00E9497858091F0
:10613000310A882311F16AE070E080E090E00E946B
:106140005E0DB801CE0101960E946B84BE016F5FA7
:106150007F4F87E493E10E9489856EE378E087E4CE
:1061600093E10E948185CE0101960E94D58364E16E
:1061700070E080E090E00E945E0D26960FB6F894E5
:10618000DEBF0FBECDBFDF91CF911F910F9108955C
:106190000F931F93CF93DF9300D000D0CDB7DEB71E
:1061A000FC0124813581232B49F18C0180915E0A09
:1061B000882329F0BF018AEA9EE00E9489856EE16A
:1061C00070E080E090E00E945E0DB80187E49FE0FF
:1061D0000E9489858091310A882381F0B801CE011F
:1061E00001960E946B84BE016F5F7F4F87E493E14D
:1061F0000E948985CE0101960E94D58326960FB60E
:10620000F894DEBF0FBECDBFDF91CF911F910F91EC
:1062100008952F923F924F925F926F927F928F924A
:106220009F92AF92BF92CF92DF92EF92FF920F9325
:106230001F93CF93DF93CDB7DEB7C258D1090FB606
:10624000F894DEBF0FBECDBF6C015B0188EE482E17
:1062500083E0582E612C712C02E114E09BE5892E1D
:10626000912C8C0E9D1E8CE0880E911C1B019FEFC3
:10627000291A390AD6015996ED90FC90F7018581CB
:10628000823008F493C082859385A485B5858F718B
:106290009927AA27BB27892B8A2B8B2B09F086C02D
:1062A00040E250E0BE016F5F7F4FC7010E94A7161A
:1062B000803209F07BC08981882309F477C0853E4C
:1062C00079F38E3269F38C8583FDEACF22961FAE77
:1062D0001EAE229782E993E09FAF8EAF24961FAE49
:1062E0002497BE016F5F7F4FE0E080E04EE2DB016C
:1062F0009D91BD019032A1F0883049F426E730E04D
:106300002C0F3D1F2E0F311DD9014C93EF5F26E757
:1063100030E02C0F3D1F2E0F311DD9019C93EF5FF4
:106320008F5F8B3021F786E790E08C0F9D1F8E0FDB
:10633000911DFC011082D60159966D917C9121E04E
:10634000AE014A585F4FCE01CE960E943618882380
:1063500069F1BE01625C7F4FCE0181960E94001CF4
:10636000AE014A585F4FBE016F5D7F4FCE01855A27
:106370009F4F0E946E1CCE01855A9F4F0E94501C59
:10638000882309F4ACC0F12CFA141B042CF569E045
:10639000CE0101960E944084CE0101960E94C83031
:1063A000CE0101960E94D583F394EECF6F961FAE77
:1063B0001EAE6F97A3964CAE5DAE6EAE7FAEA3974A
:1063C0006D961FAF0EAF6D97E6961FAE1EAEE697A9
:1063D000A8961FAEA897CFCFB401CE0101960E9418
:1063E0007484CE0101960E94C830CE0101960E94AD
:1063F000D583E696EEADFFADE697309709F447C03A
:106400008581823008F443C066E874E0CE010196CD
:106410000E947484CE0101960E947A30CE010196CA
:106420000E94D5836F968EAD9FAD6F979C838B83B3
:10643000A3968CAD9DADAEADBFADA3978D839E836E
:10644000AF83B887A7968CAD9DADAEADBFADA79716
:1064500089879A87AB87BC871A8309838DE0F4010B
:10646000DE011D9601900D928A95E1F7E6968EADBC
:106470009FADE6979B8F8A8FB101CE0101960E9456
:106480000931CE01855A9F4F0E945C1CF3CE6BE50B
:1064900074E0CE0101960E947484CE0101960E94A0
:1064A000C830CE0101960E94D583E696EEADFFADD1
:1064B000E69740E050E0BA01309721F043895489D3
:1064C00065897689CE0101960E94F881CE010196F8
:1064D0000E947A30CE0101960E94D583D2CFCE574A
:1064E000DF4F0FB6F894DEBF0FBECDBFDF91CF9167
:1064F0001F910F91FF90EF90DF90CF90BF90AF90E2
:106500009F908F907F906F905F904F903F902F90D3
:106510000895DF92EF92FF920F931F93CF93DF9333
:10652000CDB7DEB762970FB6F894DEBF0FBECDBF12
:106530008C01109265096DE574E0CE010D960E9404
:106540007484FF24F39487E49FE00E9422772091D3
:106550006509181619067CF521112DC087E49FE006
:106560000E9400778A3009F07EC089899A89892B38
:1065700009F481C0F09265096EE574E0CE010196E0
:106580000E947484BE01635F7F4FCE0101960E941A
:10659000EF82BC01CE0107960E946B84CE01079664
:1065A0000E94E12ECE0107960E94D583CE0101966E
:1065B0000E94D58360C0F12CE12CDD24D3942223EA
:1065C00009F460C089899A89019709F045C06DE294
:1065D00075E0CE0107960E947484BE01695F7F4F0B
:1065E000CE010D960E94BE82F12C811115C06EE67F
:1065F00074E0CE0101960E947484BE016F5F7F4FEC
:10660000CE010D960E94BE82FF24F3948111F12CDD
:10661000CE0101960E94D583CE0107960E94D583B4
:10662000FF20A1F050E040E0BE01635F7F4FCE014C
:1066300001960E94AB2DBE016F5F7F4F87E191E114
:106640000E949C83CE0101960E94D58364E170E094
:1066500080E090E00E945E0DBE01635F7F4FC80145
:106660000E9459848EC08D3009F47FCF682FCE01EF
:106670000D960E942C836AE070E080E090E00E941A
:106680005E0D61CF8AEA9EE00E94227718161906F5
:1066900014F58AEA9EE00E9400778A30A9F08D30D6
:1066A00099F09091650991110FC0682FCE010D9658
:1066B0000E942C838FEFE81AF80A65E070E080E012
:1066C00090E00E945E0DDECF89899A89892BA9F31B
:1066D000D0926509F2CF64E170E080E090E00E9422
:1066E0005E0DEF2809F43FC089899A89892BD9F179
:1066F0008091CD0B882389F165E876E0CE01019683
:106700000E947484BE016F5F7F4FCE010D960E9480
:10671000BE82F82ECE0101960E94D583F1101DC0D5
:1067200067E674E0CE0101960E947484CE01019662
:106730000E94C830CE0101960E94D583BE01635FDE
:106740007F4FCE0101960E946B84CE0101960E947C
:106750007A30CE0101960E94D58364E170E080E03A
:1067600090E00E945E0D89899A8920916509211126
:106770002BCF009709F028CF6DE574E0C8010E9487
:106780007484CE010D960E94D583C80162960FB61F
:10679000F894DEBF0FBECDBFDF91CF911F910F9157
:1067A000FF90EF90DF9008950F931F93CF93DF93A7
:1067B000CDB7DEB72C970FB6F894DEBF0FBECDBFB6
:1067C0002C893D89FE017496A9E4BCE090E080E04C
:1067D00032962817390734F0408151814D935D93EB
:1067E0000196F6CFCE5BDE4F88819981C254D140AD
:1067F000281739070CF044C2DC01AA0FBB1FA75BA6
:10680000B34F880F991FFC01E95BF34F80819181A1
:1068100001968D939C938C8D9D8D9093520C8093BB
:10682000510C8E8D9F8D9093540C8093530CAD968C
:106830008FADAD97BE0164597F4F8F3209F029C2E9
:10684000CE0107960E94748460E774E0CE01019641
:106850000E947484BE01695F7F4FCE0101960E9441
:10686000EF82BC018BE093E10E948583CE0101960B
:106870000E94D583CE0107960E94D5836BE073E119
:10688000CE0101960E946B84CE0101960E947A305F
:10689000CE0101960E94D58366E874E0CE01019690
:1068A0000E947484BE016F5F7F4F8BE093E10E9472
:1068B0009E82182FCE0101960E94D58340910F131E
:1068C00050911013112309F4EBC1BA016250710900
:1068D0008BE093E10E948D82682FCE0101960E9489
:1068E0004084BE016F5F7F4F8DEE92E10E949C83DA
:1068F000CE0101960E94D5836AED71E1CE01079623
:106900000E94748468E874E0CE0101960E94748449
:10691000BE01695F7F4FCE0101960E94EF82BC01EC
:1069200085E093E10E948583CE0101960E94D58384
:10693000CE0107960E94D58324968FAD24971F928F
:106940008F9323968FAD23971F928F9322968FADAF
:1069500022971F928F9321968FAD21971F928F932D
:106960008EE894E09F938F938FE59AE09F938F93A7
:106970000E94FEB8CE52DF4F88819981C25DD0401F
:106980009093730280937202BE016C527F4FCE01CE
:1069900001960E947484BE016F5F7F4FCE010796FF
:1069A0000E946B84CE0107960E944083BC018FEF4A
:1069B00092E10E948583CE0107960E94D583CE0185
:1069C00001960E94D583BE0161527F4FCE01019690
:1069D0000E947484BE016F5F7F4F89EF92E10E9435
:1069E0009C83CE0101960E94D5834091FD12509167
:1069F000FE124250510969EF72E1CE0101960E94E8
:106A0000AB2DCE0101960E9425826C5960939702AE
:106A1000CE0101960E94D583CC5EDE4F68817981DC
:106A20008A819B81C451D1400E946EB30FB6F89405
:106A3000DEBF0FBECDBF9B01AC010E942EB68823E6
:106A400089F08CE390E0A0E0B0E0CC5EDE4F88837C
:106A50009983AA83BB83C451D140CD5EDE4F188297
:106A6000C351D140CD5EDE4F8881C351D1408823D0
:106A700099F0CC5EDE4F88819981AA81BB81C45197
:106A8000D14080936E0290936F02A0937002B093F6
:106A9000710281E08093460CC85EDE4F6881798187
:106AA0008A819B81C851D1409B01AC010E942EB6C6
:106AB000882361F080E090E0A0E7B2E4C85EDE4F9A
:106AC00088839983AA83BB83C851D140C45EDE4FBB
:106AD00068817981CC51D140072E000C880B990B2D
:106AE0000E946EB39B01AC010E942EB6882341F038
:106AF00082E090E0C45EDE4F99838883CC51D14020
:106B0000CE5BDE4F68817981C254D140072E000CE4
:106B1000880B990B0E946EB39B01AC010E942EB6AC
:106B2000882341F083E090E0CE5BDE4F9983888339
:106B3000C254D140C45CDE4F08811981CC53D1408E
:106B4000B801012E000C880B990B0E946EB39B01BB
:106B5000AC010E942EB6811103C01016110644F03C
:106B600080E590E0C45CDE4F99838883CC53D140AC
:106B7000C45CDE4F88819981CC53D140909341020F
:106B80008093400288E2FE01E551FF4FA2E3BAE0A4
:106B900001900D928A95E1F7CE5CDE4F8881998154
:106BA000AA81BB81C253D1408093290290932A02CB
:106BB000A0932B02B0932C02CA5CDE4F888199818E
:106BC000AA81BB81C653D1408093250290932602AF
:106BD000A0932702B0932802C65CDE4F888199817A
:106BE000CA53D1409093320280933102CC5BDE4F86
:106BF00068817981C454D140072E000C880B990B11
:106C00000E946EB39B01AC010E942EB6882341F016
:106C100088E390E0CC5BDE4F99838883C454D140F5
:106C2000CC5BDE4F88819981C454D140909375022A
:106C30008093740210925E0AC053DF4F888199815D
:106C4000C05DD04097FD03C081E080935E0A6091F3
:106C5000DC1270E090E080E00E946CB39B01AC011C
:106C60000E942EB681111092DC122C960FB6F89469
:106C7000DEBF0FBECDBFDF91CF911F910F91089561
:106C800080914D0C90914E0C9093500C80934F0C32
:106C9000C2CDCE0107960E94748465E774E0D6CD1C
:106CA000415051096BE073E1CE0101960E94AB2D7A
:106CB000BE016F5F7F4F8DEE92E10E949C83CE01FB
:106CC00001960E94D5836BE073E1CE0101960E948C
:106CD0006B8466E874E0CE0101960E94D982BC0103
:106CE0008BE093E10E94858303CEDF92EF92FF92C7
:106CF0000F931F93CF93DF93CDB7DEB762970FB695
:106D0000F894DEBF0FBECDBF2091F002222379F1AF
:106D10002091EF02222359F17A018C016F3F7F4FBE
:106D2000A1F560E080E00E94847BD12CB80183E66D
:106D300093E10E94898562E776E083E693E10E9411
:106D4000A985F801848160E08D0D0E94847B0E94FA
:106D5000910D6093550E7093560E8093570E90933D
:106D6000580EB701FF0C880B990B0E945E0D6296BE
:106D70000FB6F894DEBF0FBECDBFDF91CF911F914C
:106D80000F91FF90EF90DF90089560E080E00E9407
:106D9000847B0E94910D28EE33E040E050E00E9499
:106DA000B1B4CA01B90120E831E541E050E00E94E8
:106DB000D3B4AB01BC0120E0CE0101960E94138444
:106DC000BE016F5F7F4FCE0107960E946B846DE11D
:106DD00077E0CE0107960E94D982BC01CE010D96C4
:106DE0000E946B84CE0107960E94D583CE01019646
:106DF0000E94D583BE01635F7F4F83E693E10E94CB
:106E00008985D98860E08D2D0E94847BCE010D9606
:106E10000E94D5838BCFCF93DF9300D000D0CDB726
:106E2000DEB70E940029CE0101960E940D2F4AE094
:106E300050E06FEF7FEFCE0101960E947536CE01D4
:106E400001960E94D58361E080E00E94847BCE01A0
:106E500001960E94A32863E673E1CE0101960E9489
:106E600021856AE974E083E693E10E9481850E94AE
:106E7000910D6093DA0B7093DB0B8093DC0B909396
:106E8000DD0B26960FB6F894DEBF0FBECDBFDF91A7
:106E9000CF9108950F931F93CF93DF9300D000D02D
:106EA000CDB7DEB78C01CE0101960E940D2F4AE0CE
:106EB00050E06FEF7FEFCE0101960E947536CE0154
:106EC00001960E94D583B801CE0101960E946B8481
:106ED0004AE050E06FEF7FEFCE0101960E94242937
:106EE000CE0101960E94D58326960FB6F894DEBF98
:106EF0000FBECDBFDF91CF911F910F910895EF92FB
:106F0000FF920F931F93CF93DF9300D01F92CDB7C3
:106F1000DEB78C017B01FB0184858830A8F080E31B
:106F200094E0F80191838083128213821482158287
:106F3000C8010F900F900F900F90DF91CF911F918C
:106F40000F91FF90EF90089580E591E00E94807A84
:106F500024E030E0AE014F5F5F4F6CE070E0F7017E
:106F600084850E94AD1EBE016F5F7F4FC8010E94E5
:106F7000DF85DECF3F924F925F926F927F928F922A
:106F80009F92AF92BF92CF92DF92EF92FF920F93B8
:106F90001F93CF93DF93CDB7DEB7EA970FB6F89480
:106FA000DEBF0FBECDBF7C012A013B0169010E94FB
:106FB000910D4B015C0187010D5B1F4FC8010E94C1
:106FC0002722181619069CF00E94910D681979095C
:106FD0008A099B09461657066806790608F466C1B1
:106FE00062E370E080E090E00E945E0DE7CF42E255
:106FF00050E0BE016F5F7F4FC8010E94DE21898192
:107000008230D1F0312C832DEA960FB6F894DEBF92
:107010000FBECDBFDF91CF911F910F91FF90EF90E9
:10702000DF90CF90BF90AF909F908F907F906F90A8
:107030005F904F903F900895F8018489958983343B
:10704000910501F76D817E818F8198850E944FB6F1
:107050004B015C01F60180829182A282B38246E0FC
:1070600050E0B701685F7F4FCE014D960E947DB81A
:10707000892B41F6F70180819181A281B381881625
:107080009906AA06BB0608F4BDCF84819581A68126
:10709000B78188159905AA05BB0508F4B3CF89897E
:1070A0009A89AB89BC8986879787A08BB18B4EEC78
:1070B00050E070E060E0C8010E94DE21312CC70181
:1070C000829698AB8FA7F701B696FAABE9AB089614
:1070D0009CAB8BAB67019AE1C90ED11CBD96FEAB90
:1070E000EDABC701429698AF8FABFD97FAAFE9AF12
:1070F0004701FEE18F0E911CF801818D928D1816CB
:1071000019060CF080CFC8010E94FD218333910540
:1071100009F4B2C014F58130910509F464C044F457
:10712000892B51F3C8010E94FD21AC01552775C080
:107130008330910509F462C00697A1F7C8010E9447
:10714000FD21B82E44E050E0B401C8010E94DE21C8
:10715000EB2DE450FF0BAF0160C08A33910509F4B9
:107160005FC084F585339105B1F1C697D9F6C801A2
:107170000E94FD215C01B601CE0189960E94DF8547
:107180008BA59CA5ADA5BEA5892B8A2B8B2BB1F019
:10719000EDA9FEA94080518062807380B601CE01C6
:1071A00083960E94DF858DA19EA1AFA1B8A5A50100
:1071B000481659066A067B0609F0B8CF44E050E04D
:1071C000B60118C08B33910509F440C08F3F91057B
:1071D00009F492CFA7CFC8010E94FD21C8010E94E7
:1071E000FD21382E89CFC8010E94FD2144E050E0E6
:1071F0006FA978ADC8010E94DE217ECFC8010E9430
:10720000FD21B82E44E050E069AD7AADC8010E947E
:10721000DE218B2D8450990BAC0170E060E0EACF49
:10722000C8010E94FD2144E050E069A97AA9C80183
:107230000E94DE21F70166A177A180A591A50E9499
:107240004FB666A377A380A791A756CFC8010E9427
:10725000FD2144E050E06BA97CA9C8010E94DE2119
:10726000F70162A573A584A595A50E944FB662A7F4
:1072700073A784A795A740CFC8010E94FD2144E0D1
:1072800050E06FA578A9C8010E94DE21F70162A134
:1072900073A184A195A10E944FB662A373A384A396
:1072A00095A366A777A780AB91AB26CF33243A94FA
:1072B000AACE2F923F924F925F926F927F928F92BF
:1072C0009F92AF92BF92CF92DF92EF92FF920F9375
:1072D0001F93CF93DF9300D000D0CDB7DEB78C01E2
:1072E0000E94D2AA2FEC37E040E050E00E94D3B4D5
:1072F000DC01CB010196A11DB11DF80184839583AA
:10730000A683B78380839183A283B3835801F3E478
:10731000AF0EB11CC5010E94FF2264E470E0C501FC
:107320000E94D325882309F445C10E94910D2B01A9
:107330003C01480182E4880E911C48EEC42E43E0D3
:10734000D42EE12CF12C52E0252E1E821D82D40178
:107350008C918330B1F1811166C0F80184819581EF
:10736000A681B7810196A11DB11D84839583A68353
:10737000B7830E94910D6419750986099709A701C1
:1073800096010E94B1B4A90161E0C8010E94932650
:1073900081E0D4018C938D819E810197C1F20E947E
:1073A000910D6419750986099709D801D6962D9112
:1073B0003D914D915C91D99726173707480759079A
:1073C00020F6C5010E94FF22F80184819581A681E3
:1073D000B7810196A11DB11D84839583A683B783D0
:1073E0000E94910DF801FE966083718382839383DE
:1073F0008D819E8126960FB6F894DEBF0FBECDBF5D
:10740000DF91CF911F910F91FF90EF90DF90CF9080
:10741000BF90AF909F908F907F906F905F904F90B4
:107420003F902F9008958430F1F4F8018481958184
:10743000A681B7810196A11DB11D84839583A68382
:10744000B7830E94910D6419750986099709A701F0
:1074500096010E94B1B4A90163E0C8010E9493267D
:10746000D4012C9298CF813051F5F80142AD53AD43
:1074700064AD75AD9E012F5F3F4FC8010E94BA37C2
:10748000382EF2E08F1390C089819A81AB81BC8144
:10749000F80184839583A683B7830E94910D6419B4
:1074A000750986099709A70196010E94B1B4A9013F
:1074B00063E0C8010E949326D4013C926CCF8230D5
:1074C00009F069CFF80142AD53AD64AD75AD9E01D1
:1074D0002F5F3F4FC8010E94BA37382EF5E08F1357
:1074E0005DC0E3E0D401EC93F80182A193A1A4A1D3
:1074F000B5A1892B8A2B8B2B41F484E893E0A0E083
:10750000B0E082A393A3A4A3B5A3F80186A197A199
:10751000A0A5B1A5892B8A2B8B2B61F482A193A105
:10752000A4A1B5A1B695A7959795879586A397A38E
:10753000A0A7B1A7F80182A593A5A4A5B5A5892BFD
:107540008A2B8B2BA9F482A193A1A4A1B5A1AC0194
:10755000BD0123E076956795579547952A95D1F714
:10756000841B950BA60BB70B82A793A7A4A7B5A75F
:10757000F80186A197A1A0A5B1A586A797A7A0AB62
:10758000B1AB82A593A5A4A5B5A582AB93ABA4ABE3
:10759000B5AB81E090E09E838D83FDCE96E08913AC
:1075A00003C0D4011C92F7CEBFEF3B12F4CEF4011E
:1075B0001082F1CE1E821D821BCF8F929F92AF92BE
:1075C000BF92EF92FF920F931F93CF93DF9300D060
:1075D00000D0CDB7DEB70091420C1091430CF12CD6
:1075E000E12C0115110509F4DAC00E94910D4B013F
:1075F0005C0178012EE3E20EF11CF701808191819C
:10760000A281B381A5019401281B390B4A0B5B0BA6
:10761000CA01B901683E33E0730781059105A0F105
:1076200028EE33E040E050E00E94B1B4861A970A99
:10763000A80AB90AD7018D929D92AD92BC92139778
:10764000F80186A597A5A0A9B1A949015A01880CFE
:10765000991CAA1CBB1C88159905AA05BB0508F036
:10766000B0C016A617A610AA11AAF80182A993A95C
:10767000A4A9B5A988159905AA05BB0508F0AAC053
:1076800012AA13AA14AA15AAF80186A597A5A0A95B
:10769000B1A9892B8A2B8B2B09F0A5C0EE5BFF4F7C
:1076A0008081833009F09FC084E08083C8010E94FC
:1076B000593901967C01F80182A993A9A4A9B5A919
:1076C000892B8A2B8B2BA1F4EE5BFF4F80818330BB
:1076D00011F081110DC01082F8013E9684E1DF01A6
:1076E0001D928A95E9F7C8010E94593903967C01D9
:1076F000B2E0EB16F10429F0E4E0EE16F10409F033
:107700004EC080E591E00E94807A6091420C7091B9
:10771000430C625F7F4FCE0101960E94DF85CE0150
:1077200003960E94B31F6091420C7091430C6A5EF5
:107730007F4FCE0101960E94DF8544E050E0BE01FC
:107740006D5F7F4F81E090E00E94551D6091420C7B
:107750007091430C6E5E7F4FCE0101960E94DF85D3
:1077600044E050E0BE016D5F7F4F85E090E00E94F5
:10777000551D6091420C7091430C625E7F4FCE01AB
:1077800001960E94DF858B819C81AD81BE818093B3
:107790003B1090933C10A0933D10B0933E10C70156
:1077A00026960FB6F894DEBF0FBECDBFDF91CF9106
:1077B0001F910F91FF90EF90BF90AF909F908F908F
:1077C0000895821B930BA40BB50B86A797A7A0ABBC
:1077D000B1AB4BCF821B930BA40BB50B82AB93AB1E
:1077E000A4ABB5AB51CFF12CE12C65CFEF92FF925A
:1077F0000F931F93CF93DF93CDB7DEB7E8970FB604
:10780000F894DEBF0FBECDBF6DE574E0CE01879664
:107810000E9474846DE574E0CE018D960E9474849C
:1078200082E0E82EF12C2496FFAEEEAE249786E09F
:10783000EBEFF2E0DE01D39601900D928A95E1F72D
:1078400086E0FE01F396DE01AC5BBF4F01900D9226
:107850008A95E1F701E010E02C961FAF0EAF2C9750
:107860002E961FAE1EAE2E9788E0E1E0F3E0DE011B
:10787000599601900D928A95E1F788E0FE0179967C
:10788000DE01A25BBF4F01900D928A95E1F788E17E
:10789000E9E0F3E0DE01119601900D928A95E1F79F
:1078A00088E1FE013196DE01AA5ABF4F01900D9288
:1078B0008A95E1F78091210390912203A0912303FF
:1078C000B0912403E2968CAF9DAFAEAFBFAFE2970D
:1078D0006EE974E0CE0187960E94C28160E0CE011D
:1078E00087960E942C834BA55CA5BE016E587F4FE6
:1078F000CE0187960E94F37F6BE877E0CE018D96EC
:107900000E94608364E275E08DEE92E10E94C28184
:1079100060E0CE018D960E942C8349A95AA9BE0130
:1079200066567F4FCE018D960E94F37F6DE574E021
:10793000CE0187960E94C2816DE574E0CE018D96DE
:107940000E94C281C250DF4F19821882CE5FD040A0
:1079500010925E0A8091720290917302C050DF4FC4
:1079600099838883C050D14080E090E0A0E7B2E4E2
:10797000CA5BDE4F88839983AA83BB83C654D140F8
:10798000C65BDE4FF982E882CA54D14080E090E0C5
:10799000A0E2B2E4C45BDE4F88839983AA83BB83F1
:1079A000CC54D14080E090E0A4E3B2E4C05BDE4F71
:1079B00088839983AA83BB83C055D14084EB90E030
:1079C000CC5ADE4F99838883C455D14088E790E034
:1079D000CA5ADE4F99838883C655D1408CE291E024
:1079E000A0E0B0E0C85ADE4F88839983AA83BB83A6
:1079F000C855D140C45ADE4F19830883CC55D140B5
:107A0000C25ADE4FF982E882CE55D14060E08FEF56
:107A100092E10E942C8360E089EF92E10E942C8326
:107A20004091031350910413BE016E5F7E4F8FEFA0
:107A300092E10E94F37F4091FD125091FE12BE012F
:107A4000635F7E4F89EF92E10E94F37F88E2E2E379
:107A5000FAE0DE01A75EBE4F01900D928A95E1F734
:107A60008CE390E0A0E0B0E0CE5BDE4F88839983AA
:107A7000AA83BB83C254D140CF5BDE4F1882C1546E
:107A8000D14084EE98E3AEE8B2E4C05ADE4F88837A
:107A90009983AA83BB83C056D14084EE98E3AEE8B5
:107AA000B1E4CC59DE4F88839983AA83BB83C45643
:107AB000D140C859DE4F19830883C856D14080E5AC
:107AC00090E0C659DE4F99838883CA56D14083E03F
:107AD00090E0C059DE4F99838883C057D14088E336
:107AE00090E0CE58DE4F99838883C257D140CC585E
:107AF000DE4F1882C457D1408FEF9FEFCB58DE4F37
:107B000099838883C557D14084EF91E090935302C5
:107B100080935202BE016E5B7F4F0E94BF2864EFCC
:107B200071E080E090E00E945E0D64E777E0CE01B6
:107B300081960E946284CE0181960E947A30CE01A5
:107B400081960E94D583CE018D960E94D583CE0169
:107B500087960E94D583E8960FB6F894DEBF0FBED5
:107B6000CDBFDF91CF911F910F91FF90EF900895BE
:107B70006F927F929F92AF92BF92CF92DF92EF92DD
:107B8000FF920F931F93CF93DF93CDB7DEB7C3510F
:107B9000D1400FB6F894DEBF0FBECDBF3C016B01E4
:107BA0005A017E0181E8E80EF11C62E072E1C70132
:107BB0000E94748466E874E08E010F5F1F4FC80155
:107BC0000E947484B701C8010E94EF82BC01CE01FB
:107BD000885F9E4F0E946B84C8010E94D583C701B5
:107BE0000E94D583B301CE01825F9E4F0E947484B0
:107BF00094E0C916D10409F094C066EA74E0CE019D
:107C0000885F9E4F0E944F839924939460E0CE0139
:107C1000885F9E4F0E942C83C45FDE4F488159814C
:107C2000CC50D140B701CE01885F9E4F0E94F37FB8
:107C30008091CD0B8823B9F062ED74E0C8010E94F9
:107C40007484C8010E94C830C8010E94D583BE0157
:107C5000685F7E4FC8010E946B84C8010E947A3021
:107C6000C8010E94D583E4E9F8E080ECDF011D92B1
:107C70008A95E9F7992009F462C0C25FDE4F6881F6
:107C80007981CE50D140CF010E94C0B86DE574E03B
:107C9000CE01825F9E4F0E94C281A0904002B090B0
:107CA00041028091D00B9091D10B01969093D10B12
:107CB0008093D00B2091EC0B222341F06EE170E019
:107CC0000E9433B6181619060CF4C7C181E08093E0
:107CD000EC0B1092D10B1092D00BA5016FE57AE05E
:107CE00089E891E10E9490246C018FE1682E712C4B
:107CF00091E0C916D10409F449C1A1E06A1A7108DA
:107D000009F49CC16AE070E080E090E00E945E0DA2
:107D1000A5016FE57AE089E891E10E9490246C0169
:107D2000E7CF66EB74E0C114D10411F065EC74E0A8
:107D3000CE01885F9E4F0E944F83912C67CFD50163
:107D40008C9111969C91C114D10491F49F938F93BF
:107D50001F921F928BEE94E09F938F93FF93EF936C
:107D60000E94FEB80FB6F894DEBF0FBECDBF8ECF17
:107D70009F938F93DF92CF92C15FDE4F8881CF5068
:107D8000D1408F93C25FDE4F8881CE50D1408F9318
:107D900082EE94E09F938F93FF93EF930E94FEB83F
:107DA000E1CF81E08093440C41E064E978E0CE01CA
:107DB0008F519F4F0E94F689CE018F519F4F0E9495
:107DC000501C882309F4ACC064EB75E089E891E1AC
:107DD0000E94CD8561E675E089E891E10E94CD853C
:107DE00060E575E089E891E10E94A985C650DF4F02
:107DF000E881F981CA5FD04040E050E0BA01309795
:107E000021F043895489658976894C535F4F6F4FC0
:107E10007F4F2AE089E891E10E94D58489E891E1C9
:107E20000E946B8589E891E10E946B8567E275E0AD
:107E300089E891E10E94CD856FEE74E089E891E1D7
:107E40000E94A98564E978E0CE018E5F9E4F0E9472
:107E50007484BE016E5F7E4FCE0184509F4F0E949E
:107E60006B846EEF74E0CE0184509F4F0E94D982E4
:107E7000BC0189E891E10E949785CE0184509F4F13
:107E80000E94D583CE018E5F9E4F0E94D58368EC01
:107E900074E089E891E10E94CD8589E891E10E9432
:107EA0006B853801B12CA12CCE018F519F4F0E94C0
:107EB000300B892BB9F0CE018F519F4F0E94C5170F
:107EC000F30181933F01FFEFAF1ABF0A80E8A816C4
:107ED000B10451F740E850E0B80189E891E10E940F
:107EE0003520DFCFA114B10431F0A501B80189E834
:107EF00091E10E94352089E891E10E946B856DE94E
:107F000074E089E891E10E94CD8589E891E10E94C1
:107F10006B85CE018F519F4F0E945C1C1092440CC8
:107F200061E070E080E090E00E945E0D1092440CF1
:107F30001092EC0BE4E9F8E080ECDF011D928A95E9
:107F4000E9F780E6F70111928A95E9F7CE01825FA1
:107F50009E4F0E94D583CE01885F9E4F0E94D5839D
:107F6000C601CD5EDE4F0FB6F894DEBF0FBECDBFAB
:107F7000DF91CF911F910F91FF90EF90DF90CF9005
:107F8000BF90AF909F907F906F900895FF92EF9277
:107F900085E195E09F938F931F930F930E94FEB806
:107FA000B80189E891E10E946F858FE59AE09F937F
:107FB0008F9386E295E09F938F931F930F930E9478
:107FC000FEB8B80189E891E10E946F850FB6F89478
:107FD000DEBF0FBECDBF9110E4CE6AE574E089E844
:107FE00091E10E94CD8584E998E0DC010D900020AC
:107FF000E9F7CD01855998409F938F9380E095E0F4
:108000009F938F931F930F930E94FEB8B80189E846
:1080100091E10E946F8564E978E089E891E10E942E
:108020006F8566E474E089E891E10E94CD850F9048
:108030000F900F900F900F900F9072CF6AE374E043
:10804000C8010E946284C8010E947A30C8010E945F
:10805000D5831092440C1092EC0B8091310A81115F
:1080600016C066EC75E0C8010E946284C8010E94D7
:10807000C830C8010E94D58364E978E0C8010E9435
:108080007484C8010E947A30C8010E94D58362E3DB
:1080900070E080E090E00E945E0D89E891E10E942E
:1080A000422489E891E10E947B24E4E9F8E080EC35
:1080B000DF011D928A95E9F780E6F70111928A9512
:1080C000E9F7D12CC12C42CFEF92FF920F931F936F
:1080D000CF93DF93CDB7DEB76E970FB6F894DEBFC0
:1080E0000FBECDBF81E08093EC0B0E94DD3A8C0186
:1080F00060ED77E080E090E00E945E0D8BE0E82E7E
:10810000F12C0D7F0130110571F481E0E81AF108BE
:1081100051F00E94DD3A8C0160ED77E080E090E064
:108120000E945E0DEECF0E94E5877C0168EE73E051
:1081300080E090E00E945E0D0BE010E0EF2899F4E3
:108140000150110981F060ED77E080E090E00E943D
:108150005E0D0E94E5877C0168EE73E080E090E0B0
:108160000E945E0DEBCF83E490E10E94A127109264
:10817000EC0B0E940B376DE574E0CE010D960E946A
:1081800074846AEF76E0CE0143960E946284CE0149
:1081900049960E94A3288E8D1F928F938D8D1F92DA
:1081A0008F938C8D1F928F938B8D1F928F938EE860
:1081B00094E09F938F938AE999E09F938F930E9415
:1081C000FEB86AE979E0CE0101960E947484BE018E
:1081D0006F5F7F4FCE010D960E949C83CE0101966A
:1081E0000E94D583BE01635F7F4FCE0101960E943E
:1081F0006B84AE014F5F5F4F63E070E080E092E020
:108200000E94B83D8C01CE0101960E94D5830FB625
:10821000F894DEBF0FBECDBF01301105A1F5BE0140
:108220006D5E7F4FCE0101960E946B84BE01635F3D
:108230007F4FCE0101960E94EF82BC01CE010796CE
:108240000E946B84CE0107960E947A30CE01079679
:108250000E94D583CE0101960E94D583CE0143961C
:108260000E94D583CE010D960E94D5836E960FB6DF
:10827000F894DEBF0FBECDBFDF91CF911F910F915C
:10828000FF90EF90089560EF76E0CE0101960E9496
:108290006284CE0101960E94C830CE0101960E94F0
:1082A000D583BE016D5E7F4FCE0101960E946B8427
:1082B000CE0101960E94C830CE0101960E94D5835E
:1082C000BE01635F7F4FCE0101960E946B84CE0199
:1082D00001960E947A30CE0101960E94D58366E510
:1082E00071E1CE0101960E946B84CE0101960E943D
:1082F0007A30CE0101960E94D583B0CF3F924F9243
:108300005F926F927F928F929F92AF92BF92CF9225
:10831000DF92EF92FF920F931F93CF93DF93CDB72E
:10832000DEB762970FB6F894DEBF0FBECDBF6DED1E
:1083300076E0CE0101960E946284CE0101960E94F1
:108340007A30CE0101960E94D58304E010E036E633
:10835000C32E39E0D32E40E3E42E53EE752E66E0B3
:10836000662E7CEE572EE1E3FE2EFEE44F2EA4E3B4
:108370003A2E68EB72E289E291E10E94D325F60180
:108380008E2D11928A95E9F77092660960926809BC
:1083900050926909F092720940927309F09274093F
:1083A0003092750962E472E0CE0101960E94DF8589
:1083B0004BE750E0BE016F5F7F4F89E291E10E9481
:1083C0005C2640E350E066E679E089E291E10E94B4
:1083D000F12589E291E10E942B2668EE73E080E0AE
:1083E00090E00E945E0D89E291E10E942722892B94
:1083F00009F053C00150110909F080C0809196091D
:1084000090919709A0919809B0919909892B8A2B8D
:108410008B2B09F08DC06DE574E084E791E10E943B
:10842000C28164E771E1CE0101960E946B84AE01C6
:108430004F5F5F4F70E060E086E792E00E94B83DDA
:108440008C01CE0101960E94D583012B71F465EC5D
:1084500076E0CE0101960E946284CE0101960E94D0
:108460007A30CE0101960E94D58362960FB6F894B9
:10847000DEBF0FBECDBFDF91CF911F910F91FF9057
:10848000EF90DF90CF90BF90AF909F908F907F90B4
:108490006F905F904F903F90089540E350E066E604
:1084A00079E089E291E10E94DE2160918E0970916C
:1084B0008F0976276727762790E080E0CB01772722
:1084C0006627009190091091910910270127102724
:1084D00030E020E0602B712B822B932B7E508A4A58
:1084E00093480E949D0D0E94500E609396097093D0
:1084F0009709809398099093990980CF8090960965
:1085000090909709A0909809B090990968EE73E04F
:1085100080E090E00E945E0D2AE0B501A40187E4AE
:108520009FE00E94D58487E49FE00E946B8521CF65
:1085300068EE73E080E090E00E945E0D0E94500EB5
:108540006093E40B7093E50B8093E60B9093E70B3D
:108550000E94500E6093DE0B7093DF0B8093E00B54
:108560009093E10BCE0101960E948E2FCE010196D1
:108570000E947A30CE0101960E94D5830E94A80EF7
:10858000BC01CE0107960E94B72D69E574E0CE01CB
:1085900007960E944F830E94A00EBC01CE01019657
:1085A0000E94B72DBE016F5F7F4FCE0107960E94DC
:1085B0005983CE0101960E94D58369E574E0CE010E
:1085C00007960E944F830E94960EBC01CE01019631
:1085D0000E94B72DBE016F5F7F4FCE0107960E94AC
:1085E0005983CE0101960E94D5836FE275E0CE01DA
:1085F00001960E947484BE01695F7F4FCE0101968F
:108600000E94EF82BC01CE010D960E946B844AE06D
:1086100050E06FEF7FEFCE010D960E947536CE01D0
:108620000D960E94D583CE0101960E94D583CE017E
:1086300007960E94D58368EE73E080E090E00E9488
:108640005E0D0E94B80EBC01CE010D960E94B72DA2
:108650000E94B00EBC01CE0101960E94B72D6FE4BE
:1086600076E0CE0107960E947484BE016F5F7F4F53
:10867000CE0107960E94EF82BC01CE010D960E94AA
:108680005983CE0107960E94D583CE0101960E94A0
:10869000D5830E94500E0E9488096091AD0B70E056
:1086A000CE0101960E94B72D6FE476E0CE010796C9
:1086B0000E947484BE016F5F7F4FCE0107960E94B7
:1086C000EF82BC01CE010D960E945983CE01079620
:1086D0000E94D583CE0101960E94D58365E375E0A3
:1086E000CE0101960E947484BE01635F7F4FCE016C
:1086F00001960E94EF82BC01CE0107960E946B8416
:108700004AE050E06FEF7FEFCE0107960E9475368A
:10871000CE0107960E94D583CE0101960E94D58393
:10872000CE010D960E94D58368EE73E080E090E064
:108730000E945E0DCE0101960E940D2F4AE050E08E
:108740006FEF7FEFCE0101960E9475368ACECF92F1
:10875000DF92EF92FF920F931F93CF93DF93CDB7EA
:10876000DEB768970FB6F894DEBF0FBECDBF6DE5DC
:1087700074E0CE0143960E94748469ED78E0CE01E6
:1087800001960E946284CE0101960E94C830CE01FB
:1087900001960E94D5836CA17DA1CE0101960E9415
:1087A000CC81CE0101960E947A30CE0101960E94C2
:1087B000D58361EC78E0CE0101960E946284CE01FF
:1087C00001960E94C830CE0101960E94D583CE5AF0
:1087D000DE4F68817981C255D140CE0101960E9459
:1087E000CC81CE0101960E947A30CE0101960E9482
:1087F000D58364EB78E0CE0101960E946284CE01BD
:1088000001960E94C830CE0101960E94D58309E4EA
:108810001CE0EE24E394F12CCE5ADE4F888199813E
:10882000C255D1408E159F050CF44AC0F8018281D3
:108830009381C6979CF16BE375E0CE0101960E948F
:108840007484CE0101960E94C830CE0101960E9428
:10885000D583F8016281738166537109CE01019657
:108860000E94CC81CE0101960E94C830CE010196B3
:108870000E94D5836AEB75E0CE0101960E94748454
:10888000CE0101960E94C830CE0101960E94D58388
:10889000FFEFEF1AFF0A0E5F1F4FBECF6DE375E0CB
:1088A000CE0101960E947484CE0101960E94C830C8
:1088B000CE0101960E94D583F80162817381CECFEB
:1088C0006AEB75E0CE0101960E947484CE01019698
:1088D0000E947A30CE0101960E94D58365EA78E045
:1088E000CE0101960E946284CE0101960E94C8309A
:1088F000CE0101960E94D5836091510C7091520C6B
:10890000CE0101960E94CC81CE0101960E94C83012
:10891000CE0101960E94D5836AEB75E0CE010196E7
:108920000E947484CE0101960E94C830CE01019647
:108930000E94D5836091530C7091540CCE01019626
:108940000E94CC81CE0101960E947A30CE01019620
:108950000E94D5836EE878E0CE0101960E94628481
:10896000CE0101960E94C830CE0101960E94D583A7
:10897000BE01605D7F4FCE0101960E947484CE01DE
:1089800001960E94C830CE0101960E94D5836AEB01
:1089900075E0CE0101960E947484CE0101960E947A
:1089A000C830CE0101960E94D583BE016C5C7F4F1A
:1089B000CE0101960E947484CE0101960E947A3005
:1089C000CE0101960E94D5836EE778E0CE01019634
:1089D0000E946284CE0101960E947A30CE010196F7
:1089E0000E94D5838E010C5D1F4FEE24E394F12C81
:1089F000680188E0C80ED11C8CA19DA18E159F0531
:108A00000CF449C0B701CE0107960E94CC8165E8FD
:108A100076E0CE0101960E947484BE01695F7F4FAB
:108A2000CE0101960E94EF82BC01CE010D960E94FC
:108A30006B84CE010D960E94C830CE010D960E9427
:108A4000D583CE0101960E94D583CE0107960E9460
:108A5000D5836FE476E0CE0101960E947484CE0146
:108A600001960E94C830CE0101960E94D583B801BC
:108A7000645E7F4FCE0101960E947484CE01019600
:108A80000E947A30CE0101960E94D583EFEFEE1A54
:108A9000FE0A8601ADCF6DE678E0CE0101960E9418
:108AA0006284CE0101960E94C830CE0101960E94D8
:108AB000D5837E01F2EBEF1AFEEFFF0A10E000E033
:108AC000F70161917F0170E0CE0101960E94CC8197
:108AD000CE0101960E94C830CE0101960E94D58336
:108AE0000330110571F06FE375E0CE0101960E942D
:108AF0007484CE0101960E94C830CE0101960E9476
:108B0000D5830F5F1F4F04301105D1F66AEB75E076
:108B1000CE0101960E947484CE0101960E947A30A3
:108B2000CE0101960E94D583C45BDE4F68817981B6
:108B3000CC54D140072E000C880B990B0E946EB3C9
:108B40009B01AC010E942EB6882341F080E590E0A5
:108B5000C45BDE4F99838883CC54D140C45BDE4F25
:108B600088819981CC54D1409093410280934002F6
:108B700063E578E0CE0101960E946284CE01019601
:108B80000E94C830CE0101960E94D5836FE57AE03D
:108B9000CE0101960E947484CE0101960E94C830D5
:108BA000CE0101960E94D58361E578E0CE01019661
:108BB0000E946284CE0101960E94C830CE010196C7
:108BC0000E94D5836091400270914102CE010196CE
:108BD0000E94CC81CE0101960E947A30CE0101968E
:108BE0000E94D58362E478E0CE0101960E946284FF
:108BF000CE0101960E94C830CE0101960E94D58315
:108C0000BE016C5A7F4FCE0101960E947484CE0142
:108C100001960E947A30CE0101960E94D58361E4CC
:108C200075E0CE0101960E947484CE0101960E94E7
:108C3000C830CE0101960E94D583BE0164587F4F93
:108C4000CE0101960E947484CE0101960E947A3072
:108C5000CE0101960E94D583C052DF4F8881998151
:108C6000C05ED040892B71F46AE378E0CE010196B2
:108C70000E946284CE0101960E947A30CE01019654
:108C80000E94D583C052DF4F88819981C05ED04059
:108C9000019771F460E378E0CE0101960E9462844E
:108CA000CE0101960E947A30CE0101960E94D583B2
:108CB000C052DF4F88819981C05ED040029771F425
:108CC00067E278E0CE0101960E946284CE010196AF
:108CD0000E947A30CE0101960E94D58361E278E04D
:108CE000CE0101960E946284CE0101960E94C83096
:108CF000CE0101960E94D583CE51DF4F68817981E4
:108D0000C25ED040CE0101960E94CC81CE01019678
:108D10000E947A30CE0101960E94D58368E178E006
:108D2000CE0101960E946284CE0101960E94C83055
:108D3000CE0101960E94D583CC5ADE4F888199815D
:108D4000C455D140C6970CF43FC16BE375E0CE012A
:108D500001960E947484CE0101960E94C830CE0113
:108D600001960E94D583CC5ADE4F68817981C45523
:108D7000D14066537109CE0101960E94CC81CE018B
:108D800001960E947A30CE0101960E94D5834091CF
:108D9000D60B5091D70B6091D80B7091D90B21E075
:108DA000CE0107960E94DD836CE475E0CE0101964A
:108DB0000E947484BE01695F7F4FCE0101960E94BC
:108DC000EF8268E575E00E94D982BC01CE010D9664
:108DD0000E946B84CE010D960E947A30CE010D96D2
:108DE0000E94D583CE0101960E94D583CE010796BD
:108DF0000E94D5834091D20B5091D30B6091D40B3C
:108E00007091D50B21E0CE0107960E94DD836DE5C0
:108E100075E0CE0101960E947484BE01695F7F4FA8
:108E2000CE0101960E94EF8268E575E00E94D9822A
:108E3000BC01CE010D960E946B84CE010D960E945E
:108E40007A30CE010D960E94D583CE0101960E9404
:108E5000D583CE0107960E94D58369EF77E0CE01D6
:108E600001960E946284CE0101960E94C830CE0114
:108E700001960E94D5834091290250912A02609167
:108E80002B0270912C0225E0CE0101960E94DD8319
:108E9000CE0101960E947A30CE0101960E94D583C0
:108EA0006EED77E0CE0101960E946284CE010196BC
:108EB0000E94C830CE0101960E94D58340912502C0
:108EC00050912602609127027091280225E0CE0180
:108ED00001960E94DD83CE0101960E947A30CE0178
:108EE00001960E94D5836DEC77E0CE0101960E9439
:108EF0006284CE0101960E94C830CE0101960E9484
:108F0000D58360916C0270916D02CE0101960E9432
:108F1000CC81CE0101960E947A30CE0101960E944A
:108F2000D58364EB77E0CE0101960E946284CE0186
:108F300001960E94C830CE0101960E94D583C65B7F
:108F4000DE4F68817981CA54D140CE0101960E94DA
:108F5000CC81CE0101960E947A30CE0101960E940A
:108F6000D5836DE977E0CE0101960E946284CE013F
:108F700001960E94C830CE0101960E94D583C95A3D
:108F8000DE4F68817981C755D140CE0101960E949C
:108F9000CC81CE0101960E947A30CE0101960E94CA
:108FA000D583CE0143960E94D58368960FB6F89478
:108FB000DEBF0FBECDBFDF91CF911F910F91FF900C
:108FC000EF90DF90CF9008956DE375E0CE010196AC
:108FD0000E947484CE0101960E94C830CE01019691
:108FE0000E94D583CC5ADE4F68817981C455D14027
:108FF000C2CE2F923F924F925F926F927F928F924A
:109000009F92AF92BF92CF92DF92EF92FF920F9317
:109010001F93CF93DF93CDB7DEB7E5970FB6F894E4
:10902000DEBF0FBECDBF63E271E1CE018E960E941E
:109030006B840EA51FA50115110571F0D8018D9146
:109040008D01882349F0082E000C990B0E9475B8F9
:10905000F80131978083F2CF6CE77DE0CE01019675
:109060000E946284BE016F5F7F4FCE018E960E9488
:10907000BE82182FCE0101960E94D583112309F4D8
:1090800001C145E050E063E271E1CE0101960E942A
:10909000AB2DBE016F5F7F4F8FEF90E10E949C83ED
:1090A000CE0101960E94D5838FEF90E10E9430821D
:1090B00060E08FEF90E10E942C834091031150916A
:1090C000041162E072E18FEF90E10E94F37F66E8A5
:1090D00074E0CE0101960E947484BE016F5F7F4FE1
:1090E0008FEF90E10E94BE82182FCE0101960E9460
:1090F000D58360E774E0111102C065E774E0CE012A
:1091000001960E9474846FEF70E1CE0101960E9477
:10911000EF82BC018BE093E10E948583CE01019632
:109120000E94D5838BE093E10E94308240910F131F
:1091300050911013415051096BE073E1CE0101963B
:109140000E94AB2DBE016F5F7F4F8DEE92E10E94BA
:109150009C83CE0101960E94D5838DEE92E10E9400
:1091600025820E946EB39B01AC010E942EB688231B
:1091700009F448C060910F13709110136250710987
:109180008BE093E10E948D82682FCE0101960E94B0
:109190004084BE016F5F7F4F8DEE92E10E949C8301
:1091A000CE0101960E94D58366E874E0CE01019657
:1091B0000E947484BE016F5F7F4F8DEE92E10E942A
:1091C000BE82182FCE0101960E94D5831123D1F0C3
:1091D00060910F1370911013635071098BE093E14C
:1091E0000E948D82682FCE0101960E944084BE01AC
:1091F0006F5F7F4F8DEE92E10E949C83CE010196BE
:109200000E94D58384EF91E09093530280935202A1
:109210006AEA71E10E94BF2864E670E080E090E0B5
:109220000E945E0D80913F02882371F063E271E13C
:10923000CE0101960E946B84CE0101960E94E12E20
:10924000CE0101960E94D583CE018E960E94D583D1
:1092500081E0E5960FB6F894DEBF0FBECDBFDF917B
:10926000CF911F910F91FF90EF90DF90CF90BF9023
:10927000AF909F908F907F906F905F904F903F90B6
:109280002F90089566E77DE0CE0101960E946284EA
:10929000BE016F5F7F4FCE018E960E94BE82182F57
:1092A000CE0101960E94D583112309F447C045E001
:1092B00050E063E271E1CE0101960E94AB2DBE0148
:1092C0006F5F7F4F8FEF90E10E949C83CE010196EC
:1092D0000E94D5838FEF90E10E94308260E08FEF93
:1092E00090E10E942C8340910311509104116AED8A
:1092F00071E18FEF90E10E94F37F6AED71E1CE01A1
:109300004C960E94748468E874E0CE0101960E9435
:109310007484BE01645E7F4FCE0101960E94EF828D
:10932000BC0185E093E10E948583CE0101960E94F5
:10933000D583CE014C960E94D58364CF62E77DE051
:10934000CE0101960E946284BE016F5F7F4FCE0105
:109350008E960E94BE82182FCE0101960E94D58360
:109360001123E1F043E050E063E271E1CE010196A8
:109370000E94AB2DBE016F5F7F4F8FEF90E10E9487
:109380009C83CE0101960E94D5836FEF70E1CE01E0
:1093900001960E946B84CE010196CDCF6DE67DE0F3
:1093A000CE0101960E946284BE016F5F7F4FCE01A5
:1093B0008E960E94BE82182FCE0101960E94D58300
:1093C000112301F144E050E063E271E1CE01019626
:1093D0000E94AB2DBE016F5F7F4F8FEF90E10E9427
:1093E0009C83CE0101960E94D5838FEF90E10E946D
:1093F0002582709369126093681270937302609370
:10940000720200CF67E67DE0CE0101960E94628481
:10941000BE016F5F7F4FCE018E960E94BE82182FD5
:10942000CE0101960E94D583112309F449C045E07D
:1094300050E063E271E1CE0101960E94AB2DBE01C6
:109440006F5F7F4F8FEF90E10E949C83CE0101966A
:109450000E94D5838FEF90E10E9425827093C51200
:109460006093C41284EF91E0909353028093520270
:109470006AEA71E10E94BF2864E670E080E090E053
:109480000E945E0D65E876E0CE0101960E9474842C
:1094900063E271E1CE0101960E94EF82BC01CE0130
:1094A0004C960E946B84CE014C960E947A30CE017D
:1094B0004C960E94D583CE0101960E94D583B2CEF0
:1094C00062E67DE0CE0101960E946284BE016F5F7C
:1094D0007F4FCE018E960E94BE82182FCE0101963C
:1094E0000E94D5831123E1F044E050E063E271E192
:1094F000CE0101960E94AB2DBE016F5F7F4F8FEFB3
:1095000090E10E949C83CE0101960E94D5838FEF4B
:1095100090E10E9425827093C7126093C612A2CF79
:1095200069E57DE0CE0101960E946284BE016F5F15
:109530007F4FCE018E960E94BE82182FCE010196DB
:109540000E94D5831123E1F048E050E063E271E12D
:10955000CE0101960E94AB2DBE016F5F7F4F8FEF52
:1095600090E10E949C83CE0101960E94D5838FEFEB
:1095700090E10E9425827093DE126093DD1272CF1B
:1095800064E57DE0CE0101960E946284BE016F5FBA
:109590007F4FCE018E960E94BE82182FCE0101967B
:1095A0000E94D5831123A1F044E050E063E271E111
:1095B000CE0101960E94AB2DBE016F5F7F4F8FEFF2
:1095C00090E10E949C83CE0101960E94D58354CFE6
:1095D0006CE47DE0CE0101960E946284BE016F5F63
:1095E0007F4FCE018E960E94BE82182FCE0101962B
:1095F0000E94D5831123A1F047E050E063E271E1BE
:10960000CE0101960E94AB2DBE016F5F7F4F8FEFA1
:1096100090E10E949C83CE0101960E94D583FCCDEF
:1096200064E47DE0CE0101960E946284BE016F5F1A
:109630007F4FCE018E960E94BE82182FCE010196DA
:109640000E94D5831111D8CF6AE37DE0CE01019647
:109650000E946284BE016F5F7F4FCE018E960E9492
:10966000BE82182FCE0101960E94D583112321F0CE
:1096700081E00E94B82CD0CD63E37DE0CE0101965D
:109680000E946284BE016F5F7F4FCE018E960E9462
:10969000BE82182FCE0101960E94D583112319F0A6
:1096A0000E946440B9CD69E27DE0CE0101960E943E
:1096B0006284BE016F5F7F4FCE018E960E94BE8294
:1096C000182FCE0101960E94D583112309F485C07D
:1096D0006EE17DE0CE0101960E946284BE016F5F63
:1096E0007F4FCE018E960E94BE82182FCE0101962A
:1096F0000E94D583112309F454C04AE050E063E28C
:1097000071E1CE0101960E94AB2DBE016F5F7F4FCC
:109710008FEF90E10E949C83CE0101960E94D58339
:109720008FEF90E10E9425820E949D0D0E94500EB5
:109730006093E40B7093E50B8093E60B9093E70B3B
:109740000E94500E6093DE0B7093DF0B8093E00B52
:109750009093E10BCE014C960E948E2F64EA75E047
:10976000CE0101960E947484BE01645E7F4FCE01DB
:1097700001960E94EF82BC01CE0182960E946B840A
:10978000CE0182960E947A30CE0182960E94D583C5
:10979000CE0101960E94D583CE014C960E94D583BE
:1097A00041CD4BE050E063E271E1CE0101960E94B1
:1097B000AB2DBE016F5F7F4F8FEF90E10E949C83C6
:1097C000CE0101960E94D5838FEF90E10E94258201
:1097D00060587F488F4F9F4FA7CF68E17DE0CE0153
:1097E00001960E946284BE016F5F7F4FCE018E960C
:1097F0000E94BE82182FCE0101960E94D5831123AC
:1098000009F46AC045E050E063E271E1CE010196DF
:109810000E94AB2DBE016F5F7F4F8FEF90E10E94E2
:109820009C83CE0101960E94D5830E94500E6093C6
:10983000E40B7093E50B8093E60B9093E70B8FEFAF
:1098400090E10E94258260936E0270936F02809374
:109850007002909371026093AA127093AB1280937E
:10986000AC129093AD122091A9122093460C672B55
:10987000682B692B11F41092460C84EF91E09093C1
:109880005302809352026AEA71E10E94BF2864E6A3
:1098900070E080E090E00E945E0D69E07DE0CE0126
:1098A00001960E946284CE0101960E94C830CE01CA
:1098B00001960E94D58340916E0250916F02609193
:1098C000700270917102CE0101960E94F881CE0162
:1098D00001960E947A30DBC16EEF7CE0CE010196EA
:1098E0000E946284BE016F5F7F4FCE018E960E9400
:1098F000BE82182FCE0101960E94D5831123D9F183
:109900004AE050E063E271E1CE0101960E94AB2D86
:10991000BE016F5F7F4F8FEF90E10E949C83CE016D
:1099200001960E94D5838FEF90E10E9425826130DD
:1099300071058105910519F481E08093A9128FEFDB
:1099400090E10E942582672B682B692B11F41092FD
:10995000A9128091A9128093460C882309F482CD24
:109960000E94500E6093E40B7093E50B8093E60B1E
:109970009093E70B77CD65EF7CE0CE0101960E94D6
:109980006284BE016F5F7F4FCE018E960E94BE82C1
:10999000182FCE0101960E94D5831123A1F048E033
:1099A00050E063E271E1CE0101960E94AB2DBE0151
:1099B0006F5F7F4F8FEF90E10E949C83CE010196F5
:1099C0000E94D5835FCD6FEE7CE0CE0101960E94B0
:1099D0006284BE016F5F7F4FCE018E960E94BE8271
:1099E000182FCE0101960E94D583112321F145E065
:1099F00050E063E271E1CE0101960E94AB2DBE0101
:109A00006F5F7F4F8FEF90E10E949C83CE010196A4
:109A10000E94D5838FEF90E10E942582613071050D
:109A200021F481E08093470CFDCB672B09F0FACB42
:109A30001092470CF7CB6BEE7CE0CE0101960E94B2
:109A40006284BE016F5F7F4FCE018E960E94BE8200
:109A5000182FCE0101960E94D583112351F163E0A6
:109A600070E083E291E10E948D82682FCE01019621
:109A70000E944084BE016F5F7F4F8FEF90E10E9494
:109A80009C83CE0101960E94D5838FEF90E10E94C6
:109A900030828FEF90E10E9425829B012150310995
:109AA0002330310508F0BECB7093D9126093D812E1
:109AB000A9CB64EE7CE0CE0101960E946284BE01D7
:109AC0006F5F7F4FCE018E960E94BE82182FCE010F
:109AD00001960E94D583112309F46AC066E070E004
:109AE00083E291E10E948D82682FCE0101960E944F
:109AF0004084BE016F5F7F4F8FEF90E10E949C8397
:109B0000CE0101960E94D5838FEF90E10E943082B2
:109B100060E08FEF90E10E942C838FEF90E10E9434
:109B200025826B01CB010197039708F07BCB48E0BE
:109B300050E063E271E1CE0101960E94AB2DBE01BF
:109B40006F5F7F4F8FEF90E10E949C83CE01019663
:109B50000E94D5838FEF90E10E94308280910311A3
:109B6000909104110997A8F028E030E050E040E01F
:109B70006FEF70E1CE0101960E948984BE016F5F94
:109B80007F4F8FEF90E10E949C83CE0101960E944F
:109B9000D583B601B3E0660F771FBA95E1F762543B
:109BA0007E4E48E050E08FEF90E10E94F37F2ACB99
:109BB0006CED7CE0CE0101960E946284BE016F5F75
:109BC0007F4FCE018E960E94BE82182FCE01019645
:109BD0000E94D583112309F486C06DE574E0CE019F
:109BE00001960E94748447E050E0BE01625D7F4FA1
:109BF000CE014C960E94AB2DBE01645E7F4FCE011C
:109C000001960E949C83CE014C960E94D5836BE303
:109C100075E0CE014C960E947484BE01645E7F4F55
:109C2000CE0101960E94BE82182FCE014C960E9452
:109C3000D583112379F141E050E0BE016F5F7F4F82
:109C4000CE014C960E94AB2DCE014C960E942582EF
:109C50008B010A5C1F4FCE014C960E94D583109356
:109C6000DB120093DA12109375020093740284EFF2
:109C700091E090935302809352026AEA71E10E944C
:109C8000BF2864E670E080E090E00E945E0DCE01A7
:109C9000019684CD6DE375E0CE014C960E947484EC
:109CA000BE01645E7F4FCE0101960E94BE82182FD6
:109CB000CE014C960E94D583112379F041E050E00B
:109CC000BE016F5F7F4FCE014C960E94AB2DCE013F
:109CD0004C960E9425828B01BECFCE0101960E9438
:109CE00025828B01BCCF65ED7CE0CE0101960E9400
:109CF0006284BE016F5F7F4FCE018E960E94BE824E
:109D0000182FCE0101960E94D583112309F4AAC011
:109D10006DEB75E0CE0101960E94748446E050E040
:109D2000BE016F5F7F4FCE018E960E9440A98C01CD
:109D3000CE0101960E94D583980146E050E0BE0115
:109D4000625D7F4FCE0101960E948984CE0101960B
:109D50000E9425826B01CE0101960E94D5836DE59C
:109D600074E0CE0101960E947484A8014F5F5F4F9A
:109D7000BE01625D7F4FCE014C960E94AB2DBE01AD
:109D8000645E7F4FCE0101960E949C83CE014C966B
:109D90000E94D5836BE375E0CE014C960E947484DB
:109DA000BE01645E7F4FCE0101960E94BE82182FD5
:109DB000CE014C960E94D583112321F141E050E061
:109DC000BE016F5F7F4FCE014C960E94AB2DCE013E
:109DD0004C960E9425828B010A5C1F4FCE014C9647
:109DE0000E94D583F6013196EE0FFF1FE655FE4E19
:109DF00011830083F601EE0FFF1FE75BF34F118322
:109E0000008335CF6DE375E0CE014C960E947484DB
:109E1000BE01645E7F4FCE0101960E94BE82182F64
:109E2000CE014C960E94D583112379F041E050E099
:109E3000BE016F5F7F4FCE014C960E94AB2DCE01CD
:109E40004C960E9425828B01C9CFCE0101960E94BB
:109E5000258200914B0C10914C0C01501109060FFA
:109E6000171FC0CF6EEC7CE0CE014C960E9462843E
:109E7000BE01645E7F4FCE018E960E94BE8211E0CD
:109E8000811115C067EC7CE0CE0101960E946284CE
:109E9000BE016F5F7F4FCE018E960E94BE8211E0A1
:109EA000811101C010E0CE0101960E94D583CE0140
:109EB0004C960E94D583112309F4F0C16AEB75E03A
:109EC000CE014C960E94748465EB75E0CE0101963C
:109ED0000E947484AE01445E5F4FBE016F5F7F4F8E
:109EE000CE018E960E9447A8CE0101960E94D5838E
:109EF000CE014C960E94D5836AEB75E0CE014C965C
:109F00000E94748467EB75E0CE0101960E94748410
:109F1000AE01445E5F4FBE016F5F7F4FCE018E96F4
:109F20000E9447A8CE0101960E94D583CE014C968F
:109F30000E94D5836AEB75E0CE014C960E94748432
:109F400069EB75E0CE0101960E947484AE01445E17
:109F50005F4FBE016F5F7F4FCE018E960E9447A874
:109F6000CE0101960E94D583CE014C960E94D583E6
:109F70006DEB75E0CE014C960E9474846CEB75E03D
:109F8000CE0101960E947484AE01445E5F4FBE0113
:109F90006F5F7F4FCE018E960E9447A8CE0101963B
:109FA0000E94D583CE014C960E94D5836DEB75E05F
:109FB000CE014C960E94748467ED76E0CE01019646
:109FC0000E947484AE01445E5F4FBE016F5F7F4F9D
:109FD000CE018E960E9447A8CE0101960E94D5839D
:109FE000CE014C960E94D583CE018E960E9430827F
:109FF0000E94500E6093E80B7093E90B8093EA0B7C
:10A000009093EB0B06E010E054E6852E912CA12CEA
:10A01000B12C22242394312C6801B3E0CB0ED11C47
:10A020008AA99BA90197C816D90608F0FBC8B801F0
:10A03000CE018E960E948D82682FCE014C960E9492
:10A0400040847801E2E0EE0EF11C0F5F1F4F970194
:10A05000A801BE01625D7F4FCE0101960E948984F6
:10A06000CE0101960E9425822B01CE0101960E940D
:10A07000D5836AEB75E0CE0101960E947484A70136
:10A08000BE016F5F7F4FCE018E960E9440A97C017A
:10A09000CE0101960E94D5836DE574E0CE01019654
:10A0A0000E947484C20101979DAB8CAB1E141F04E7
:10A0B00024F59701A601BE01625D7F4FCE01829615
:10A0C0000E948984BE016E5D7F4FCE0101960E9481
:10A0D0009C83CE0182960E94D583ACA9BDA913971B
:10A0E00018F187010F5F1F4FCE0101960E94D583A3
:10A0F000CE014C960E94D5838FCFA601BE01625D32
:10A100007F4FCE0182960E94AB2DBE016E5D7F4FC8
:10A11000CE0101960E949C83CE0182960E94D58337
:10A12000ECA9FDA9339700F770E060E0CE014C96F2
:10A130000E948D82823509F050C0CE0101960E94A6
:10A140002582672B682B692BB1F4F201EE0FFF1FFC
:10A15000E952FD4F11821082F201EE0FFF1FEE0F48
:10A16000FF1FE154FD4F82E090E0A0E0B0E080836B
:10A170009183A283B383CE0101960E942582613030
:10A1800071058105910509F067C0F201EE0FFF1F0F
:10A19000E952FD4F31822082440C551C440C551C61
:10A1A000F201E154FD4F80819181A281B3811816A3
:10A1B00019061A061B0624F080829182A282B382BD
:10A1C000CE0101960E9425826230710581059105BC
:10A1D000D4F1F201E154FD4F51C0863409F041C081
:10A1E000CE0101960E942582672B682B692B39F4DA
:10A1F000F201EE0FFF1FEC5AFD4F11821082CE01CB
:10A2000001960E942582613071058105910539F41E
:10A21000F201EE0FFF1FEC5AFD4F31822082440CF9
:10A22000551C440C551CF201E154FD4F8081918175
:10A23000A281B381181619061A061B0624F0808223
:10A240009182A282B3820E94500EF201E152FD4F30
:10A2500060837183828393831E141F040CF441CFA7
:10A2600043CF843481F4CE0101960E942582440CB0
:10A27000551C440C551CF201E45AFD4F6083718358
:10A2800082839383E0CF843539F7CE0101960E9413
:10A290002582440C551C440C551C9BCF61EC7CE082
:10A2A000CE0101960E946284BE016F5F7F4FCE0196
:10A2B0008E960E94BE82082FCE0101960E94D58301
:10A2C000002309F49DC045E050E063E271E1CE0156
:10A2D00001960E94AB2DBE016F5F7F4F8FEF90E123
:10A2E0000E949C83CE0101960E94D5838FEF90E15E
:10A2F0000E94308260E08FEF90E10E942C836FE338
:10A3000075E0CE014C960E9474846FEF70E1CE012F
:10A3100001960E946B84AE014E5D5F4FBE01645E8C
:10A320007F4FCE0101960E945CA9182FCE010196A5
:10A330000E94D583CE014C960E94D583112311F43F
:10A340000C9412498E010E5D1F4F64EDA62E62E142
:10A35000B62E72E4C72E72E0D72EF12CE12CD80174
:10A360006D918D01F50161935F01D6016D936D01D2
:10A37000CE0101960E94C4A7CE0101960E94C8306A
:10A38000CE0101960E94D583B3E0EB16F10471F083
:10A390006FE375E0CE0101960E947484CE010196B0
:10A3A0000E94C830CE0101960E94D583EFEFEE1ACD
:10A3B000FE0AF4E0EF16F10491F66DE574E0CE01CB
:10A3C00001960E947484CE0101960E947A30CE01DB
:10A3D00001960E94D5836AEA71E1809152029091C0
:10A3E00053020E94BF2864E670E080E090E00E9483
:10A3F0005E0D69EA7CE0CE0101960E94628467CA24
:10A4000064EA7CE0CE0101960E946284BE016F5F27
:10A410007F4FCE018E960E94BE82082FCE010196FC
:10A420000E94D583002309F47CC044E050E063E23D
:10A4300071E1CE0101960E94AB2DBE016F5F7F4F8F
:10A440008FEF90E10E949C83CE0101960E94D583FC
:10A450008FEF90E10E94308260E08FEF90E10E94E8
:10A460002C8340910311509104116FE57AE08FEF36
:10A4700090E10E94F37F6FE375E0CE014C960E945D
:10A4800074846FEF70E1CE0101960E946B84AE017F
:10A490004E5D5F4FBE01645E7F4FCE0101960E940C
:10A4A0005CA9182FCE0101960E94D583CE014C964F
:10A4B0000E94D583112311F40C9412498E010E5D74
:10A4C0001F4F56EDE52E51E1F52E6E0186E2C80EC6
:10A4D000D11CD8016D918D01F70161937F01CE01EF
:10A4E00001960E94C4A7CE0101960E947A30CE0147
:10A4F00001960E94D5830C151D0559F784EF91E054
:10A5000090935302809352026AEA71E10E94BF283D
:10A5100064E670E080E090E00E945E0D69E97CE016
:10A520006ACF62E97CE0CE0101960E946284BE019E
:10A530006F5F7F4FCE018E960E94BE82082FCE01A4
:10A5400001960E94D5830023F1F146E050E063E2DA
:10A5500071E1CE0101960E94AB2DBE016F5F7F4F6E
:10A560008FEF90E10E949C83CE0101960E94D583DB
:10A570008FEF90E10E94308280910311909104113D
:10A58000892B11F40C9412498FEF90E10E942582DF
:10A590007093D3126093D212709341026093400281
:10A5A00084EF91E090935302809352026AEA71E142
:10A5B0000E94BF2864E670E080E090E00E945E0D9B
:10A5C0006EE77CE018CF67E77CE0CE0101960E9441
:10A5D0006284BE016F5F7F4FCE018E960E94BE8265
:10A5E000082FCE0101960E94D583002321F16AE64F
:10A5F0007CE0CE0101960E94628444E650E06FEF59
:10A600007FEFCE0101960E942429CE0101960E947F
:10A61000D58381E08093DC1284EF91E09093530224
:10A62000809352026AEA71E10E94BF28F0E0E0E004
:10A6300019950C94124962E67CE0CE0101960E94C5
:10A640006284BE016F5F7F4FCE018E960E94BE82F4
:10A65000082FCE0101960E94D583002309F4ECC097
:10A660008091440C882331F068EB7BE080E090E03F
:10A670000E945E0D8091440C81110C94124963E09C
:10A680007AE186E792E00E942B8064EF71E080E03F
:10A6900090E00E945E0D43E166E772E0CE01019614
:10A6A0000E94F689BE016F5F7F4F87E493E10E94AD
:10A6B000872C11E01093440C87E493E10E94501C16
:10A6C000811109C064E670E080E090E00E945E0DB8
:10A6D00069E47CE090CE6BEE78E087E493E10E9441
:10A6E000A985CE0101960E940D2FBE016F5F7F4F9D
:10A6F00087E493E10E94898569EE78E087E493E13D
:10A700000E94A985CE0101960E94D5836AE070E07F
:10A7100080E090E00E945E0D1093310A6EE170E0DF
:10A7200080E090E00E945E0D8DB79EB7855391400A
:10A730000FB6F8949EBF0FBE8DBFADB7BEB71196D2
:10A7400085E391E0EAEAF1E101900D920197E1F7EA
:10A750000E94A7431092310A0FB6F894DEBF0FBED5
:10A76000CDBF62E370E080E090E00E945E0D87E480
:10A7700093E10E945C1C66E970E080E090E00E943A
:10A780005E0D1092440C66E772E0CE0101960E94C5
:10A790007484BE016F5F7F4F84E491E10E949C83CB
:10A7A000CE0101960E94D58364E471E1CE01019649
:10A7B0000E946B84AE014F5F5F4F64E070E086E7FC
:10A7C00092E00E94B83D9093300A80932F0ACE0108
:10A7D00001960E94D58387E493E10E945C1C66E9A0
:10A7E00070E080E090E00E945E0D1092440C809139
:10A7F0002F0A9091300A019711F40C94124966E5E2
:10A8000071E1CE014C960E946B8464E471E1CE014B
:10A810004C960E94EF82BC01CE0101960E946B848F
:10A82000CE0101960E947A30CE0101960E94D58316
:10A83000CE014C960C945D4A61E47CE0CE01019619
:10A840000E946284BE016F5F7F4FCE018E960E9490
:10A85000BE82082FCE0101960E94D583002301F10C
:10A860006FEB75E0CE0101960E94748463EF72E194
:10A87000CE0101960E94EF82BC0185E091E10E9429
:10A880008583CE0101960E94D58365E071E1CE01FA
:10A8900001960E946B84CE0101960E947A308EC48C
:10A8A0006AE37CE0CE0101960E946284BE016F5F84
:10A8B0007F4FCE018E960E94BE82082FCE01019658
:10A8C0000E94D5830023B1F16BE27CE085E091E149
:10A8D0000E9460836FEF72E189EF92E10E948583AD
:10A8E00069EF72E1CE0101960E946B84BE016F5F39
:10A8F0007F4FCE014C960E946B84CE014C960E94F5
:10A900004083BC0185E091E10E945983CE014C96C1
:10A910000E94D583CE0101960E94D58365E071E146
:10A92000CE0101960E946B84CE0101960E947A307E
:10A930000C940B4B62E27CE0CE0101960E94628493
:10A94000BE016F5F7F4FCE018E960E94BE82082FA0
:10A95000CE0101960E94D583002331F00E947E41F2
:10A9600010923F020C9412496DE17CE0CE010196F9
:10A970000E946284BE016F5F7F4FCE018E960E945F
:10A98000BE82082FCE0101960E94D583002309F4D0
:10A9900041C06DEB75E0CE0101960E947484409138
:10A9A0002711509128118D819E81481B590BBE01A2
:10A9B0006F5F7F4F83E291E10E94F9A7AC014F5F87
:10A9C0005F4F63E271E1CE014C960E94AB2DBE0158
:10A9D000645E7F4F8FEF90E10E949C83CE014C9686
:10A9E0000E94D583CE0101960E94D5838FEF90E11E
:10A9F0000E9425826115710531F481E08093F00297
:10AA00000E94018DADCF6130710509F0A9CF109280
:10AA1000F002F6CF69E17CE0CE0101960E946284EB
:10AA2000BE016F5F7F4FCE018E960E94BE82082FBF
:10AA3000CE0101960E94D583002309F439C143E079
:10AA400050E063E271E1CE0101960E94AB2DBE01A0
:10AA50006F5F7F4F8FEF90E10E949C83CE01019644
:10AA60000E94D5836FEF70E1CE0101960E946B8446
:10AA7000CE0101960E94E12ECE0101960E94D5835F
:10AA800084EF91E090935302809352026FEF70E154
:10AA9000CE0101960E946B84CE0101960E944083F4
:10AAA000BC018FEF92E10E948583CE0101960E9446
:10AAB000D5836FEF70E1CE0101960E946B84CE01C9
:10AAC00001960E944083BC0189EF92E10E94858338
:10AAD000CE0101960E94D583409103135091041337
:10AAE0006AE672E18FEF92E10E94F37F4091FD12DE
:10AAF0005091FE1265E772E189EF92E10E94F37FC7
:10AB00006AEA71E180915202909153020E94BF283B
:10AB10006AEC75E0CE0101960E9474846FEF70E1DB
:10AB2000CE0101960E94EF82BC01CE0182960E9466
:10AB30006B84CE0101960E94D5838091661290911C
:10AB40006712892B39F4BE016E5D7F4F8AEA9EE061
:10AB50000E94898568EB7BE080E090E00E945E0DBA
:10AB60008091661290916712029709F087C06FEF8B
:10AB700070E1CE0188960E946B8462ED75E0CE0193
:10AB800001960E947484CE0101960E942D8DCE0103
:10AB900001960E94D58364EF71E080E090E00E940E
:10ABA0005E0D65ED75E0CE0101960E947484CE01C4
:10ABB00001960E942D8DCE0101960E94D5836CEDE9
:10ABC00075E080E090E00E945E0D6EED75E0CE01D4
:10ABD00001960E947484CE0101960E942D8DCE01B3
:10ABE00001960E94D58364EF71E080E090E00E94BE
:10ABF0005E0D6CEE75E0CE0101960E947484CE016C
:10AC000001960E942D8DCE0101960E94D58364EF9E
:10AC100071E080E090E00E945E0D6AEC75E0CE018C
:10AC200001960E947484BE01685D7F4FCE0101963B
:10AC30000E94EF82BC01CE014C960E946B84CE0133
:10AC400001960E94D583CE014C960E943082BE01AF
:10AC5000645E7F4FCE0101960E946B84CE01019607
:10AC60000E942D8DCE0101960E94D583CE014C9677
:10AC70000E94D583CE0188960E94D58368EB7BE045
:10AC800080E090E00E945E0D6AE672E1CE010196DE
:10AC90000E947484CE0101960E94E12ECE0101969D
:10ACA0000E94D58310923F02CE0182960C94CE4B27
:10ACB00064E17CE0CE0101960E946284BE016F5F78
:10ACC0007F4FCE018E960E94BE82811110915E0A46
:10ACD000CE0101960E94D583112309F486C044E079
:10ACE00050E063E271E1CE0101960E94AB2DBE01FE
:10ACF0006F5F7F4F8FEF90E10E949C83CE010196A2
:10AD00000E94D5836AEF75E0CE0101960E9474849B
:10AD10006FEF70E1CE0101960E94EF82BC01CE017F
:10AD20004C960E946B84CE0101960E94D58380913F
:10AD3000661290916712892B39F4BE01645E7F4FD1
:10AD40008AEA9EE00E94898568E873E180E090E0ED
:10AD50000E945E0D8091661290916712029759F5DC
:10AD600061E076E0CE0101960E9474848091031127
:10AD700090910411892B19F56AE076E0CE010196D5
:10AD80000E94C281BE01645E7F4FCE0182960E9406
:10AD90006B84CE0182960E942D8DCE0182960E94F8
:10ADA000D58368E873E180E090E00E945E0DCE01FB
:10ADB00001960E94D58310923F020C94CC4BBE01A9
:10ADC0006F5F7F4FCE0182960E946B84CE01829688
:10ADD0000E942D8DCE0182960E94D58360E777E197
:10ADE00080E090E00E945E0DCDCF60E17CE0CE017E
:10ADF00001960E946284BE016F5F7F4FCE018E96E6
:10AE00000E94BE82811110915E0ACE0101960E94BD
:10AE1000D583112309F462C063E271E18FEF90E101
:10AE20000E94858381E080933F0263E271E1CE015D
:10AE300001960E946B84CE0101960E94E12ECE0104
:10AE400001960E94D58380916612909167120297B5
:10AE500009F16FEF70E18AEA9EE00E94898568EB54
:10AE60007BE080E090E00E945E0DCE0101960E94A2
:10AE7000C68DBE016F5F7F4F83E291E10E949C838C
:10AE8000CE0101960E94D58360ED77E080E090E0EE
:10AE90000E945E0D8091661290916712029771F484
:10AEA0006FEF70E1CE0101960E946B84CE01019696
:10AEB0000E942D8DCE0101960E94D583809127118D
:10AEC00090912811892B09F44BCD65E876E0CE01ED
:10AED00001960E94748463E271E1A2C46AE07CE09E
:10AEE000CE0101960E946284BE016F5F7F4FCE014A
:10AEF0008E960E94BE82182FCE0101960E94D583A5
:10AF0000112309F495C180916612909167120197FF
:10AF100009F026CD63E176E0CE0188960E94748424
:10AF2000BE01685D7F4F8AEA9EE00E9489856CE2DF
:10AF300071E080E090E00E945E0DCE0182960E945A
:10AF4000C68D64E670E080E090E00E945E0D10E047
:10AF500000E035E0C32ED12C4AE0A42EB12C6EE1E6
:10AF600076E0CE0101960E94748450E040E0BE017C
:10AF70006F5F7F4FCE0182960E9440A97C01CE0177
:10AF800001960E94D583A7014F5F5F4FBE016E5DA2
:10AF90007F4FCE0101960E94AB2DBE016F5F7F4FA8
:10AFA000CE0188960E949C83CE0101960E94D58393
:10AFB0008CA59DA5892B09F170E060E0CE018896F3
:10AFC0000E948D82082E000C990BC0970A97A8F456
:10AFD00060E276E0CE0101960E947484BE016F5F4C
:10AFE0007F4FCE0188960E94BE82E82ECE01019648
:10AFF0000E94D583FF24F394E110F12C6DEF78E0EB
:10B00000CE0101960E94628464E170E0CE01019657
:10B010000E9416AACE0101960E94D5830F5F1F4F92
:10B0200062E370E080E090E00E945E0DC801B6012E
:10B030000E9433B60197C1F4CE0101960E94893275
:10B040008D819E81892B09F4BEC0BE016F5F7F4F49
:10B0500083E291E10E9485830E94F947FF24F394E3
:10B06000CE0101960E94D583CE0101960E94C68D25
:10B07000BE016F5F7F4FCE0182960E949C83CE01FE
:10B0800001960E94D58362E370E080E090E00E9428
:10B090005E0D0436110519F0FF2009F460CF809190
:10B0A000CD0B8823F1F065E876E0CE014C960E9446
:10B0B0007484BE01685D7F4FCE014C960E94EF8282
:10B0C000BC01CE0101960E946B84CE0101960E94C4
:10B0D0007A30CE0101960E94D583CE014C960E9413
:10B0E000D5838CA59DA5892B69F070E060E0CE0129
:10B0F00088960E948D82082E000C990BC0970A97A3
:10B1000008F47AC068E276E0CE0101960E94748469
:10B11000CE0182960E94D583CE0188960E94D58367
:10B120008D819E81009709F449C0E981FA812081CF
:10B13000222309F443C0079708F440C061E07CE093
:10B14000CE014C960E94628468EC70E0CE014C9671
:10B150000E9416AACE014C960E94D583BE016F5F55
:10B160007F4FCE014C960E946B8440ED57E06FEF0D
:10B170007FEFCE014C960E942429CE014C960E946E
:10B18000D58364E376E0CE014C960E94748463E23A
:10B1900071E1CE014C960E94EF82BC01CE018296F5
:10B1A0000E946B84CE0182960E947A30CE018296F4
:10B1B0000E94D583CE014C960E94D583CE01019684
:10B1C0000E94D583CDCB043111050CF449CFC801C1
:10B1D000B5010E9433B6892B09F042CFBE01685DEC
:10B1E0007F4F8AEA9EE00E94898568EC70E080E0EB
:10B1F00090E00E945E0D34CF60E276E0CE010196D1
:10B200000E947484BE016F5F7F4FCE0188960E94BA
:10B21000BE82182FCE0101960E94D583111172CFE4
:10B22000BE01685D7F4FCE0101960E94598470CFA8
:10B230006CEF7BE0CE0101960E946284BE016F5FDD
:10B240007F4FCE018E960E94BE82182FCE010196AE
:10B250000E94D583112309F4F7C025E030E044E0D3
:10B2600050E063E271E1CE0101960E948984BE0143
:10B270006F5F7F4F8FEF90E10E949C83CE0101961C
:10B280000E94D58363E271E1CE0101960E946B8436
:10B29000CE0101960E94E12ECE0101960E94D58337
:10B2A0008FEF90E10E9425826130710509F06EC038
:10B2B00070936712609366126CE279E0CE0101969A
:10B2C0000E946284CE0101960E94E12ECE01019679
:10B2D0000E94D58362E476E0CE014C960E9474848D
:10B2E00069EF72E1CE014C960E94EF82BC01CE0163
:10B2F00001960E946B8448EC50E06FEF7FEFCE0127
:10B3000001960E947536CE0101960E94D583CE012A
:10B310004C960E94D5830E94A7A740E052EC61E0C2
:10B3200070E08AEA9EE00E94B17B84EF91E0909306
:10B3300053028093520281E080935E0A6AEA71E1CF
:10B3400084EF91E00E94BF2861E576E0CE014C9643
:10B350000E94748463EF72E1CE014C960E94EF82EA
:10B36000BC01CE0101960E946B8440ED57E06FEF67
:10B370007FEFCE0101960E942429CE0101960E9402
:10B38000D583CE014C960E94D583EACA611571051A
:10B39000D1F510926712109266126EE179E0CE013B
:10B3A00001960E946284CE0101960E94E12ECE0198
:10B3B00001960E94D58368E476E0CE014C960E9407
:10B3C000748469EF72E1CE014C960E94EF82BC0159
:10B3D000CE0101960E946B8448EC50E06FEF7FEF46
:10B3E000CE0101960E947536CE0101960E94D5834A
:10B3F000CE014C960E94D5830E94A7A740E855E253
:10B4000060E070E08ECF62307105A9F4709367122E
:10B41000609366126DE079E0CE0101960E9462842D
:10B42000CE0101960E94E12ECE0101960E94D583A5
:10B430006CE476E0C2CF77FF93CA10925E0A7093F5
:10B440006712609366128CCA64EF7BE0CE010196AE
:10B450000E946284BE016F5F7F4FCE018E960E9474
:10B46000BE82182FCE0101960E94D583112309F4C4
:10B4700041C047E050E063E271E1CE0101960E94D5
:10B48000AB2DBE016F5F7F4F8FEF90E10E949C83D9
:10B49000CE0101960E94D58366E276E0CE01019648
:10B4A0000E947484BE016F5F7F4F8FEF90E10E9416
:10B4B000BE82182FCE0101960E94D58311111092E1
:10B4C000450C64E275E0CE0101960E947484BE01D1
:10B4D0006F5F7F4F8FEF90E10E94BE82182FCE01E9
:10B4E00001960E94D583112309F4EFCC81E080936B
:10B4F000450CEBCC6DEE7BE0CE0101960E946284A0
:10B50000BE016F5F7F4FCE018E960E94BE82182FC4
:10B51000CE0101960E94D583112381F146E050E0CF
:10B5200063E271E1CE0101960E94AB2DBE016F5F17
:10B530007F4F8FEF90E10E949C83CE0101960E9485
:10B54000D5838FEF90E10E94EEA76093AE127093C7
:10B55000AF128093B0129093B11284EF91E0909368
:10B560005302809352026AEA71E10E94BF2864E6A6
:10B5700070E080E090E00E945E0DA7CC64EE7BE07E
:10B58000CE0101960E946284BE016F5F7F4FCE01A3
:10B590008E960E94BE82182FCE0101960E94D583FE
:10B5A000112301F148E050E063E271E1CE01019620
:10B5B0000E94AB2DBE016F5F7F4F8FEF90E10E9425
:10B5C0009C83CE0101960E94D5838FEF90E10E946B
:10B5D000EEA76093B4127093B5128093B612909355
:10B5E000B712BBCF6AED7BE0CE0101960E94628468
:10B5F000BE016F5F7F4FCE018E960E94BE82182FD4
:10B60000CE0101960E94D583112301F149E050E05B
:10B6100063E271E1CE0101960E94AB2DBE016F5F26
:10B620007F4F8FEF90E10E949C83CE0101960E9494
:10B63000D5838FEF90E10E94EEA76093B8127093CC
:10B64000B9128093BA129093BB1287CF60ED7BE062
:10B65000CE0101960E946284BE016F5F7F4FCE01D2
:10B660008E960E94BE82182FCE0101960E94D5832D
:10B670001123F1F049E050E063E271E1CE0101965F
:10B680000E94AB2DBE016F5F7F4F8FEF90E10E9454
:10B690009C83CE0101960E94D5838FEF90E10E949A
:10B6A000EEA70E94F3B57093BF126093BE1255CF00
:10B6B00065EC7BE0CE0101960E946284BE016F5F63
:10B6C0007F4FCE018E960E94BE82182FCE0101962A
:10B6D0000E94D5831123F1F04AE050E063E271E16A
:10B6E000CE0101960E94AB2DBE016F5F7F4F8FEFA1
:10B6F00090E10E949C83CE0101960E94D5838FEF3A
:10B7000090E10E94EEA70E94F3B57093BD12609382
:10B71000BC1223CF69EB7BE0CE0101960E946284CC
:10B72000BE016F5F7F4FCE018E960E94BE82182FA2
:10B73000CE0101960E94D583112311F14BE050E018
:10B7400063E271E1CE0101960E94AB2DBE016F5FF5
:10B750007F4F8FEF90E10E949C83CE0101960E9463
:10B76000D5838FEF90E10E94EEA70E94F3B560931E
:10B77000C0127093C1128093C2129093C312EDCE87
:10B7800062EB7BE0CE0101960E946284BE016F5F96
:10B790007F4FCE018E960E94BE82182FCE01019659
:10B7A0000E94D583112309F44FC046E050E063E2C4
:10B7B00071E1CE0101960E94AB2DBE016F5F7F4FFC
:10B7C0008FEF90E10E949C83CE0101960E94D58369
:10B7D0008FEF90E10E9425827093B3116093B211B4
:10B7E0008FEF90E10E9425827093520C6093510C70
:10B7F00084EF91E090935302809352026AEA71E1E0
:10B800000E94BF2864E670E080E090E00E945E0D38
:10B8100066E576E0CE0101960E9474846FEF70E1D8
:10B82000CE0101960E94EF82BC01CE014C960E948F
:10B830006B84CE014C960E947A30CE014C960E94C9
:10B84000D583CE0101969FCD6AEA7BE0CE010196B9
:10B850000E946284BE016F5F7F4FCE018E960E9470
:10B86000BE82182FCE0101960E94D5831123B1F11B
:10B8700047E050E063E271E1CE0101960E94AB2DFA
:10B88000BE016F5F7F4F8FEF90E10E949C83CE01DE
:10B8900001960E94D5838FEF90E10E9425827093DC
:10B8A000B5116093B4118FEF90E10E9425827093DF
:10B8B000540C6093530C84EF91E090935302809367
:10B8C00052026AEA71E10E94BF2864E670E080E0FB
:10B8D00090E00E945E0D62E676E09CCF64EA7BE039
:10B8E000CE0101960E946284BE016F5F7F4FCE0140
:10B8F0008E960E94BE82182FCE0101960E94D5839B
:10B900001123E1F045E050E063E271E1CE010196E0
:10B910000E94AB2DBE016F5F7F4F8FEF90E10E94C1
:10B920009C83CE0101960E94D5838FEF90E10E9407
:10B9300025827093B3126093B2120FCE6EE97BE052
:10B94000CE0101960E946284BE016F5F7F4FCE01DF
:10B950008E960E94BE82182FCE0101960E94D5833A
:10B96000112361F00E94500E6093E80B7093E90B75
:10B970008093EA0B9093EB0B0C94B0546AE97BE054
:10B98000CE0101960E946284BE016F5F7F4FCE019F
:10B990008E960E94BE82182FCE0101960E94D583FA
:10B9A000112389F143E050E0BE01625D7F4FCE017B
:10B9B00001960E94AB2DBE016F5F7F4F8FEF90E12C
:10B9C0000E949C83CE0101960E94D5838091031131
:10B9D00090910411892B41F08FEF90E10E94258214
:10B9E00070936D0260936C0280916C0290916D0275
:10B9F0000197029708F469CA81E090E090936D0284
:10BA000080936C0262CA63E97BE0CE014C960E948F
:10BA10006284BE01645E7F4FCE018E960E94BE821C
:10BA200011E0811115C060E97BE0CE0101960E9412
:10BA30006284BE016F5F7F4FCE018E960E94BE82F0
:10BA400011E0811101C010E0CE0101960E94D58362
:10BA5000CE014C960E94D583112309F468C069E891
:10BA60007BE0CE0101960E946284BE016F5F7F4F32
:10BA7000CE018E960E94BE82182FCE0101960E94A2
:10BA8000D5831123A1F046E050E0BE01625D7F4FF7
:10BA9000CE0101960E94AB2DBE016F5F7F4F8FEFED
:10BAA00090E10E949C83CE0101960E94D58366E8B6
:10BAB0007BE0CE0101960E946284BE016F5F7F4FE2
:10BAC000CE018E960E94BE82182FCE0101960E9452
:10BAD000D5831123A1F042E050E0BE01625D7F4FAB
:10BAE000CE0101960E94AB2DBE016F5F7F4F8FEF9D
:10BAF00090E10E949C83CE0101960E94D5838091A3
:10BB0000031190910411892B09F4DFC96FEF70E1E3
:10BB1000CE0101960E946B8461E070E0CE01019637
:10BB20000E94678ECE0101960E94D583CEC96FE731
:10BB30007BE0CE0182960E946284BE016E5D7F4FE3
:10BB4000CE018E960E94BE8211E0811129C067E766
:10BB50007BE0CE014C960E946284BE01645E7F4F02
:10BB6000CE018E960E94BE8211E0811115C06FE653
:10BB70007BE0CE0101960E946284BE016F5F7F4F21
:10BB8000CE018E960E94BE8211E0811101C010E0AC
:10BB9000CE0101960E94D583CE014C960E94D5839A
:10BBA000CE0182960E94D583112309F4E6C068E68F
:10BBB0007BE0CE0101960E946284BE016F5F7F4FE1
:10BBC000CE018E960E94BE82182FCE0101960E9451
:10BBD000D583112309F466C046E050E0BE01625DE2
:10BBE0007F4FCE0101960E94AB2DBE016F5F7F4F4C
:10BBF0008FEF90E10E949C83CE0101960E94D58335
:10BC00008FEF90E10E94EEA76B017C0120E030E015
:10BC1000A9010E9429B618160CF08EC0A701960142
:10BC200060E070E08AE794E40E9481B50E94F3B579
:10BC300060933B0270933C0280933D0290933E02DE
:10BC400080913B0290913C02A0913D02B0913E0256
:10BC5000181619061A061B0664F081E090E0A0E0B1
:10BC6000B0E080933B0290933C02A0933D02B093DE
:10BC70003E0280916C0290916D028130910509F035
:10BC800068C080913B0290913C02A0913D02B0912E
:10BC90003E028093370290933802A0933902B0930A
:10BCA0003A0213C947E050E0BE01625D7F4FCE010A
:10BCB00001960E94AB2DBE016F5F7F4F8FEF90E129
:10BCC0000E949C83CE0101960E94D5836CE974E0AA
:10BCD000CE0101960E947484BE016F5F7F4FCE013A
:10BCE0008E960E94BE82182FCE0101960E94D583A7
:10BCF000112331F081E090E090936D0280936C020B
:10BD000063ED75E0CE0101960E947484BE016F5F01
:10BD10007F4FCE018E960E94BE82182FCE010196D3
:10BD20000E94D583112309F46BCF82E090E09093B9
:10BD30006D0280936C0264CF81E090E0A0E0B0E0FF
:10BD400080933B0290933C02A0933D02B0933E024D
:10BD500077CF029709F0B9C880913B0290913C02DD
:10BD6000A0913D02B0913E02809333029093340241
:10BD7000A0933502B0933602A8C863E67BE0CE01FB
:10BD80004C960E946284BE01645E7F4FCE018E9607
:10BD90000E949E8211E0811115C06CE57BE0CE010E
:10BDA00001960E946284BE016F5F7F4FCE018E9626
:10BDB0000E94BE8211E0811101C010E0CE01019607
:10BDC0000E94D583CE014C960E94D583112309F49D
:10BDD0008EC268E57BE0CE0101960E946284BE01BE
:10BDE0006F5F7F4FCE018E960E94BE82182FCE01CC
:10BDF00001960E94D583112309F4FCC001E010E0F4
:10BE000010936D0200936C02109332020093310282
:10BE10006FE676E08FEF90E10E94C28110933202CC
:10BE20000093310281E090E0A0E0B0E080933B021B
:10BE300090933C02A0933D02B0933E028093370260
:10BE400090933802A0933902B0933A026FEF70E1F9
:10BE5000CE0101960E946B8462E070E0CE010196F3
:10BE60000E94678ECE0101960E94D58367E47BE035
:10BE7000CE0101960E946284CE0101960E947A3022
:10BE8000CE0101960E94D58367E37BE0CE01019647
:10BE90000E946284CE0101960E944A37CE0101962B
:10BEA0000E94D58366E276E08FEF90E10E94C28126
:10BEB0006FEF70E1CE0101960E946B8463E070E049
:10BEC000CE0101960E94678ECE0101960E94D58315
:10BED00082E090E090936D0280936C0266E27BE0DA
:10BEE000CE0101960E946284CE0101960E947A30B2
:10BEF000CE0101960E94D5836AE17BE0CE010196D6
:10BF00000E946284CE0101960E944A37CE010196BA
:10BF10000E94D5836FE676E08FEF90E10E94C281A8
:10BF20008091D0129091D11297FF06C063E776E01E
:10BF30008FEF90E10E94C2816FEF70E1CE01019618
:10BF40000E946B8462E070E0CE0101960E94678ED1
:10BF5000CE0101960E94D58366E276E08FEF90E1F4
:10BF60000E94C28182E090E090936D0280936C0207
:10BF70006FEF70E1CE0101960E946B8463E070E088
:10BF8000CE0101960E94678ECE0101960E94D58354
:10BF900084EF91E090935302809352026AEA71E138
:10BFA0000E94BF2864E670E080E090E00E945E0D91
:10BFB00081E090E090936D0280936C021092DA021F
:10BFC0001092D90282E090E0A0E0B0E08093C3023A
:10BFD0009093C402A093C502B093C6020E94500E73
:10BFE0006093E3027093E4028093E5029093E6028B
:10BFF0000C94655765E17BE0CE0101960E94628456
:10C00000BE016F5F7F4FCE018E960E94BE82182FB9
:10C01000CE0101960E94D58311110C94655763E1FE
:10C020007BE0CE0101960E946284BE016F5F7F4F6C
:10C03000CE018E960E94BE82182FCE0101960E94DC
:10C04000D583112331F081E090E090936D028093CD
:10C050006C0261E17BE0CE0101960E946284BE0128
:10C060006F5F7F4FCE018E960E94BE82182FCE0149
:10C0700001960E94D583112331F082E090E09093E5
:10C080006D0280936C0281E090E0A0E0B0E08093CC
:10C090003B0290933C02A0933D02B0933E028091FC
:10C0A0006C0290916D028130910509F099C09093D6
:10C0B0003202809331026AE07BE0CE0101960E9459
:10C0C0006284BE016F5F7F4FCE018E960E94BE825A
:10C0D000182FCE0101960E94D583112319F146E055
:10C0E00050E0BE01625D7F4FCE014C960E94AB2DA9
:10C0F00067E776E0CE0101960E947484BE01645E1B
:10C100007F4FCE0101960E94EF82BC018FEF90E13C
:10C110000E948583CE0101960E94D583CE014C9664
:10C120000E94D58380913B0290913C02A0913D02F8
:10C13000B0913E028093370290933802A093390267
:10C14000B0933A026FE676E08FEF90E10E94C281F1
:10C150006FEF70E1CE0101960E946B8462E070E0A7
:10C16000CE0101960E94678ECE0101960E94D58372
:10C1700069EF7AE0CE0101960E946284CE010196B9
:10C180000E947A30CE0101960E94D58381E090E032
:10C19000909332028093310266E276E08FEF90E175
:10C1A0000E94C2816FEF70E1CE0101960E946B8404
:10C1B00063E070E0CE0101960E94678ECE01019689
:10C1C0000E94D58369EE7AE0CE0101960E946284D6
:10C1D000CE0101960E944A37CE0101960E94D58376
:10C1E00080916C0290916D02029711F00C9465574A
:10C1F00065EE7AE08FEF90E10E9460838091D0122B
:10C200009091D11297FF06C061EE7AE08FEF90E136
:10C210000E94608301E010E010933202009331022B
:10C220006FEF70E1CE0101960E946B8462E070E0D6
:10C23000CE0101960E94678ECE0101960E94D583A1
:10C2400066E276E08FEF90E10E94C28160ED7AE0D5
:10C25000CE0101960E946284CE0101960E947A303E
:10C26000CE0101960E94D5836FEF70E1CE01019659
:10C270000E946B8463E070E0CE0101960E94678E9D
:10C28000CE0101960E94D58364EC7AE0CE0101963E
:10C290000E946284CE0101960E944A37CE01019627
:10C2A0000E94D5838091D0129091D1129195819561
:10C2B00091099093D1128093D0121093320200937F
:10C2C000310284EF91E090935302809352026AEA24
:10C2D00071E10E94BF2864E670E080E090E00E9477
:10C2E0005E0D10936D0200936C020C9465576DEB1C
:10C2F0007AE0CE0188960E946284BE01685D7F4F1D
:10C30000CE018E960E94BE8201E081113DC06AEB93
:10C310007AE0CE0182960E946284BE016E5D7F4FFC
:10C32000CE018E960E94BE8201E0811129C066EB8B
:10C330007AE0CE014C960E946284BE01645E7F4F1B
:10C34000CE018E960E94BE8201E0811115C062EB83
:10C350007AE0CE0101960E946284BE016F5F7F4F3A
:10C36000CE018E960E94BE8201E0811101C000E0E4
:10C37000CE0101960E94D583CE014C960E94D583B2
:10C38000CE0182960E94D583CE0188960E94D583E5
:10C39000002309F41FC26BEA7AE0CE0101960E94E5
:10C3A0006284BE016F5F7F4FCE018E960E94BE8277
:10C3B000082FCE0101960E94D58346E050E001117E
:10C3C00017C069E776E0CE0101960E947484BE0131
:10C3D0006F5F7F4FCE018E960E94BE82082FCE01E6
:10C3E00001960E94D583002309F48BC042E050E0FF
:10C3F000BE01625D7F4FCE0101960E94AB2DBE0152
:10C400006F5F7F4F8FEF90E10E949C83CE0101967A
:10C410000E94D5838091031190910411892B11F40E
:10C420000C94655767E776E0CE014C960E947484C1
:10C43000BE01645E7F4F8FEF90E10E94BE8281114A
:10C4400014C069EA7AE0CE0101960E946284BE01BE
:10C450006F5F7F4F8FEF90E10E94BE8211E08111EC
:10C4600010E0CE0101960E94D583CE014C960E9429
:10C47000D583C12CD12C7601112309F46AC18FEF29
:10C4800090E10E94EEA76B017C0180916C0290917B
:10C490006D02019709F09FC08FEF90E10E94EEA717
:10C4A0009B01AC0160915A0A70915B0A80915C0A11
:10C4B00090915D0A0E9415B560935A0A70935B0AC9
:10C4C00080935C0A90935D0A80905A0A90905B0A70
:10C4D000A0905C0AB0905D0A20E030E044EB53E4A9
:10C4E000C501B4010E9429B687FD86C020E030E076
:10C4F00044EB53E4C501B4010E9414B54B015C0147
:10C50000EBCF43E050E0BE01625D7F4FCE0101966C
:10C510000E94AB2DBE016F5F7F4F8FEF90E10E94B5
:10C520009C83CE0101960E94D5836CE974E0CE0114
:10C5300001960E947484BE016F5F7F4FCE018E967C
:10C540000E94BE82082FCE0101960E94D58300234F
:10C55000B1F081E090E090936D0280936C02809145
:10C56000D60B9091D70BA091D80BB091D90B80939B
:10C570005A0A90935B0AA0935C0AB0935D0A63ED3C
:10C5800075E0CE0101960E947484BE016F5F7F4FFB
:10C59000CE018E960E94BE82082FCE0101960E9487
:10C5A000D583002309F436CF82E090E090936D02AA
:10C5B00080936C028091D20B9091D30BA091D40BFD
:10C5C000B091D50B80935A0A90935B0AA0935C0AB2
:10C5D000B0935D0A1FCF8FEF90E10E94EEA79B0101
:10C5E000AC0160915A0A70915B0A80915C0A90914B
:10C5F0005D0A0E9414B560CF20E030E0A901C501BA
:10C60000B4010E9467B387FF0BC020E030E044EB29
:10C6100053E4C501B4010E9415B54B015C01ECCF98
:10C6200080925A0A90925B0AA0925C0AB0925D0ACC
:10C6300020E030E0A901C701B6010E9429B687FDBC
:10C6400015C067E277E0CE0101960E9474846FEF17
:10C6500070E1CE0101960E94EF82BC018FEF90E164
:10C660000E948583CE0101960E94D58320E030E0B0
:10C67000A901C701B6010E9467B387FF6AC0809114
:10C680006C0290916D02019799F520E030E0A901CC
:10C69000C701B6010E9429B618160CF092C020E01E
:10C6A00030E040E251E4C701B6010E9415B522E036
:10C6B000AB01BC01CE014C960E94DD8367E776E0BA
:10C6C000CE0101960E947484BE01645E7F4FCE014C
:10C6D00001960E94EF82BC018FEF90E10E9485835A
:10C6E000CE0101960E94D583CE014C960E94D5833F
:10C6F00080916C0290916D02019759F120E030E039
:10C70000A901C701B6010E9429B6B701A6011816F2
:10C710000CF0705822E0CE014C960E94DD8367E752
:10C7200076E0CE0101960E947484BE01645E7F4F64
:10C73000CE0101960E94EF82BC018FEF90E10E9432
:10C740008583CE0101960E94D583CE014C960E942E
:10C75000D58381E090E090933202809331026FEFB5
:10C7600070E1CE0101960E946B8462E070E0CE0120
:10C7700001960E94678ECE0101960E94D58320E02B
:10C7800030E0A901C701B6010E9467B387FD02C06E
:10C790000C94655780916C0290916D02019711F095
:10C7A0000C9465576CE776E08FEF90E10E94C281B0
:10C7B0006FEF70E1CE0101960E946B8462E070E041
:10C7C000ADC9A701960160E070E080E291E40E94AB
:10C7D00014B56DCF63EA7AE0CE0182960E9462843E
:10C7E000BE016E5D7F4FCE018E960E94BE8211E02B
:10C7F000811129C06CE97AE0CE014C960E946284D6
:10C80000BE01645E7F4FCE018E960E94BE8211E013
:10C81000811115C065E97AE0CE0101960E9462841B
:10C82000BE016F5F7F4FCE018E960E94BE8211E0E7
:10C83000811101C010E0CE0101960E94D583CE0186
:10C840004C960E94D583CE0182960E94D5831123F7
:10C8500009F49BC0CE018E960E9430826FE676E08E
:10C860008FEF90E10E94C2816CE974E0CE010196E5
:10C870000E947484BE016F5F7F4FCE018E960E942E
:10C88000BE82182FCE0101960E94D583112331F06C
:10C8900081E090E090936D0280936C0263ED75E00F
:10C8A000CE0101960E947484BE016F5F7F4FCE015E
:10C8B0008E960E94BE82182FCE0101960E94D583CB
:10C8C000112391F082E090E090936D0280936C02CE
:10C8D0008091D0129091D11297FF06C061E97AE061
:10C8E0008FEF90E10E94608381E090E090933202AC
:10C8F000809331026FEF70E1CE0101960E946B844C
:10C9000062E070E0CE0101960E94678ECE01019632
:10C910000E94D5836BE87AE0CE0101960E94628482
:10C92000BE016F5F7F4FCE018E960E94BE82182F90
:10C93000CE0101960E94D58345E050E0111102C05E
:10C9400046E050E0BE01625D7F4FCE0101960E943D
:10C95000AB2DBE016F5F7F4F8FEF90E10E949C83F4
:10C96000CE0101960E94D58380910311909104110C
:10C97000892B11F40C9465576FEF70E1CE0101968D
:10C980000E946B8463E070E0C9C865E87AE0CE017C
:10C9900082960E946284BE016E5D7F4FCE018E96AC
:10C9A0000E94BE8211E0811129C06EE77AE0CE01BB
:10C9B0004C960E946284BE01645E7F4FCE018E96CB
:10C9C0000E94BE8211E0811115C067E77AE0CE01B6
:10C9D00001960E946284BE016F5F7F4FCE018E96EA
:10C9E0000E94BE8211E0811101C010E0CE010196CB
:10C9F0000E94D583CE014C960E94D583CE018296AB
:10CA00000E94D583112309F426C161E77AE0CE01A3
:10CA100001960E946284BE016F5F7F4FCE018E96A9
:10CA20000E94BE82182FCE0101960E94D583112349
:10CA300009F443C045E050E0BE01625D7F4FCE0186
:10CA400001960E94AB2DBE016F5F7F4F8FEF90E18B
:10CA50000E949C83CE0101960E94D5838091031190
:10CA600090910411892B61F08FEF90E10E94EEA765
:10CA700060935A0A70935B0A80935C0A90935D0AF4
:10CA8000C0905A0AD0905B0AE0905C0AF0905D0A70
:10CA900020E030E044EB53E4C701B6010E9429B620
:10CAA00087FD55C020E030E044EB53E4C701B601F8
:10CAB0000E9414B56B017C01EBCF46E050E0BE0153
:10CAC000625D7F4FCE0101960E94AB2DBE016F5F6C
:10CAD0007F4F8FEF90E10E949C83CE0101960E94D0
:10CAE000D5836CE974E0CE0101960E947484BE0186
:10CAF0006F5F7F4FCE018E960E94BE82182FCE01AF
:10CB000001960E94D583112331F081E090E090934B
:10CB10006D0280936C0263ED75E0CE0101960E9478
:10CB20007484BE016F5F7F4FCE018E960E94BE82DD
:10CB3000182FCE0101960E94D583112309F48ECFC0
:10CB400082E090E090936D0280936C0287CF20E0AA
:10CB500030E0A901C701B6010E9467B387FF0BC08F
:10CB600020E030E044EB53E4C701B6010E9415B564
:10CB70006B017C01ECCFC0925A0AD0925B0AE09222
:10CB80005C0AF0925D0A80916C0290916D020197AF
:10CB900071F4C092D60BD092D70BE092D80BF092E2
:10CBA000D90B66E67AE085E091E10E94608380918E
:10CBB0005A0A90915B0AA0915C0AB0915D0A20919B
:10CBC0006C0230916D022230310571F48093D20BEA
:10CBD0009093D30BA093D40BB093D50B6FE57AE071
:10CBE00085E091E10E94608340915A0A50915B0A6E
:10CBF00060915C0A70915D0A21E0CE014C960E9422
:10CC0000DD8365E071E1CE0101960E946B84BE0177
:10CC1000645E7F4FCE0101960E94EF8268E575E069
:10CC20000E94D982BC0185E091E10E948583CE01FA
:10CC300001960E94D583CE014C960E94D58365E073
:10CC400071E1CE0101960E946B84CE0101960E9493
:10CC50004A370C94925D6AE57AE0CE0182960E9492
:10CC60006284BE016E5D7F4FCE018E960E94BE82B1
:10CC700011E0811129C064E57AE0CE014C960E9452
:10CC80006284BE01645E7F4FCE018E960E94BE829A
:10CC900011E0811115C06EE47AE0CE0101960E9488
:10CCA0006284BE016F5F7F4FCE018E960E94BE826E
:10CCB00011E0811101C010E0CE0101960E94D583E0
:10CCC000CE014C960E94D583CE0182960E94D583D8
:10CCD000112309F412C2C0903B02D0903C02E090B4
:10CCE0003D02F0903E0269E47AE0CE0101960E9496
:10CCF0006284BE016F5F7F4FCE018E960E94BE821E
:10CD0000182FCE0101960E94D583112309F465C026
:10CD100044E050E0BE01625D7F4FCE0101960E946B
:10CD2000AB2DBE016F5F7F4F8FEF90E10E949C8320
:10CD3000CE0101960E94D58380916C0290916D0284
:10CD40008130910509F093C0C0903702D09038022D
:10CD5000E0903902F0903A0281E090E0A0E0B0E08B
:10CD60008093370290933802A0933902B0933A022D
:10CD70008091031190910411892B09F090C063E414
:10CD80007AE08FEF90E10E9460838091031190918F
:10CD90000411892B81F06FEF70E1CE0101960E94A2
:10CDA0006B8470E060E0CE0101960E94678ECE0138
:10CDB00001960E94D58380916C0290916D02813022
:10CDC000910509F08CC1C0923702D0923802E092EE
:10CDD0003902F0923A020C94655745E050E0BE01EA
:10CDE000625D7F4FCE0101960E94AB2DBE016F5F49
:10CDF0007F4F8FEF90E10E949C83CE0101960E94AD
:10CE0000D5836CE974E0CE0101960E947484BE0162
:10CE10006F5F7F4FCE018E960E94BE82182FCE018B
:10CE200001960E94D583112331F081E090E0909328
:10CE30006D0280936C0263ED75E0CE0101960E9455
:10CE40007484BE016F5F7F4FCE018E960E94BE82BA
:10CE5000182FCE0101960E94D583112309F46CCFBF
:10CE600082E090E090936D0280936C0265CF029710
:10CE700009F07ECFC0903302D0903402E0903502AA
:10CE8000F090360281E090E0A0E0B0E080933302C1
:10CE900090933402A0933502B093360269CF60E8D4
:10CEA00076E0CE0101960E947484BE016F5F7F4FD1
:10CEB0008FEF90E10E949E82182FCE0101960E9472
:10CEC000D583112309F477CF8FEF90E10E94EEA76D
:10CED00020E030E0A9010E9467B3811128C0809151
:10CEE0006C0290916D02019731F46EE37AE08FEF5E
:10CEF00090E10E94608380916C0290916D02029794
:10CF000031F468E37AE08FEF90E10E9460838091D2
:10CF1000031190910411892B09F44DCF6FEF70E14B
:10CF2000CE0101960E946B8461E070E03CCF6DEB16
:10CF300075E0CE0101960E947484BE016F5F7F4F41
:10CF40008FEF90E10E949E82182FCE0101960E94E1
:10CF5000D583112309F42FCF41E050E06FEF70E14A
:10CF6000CE0101960E94AB2DCE0101960E94EEA744
:10CF70004B015C01CE0101960E94D58320E030E098
:10CF8000A901C501B4010E9467B3181634F0812CC1
:10CF9000912C20E8A22E2FE3B22E00916C0210916A
:10CFA0006D020130110509F075C0A501940160E022
:10CFB00070E48CE995E40E9481B560932D02709332
:10CFC0002E0280932F02909330026093C8127093C8
:10CFD000C9128093CA129093CB1260932902709366
:10CFE0002A0280932B0290932C02B801CE014C961A
:10CFF0000E94CC8163E876E0CE0101960E947484A1
:10D00000BE01645E7F4FCE0101960E94EF82BC019B
:10D01000CE0182960E946B84CE0182960E94C83017
:10D02000CE0182960E94D583CE0101960E94D583BF
:10D03000CE014C960E94D58366E27AE0CE0101963D
:10D040000E946284CE0101960E94C830CE010196F2
:10D050000E94D58340912D0250912E0260912F02A3
:10D060007091300225E0CE0101960E94DD83CE0151
:10D0700001960E947A30CE0101960E94D58384EFFA
:10D0800091E090935302809352026AEA71E10E9408
:10D09000BF2891CE0230110509F0A7CFA501940158
:10D0A00060E070E48CE196E40E9481B560932D020B
:10D0B00070932E0280932F02909330026093CC12D3
:10D0C0007093CD128093CE129093CF12609325026D
:10D0D00070932602809327029093280286CF0297AE
:10D0E00011F00C946557C0923302D0923402E09252
:10D0F0003502F09236020C94655761E27AE0CE0177
:10D1000082960E946284BE016E5D7F4FCE018E9634
:10D110000E94BE8211E0811129C06BE17AE0CE014C
:10D120004C960E946284BE01645E7F4FCE018E9653
:10D130000E94BE8211E0811115C065E17AE0CE0146
:10D1400001960E946284BE016F5F7F4FCE018E9672
:10D150000E94BE8211E0811101C010E0CE01019653
:10D160000E94D583CE014C960E94D583CE01829633
:10D170000E94D583112309F429C18AA99BA9059787
:10D1800010F40C94655744E050E0BE01625D7F4F9F
:10D19000CE0101960E94AB2DBE016F5F7F4F8FEFD6
:10D1A00090E10E949C83CE0101960E94D58360E1AC
:10D1B0007AE0CE0101960E946284BE016F5F7F4FCC
:10D1C000CE018E960E94BE82182FCE0101960E943B
:10D1D000D583112309F49BC044E050E0BE01625D99
:10D1E0007F4FCE0101960E94AB2DBE016F5F7F4F36
:10D1F0008FEF90E10E949C83CE0101960E94D5831F
:10D200008FEF90E10E94EEA720E030E0A9010E949C
:10D2100029B6181614F00C9465578FEF90E10E9410
:10D22000EEA760932D0270932E0280932F029093AD
:10D23000300220916C0230916D022130310509F0ED
:10D24000B0C06093C8127093C9128093CA129093B1
:10D25000CB126093290270932A0280932B02909341
:10D260002C02B901CE014C960E94CC8163E876E095
:10D27000CE0101960E947484BE01645E7F4FCE0190
:10D2800001960E94EF82BC01CE0182960E946B84BF
:10D29000CE0182960E94C830CE0182960E94D5832C
:10D2A000CE0101960E94D583CE014C960E94D58373
:10D2B0006EEF79E0CE0101960E946284CE01019664
:10D2C0000E94C830CE0101960E94D58340912D0264
:10D2D00050912E0260912F027091300225E0CE0114
:10D2E00001960E94DD83CE0101960E947A30CE0124
:10D2F00001960E94D58384EF91E09093530280932E
:10D3000052026AEA71E10E94BF280C94655745E019
:10D3100050E0BE01625D7F4FCE0101960E94AB2DB1
:10D32000BE016F5F7F4F8FEF90E10E949C83CE0123
:10D3300001960E94D5836CE974E0CE0101960E94AB
:10D340007484BE016F5F7F4FCE018E960E94BE82B5
:10D35000182FCE0101960E94D583112331F081E070
:10D3600090E090936D0280936C0263ED75E0CE01C6
:10D3700001960E947484BE016F5F7F4FCE018E962E
:10D380000E94BE82182FCE0101960E94D5831123E0
:10D3900009F436CF82E090E090936D0280936C02A6
:10D3A0002FCF2230310509F05CCF6093CC127093FF
:10D3B000CD128093CE129093CF126093250270937A
:10D3C000260280932702909328024BCF6BEF79E0DF
:10D3D000CE014C960E946284BE01645E7F4FCE01F6
:10D3E0008E960E94BE8211E0811115C067EF79E030
:10D3F000CE0101960E946284BE016F5F7F4FCE0115
:10D400008E960E94BE8211E0811101C010E0CE0113
:10D4100001960E94D583CE014C960E94D58311239C
:10D4200009F463C064EF79E0CE0101960E94628442
:10D43000BE016F5F7F4FCE018E960E94BE82182F75
:10D44000CE0101960E94D583112399F042E050E06D
:10D4500063E271E1CE0101960E94AB2DBE016F5FC8
:10D460007F4F8FEF90E10E949C83CE0101960E9436
:10D47000D58360EF79E0CE0101960E946284BE01FF
:10D480006F5F7F4FCE018E960E94BE82182FCE0115
:10D4900001960E94D583112399F043E050E063E2A6
:10D4A00071E1CE0101960E94AB2DBE016F5F7F4FEF
:10D4B0008FEF90E10E949C83CE0101960E94D5835C
:10D4C0008FEF90E10E942582653B710510F40C946A
:10D4D00065576DED79E0CE0101960E946284CE0120
:10D4E00001960E94C8300C94925D69ED79E0CE01FE
:10D4F00001960E946284BE016F5F7F4FCE018E96BF
:10D500000E94BE82182FCE0101960E94D58311235E
:10D5100009F474C026E030E044E050E063E271E1D9
:10D52000CE0101960E948984BE016F5F7F4F8FEF0D
:10D5300090E10E949C83CE0101960E94D5836DEB01
:10D5400075E0CE0101960E9474844091271150919C
:10D5500028118D819E81481B590BBE016F5F7F4F43
:10D5600083E291E10E94F9A7AC014F5F5F4F63E254
:10D5700071E1CE014C960E94AB2DBE01645E7F4FDF
:10D580008FEF90E10E949C83CE014C960E94D58340
:10D59000CE0101960E94D5838FEF90E10E94EEA705
:10D5A00088E2E2E3FAE0A1E8B2E101900D928A9507
:10D5B000E1F784EF91E090935302809352026AEA7C
:10D5C00071E10E94BF2868EB79E085E091E10E945B
:10D5D000608344E050E063E271E1CE0101960E9475
:10D5E000AB2DBE016F5F7F4F85E091E10E945983B3
:10D5F000CE0101960E94D5830C94455460EB79E0EE
:10D60000CE0101960E946284BE016F5F7F4FCE0102
:10D610008E960E94BE82182FCE0101960E94D5835D
:10D6200011110C94395A69EA79E0CE0101960E94F1
:10D630006284BE016F5F7F4FCE018E960E94BE82D4
:10D64000182FCE0101960E94D583112371F141E07C
:10D6500068E972E0CE0101960E94F689BE016F5F13
:10D660007F4F81E193E10E94872C81E193E10E9449
:10D67000501C811104C065E379E00C94FB5181E1F9
:10D6800093E10E94300B892B51F081E193E10E94DC
:10D69000C517682F87E49FE00E946477F0CF81E18F
:10D6A00093E10E945C1C0C94124960EA79E0CE017F
:10D6B00001960E946284BE016F5F7F4FCE018E96FD
:10D6C0000E94BE82182FCE0101960E94D58311239D
:10D6D000E9F0EDB7FEB7E553F1400FB6F894FEBFA1
:10D6E0000FBEEDBFADB7BEB7119685E391E0EAEA94
:10D6F000F1E101900D920197E1F70E94A7430FB667
:10D70000F894DEBF0FBECDBF0C9412496AE979E0F0
:10D71000CE0101960E946284BE016F5F7F4FCE01F1
:10D720008E960E94BE82182FCE0101960E94D5834C
:10D73000112309F45AC0ADB7BEB7A553B1400FB617
:10D74000F894BEBF0FBEADBF119685E391E0EAEA43
:10D75000F1E101900D920197E1F70E94F63B0FB6BF
:10D76000F894DEBF0FBECDBF69E879E0CE01019627
:10D770000E9462848DB79EB7855391400FB6F8948E
:10D780009EBF0FBE8DBFADB7BEB7119685E391E0CA
:10D79000EAEAF1E101900D920197E1F70E94D4339A
:10D7A000ADB7BEB7AB5CBE4F0FB6F894DEBF0FBED1
:10D7B000CDBFEDB7FEB7E553F1400FB6F894FEBF0D
:10D7C0000FBEEDBFA453B14085E391E0EAEAF1E179
:10D7D00001900D920197E1F70E94A7430FB6F894CC
:10D7E000DEBF0FBECDBF0C94474E65E879E0CE0199
:10D7F00001960E946284BE016F5F7F4FCE018E96BC
:10D800000E94BE82182FCE0101960E94D58311235B
:10D8100001F162E779E0CE0101960E946284BE01C7
:10D820006F5F7F4FCE014C960E946B84CE014C9669
:10D830000E947A30CE014C960E94D583ADB7BEB718
:10D84000A553B1400FB6F894BEBF0FBEADBF119641
:10D85000BBCF6EE679E0CE0101960E946284BE01E4
:10D860006F5F7F4FCE018E960E94BE82182FCE0131
:10D8700001960E94D583112309F4F0C062E479E097
:10D88000CE0182960E946284BE016E5D7F4FCE0102
:10D8900001960E946B84AE014F5F5F4F62E070E0C3
:10D8A00083E892E00E94B83D8C01CE0101960E946F
:10D8B000D5830130110511F1BE016E5D7F4FCE01A0
:10D8C0004C960E946B8467E876E0CE014C960E94ED
:10D8D000D98266E571E10E94EF82BC01CE0101961A
:10D8E0000E946B84CE0101960E947A30CE0101968F
:10D8F0000E94D583CE014C960E94D58368EE73E0DA
:10D9000080E090E00E945E0DBE016E5D7F4FCE0113
:10D9100001960E946B84AE014F5F5F4F63E070E041
:10D9200086E792E00E94B83D8C01CE0101960E94EC
:10D93000D58301301105F1F0BE016E5D7F4FCE0140
:10D940004C960E946B8466E571E1CE014C960E9474
:10D95000EF82BC01CE0101960E946B84CE0101963C
:10D960000E947A30CE0101960E94D583CE014C965A
:10D970000E94D58368EE73E080E090E00E945E0D27
:10D980006AE471E1CE0101960E946B84AE014F5FA3
:10D990005F4F61E070E082EB92E00E94B83D8C0145
:10D9A000CE0101960E94D58301301105E9F06AE4A9
:10D9B00071E1CE014C960E946B8466E571E1CE0167
:10D9C0004C960E94EF82BC01CE0101960E946B84AE
:10D9D000CE0101960E947A30CE0101960E94D58335
:10D9E000CE014C960E94D58368EE73E080E090E013
:10D9F0000E945E0D8091450C882311F40C945456BE
:10DA000043E162EB72E0CE0101960E94F689BE010D
:10DA10006F5F7F4F87E493E10E94872C87E493E157
:10DA20000E94501C882311F40C9454566AE471E14E
:10DA300087E493E10E94978566E970E080E090E0DA
:10DA40000E945E0D87E493E10E945C1C62E370E03B
:10DA500080E090E00E945E0D0C9454566AE679E0F6
:10DA6000CE0101960E946284BE016F5F7F4FCE019E
:10DA70008E960E94BE82182FCE0101960E94D583F9
:10DA80001123C1F00BE41CE091E5E92E9CE0F92E96
:10DA9000D8018C910E5F1F4F60E00E94D4866CE22B
:10DAA00071E080E090E00E945E0DE016F10681F7E3
:10DAB0000C94124965E679E0CE0101960E946284D9
:10DAC000BE016F5F7F4FCE018E960E94BE82182FDF
:10DAD000CE0101960E94D5831123C1F00BE41CE016
:10DAE00081E5E82E8CE0F82EF80180810E5F1F4F53
:10DAF00061E00E94D4866CE271E080E090E00E94D8
:10DB00005E0DE016F10681F70C9412496EE579E09E
:10DB1000CE0101960E946284BE016F5F7F4FCE01ED
:10DB20008E960E94BE82182FCE0101960E94D58348
:10DB3000112311F40C94124927E030E046E050E044
:10DB400063E271E1CE0101960E948984BE016F5F9C
:10DB50007F4F8FEF90E10E949C83CE0101960E943F
:10DB6000D5838FEF90E10E942582672B71F410928C
:10DB7000CD0B63E271E1CE0101960E946B84CE0170
:10DB800001960E94E12E0C94DE5881E08093CD0B2B
:10DB9000F0CF2F923F924F925F926F927F928F922F
:10DBA0009F92AF92BF92CF92DF92EF92FF920F932C
:10DBB0001F93CF93DF9300D000D01F921F92CDB759
:10DBC000DEB760917402709175028091720290913B
:10DBD00073020E948E2984E1482E512C612C712CF5
:10DBE000312C212C8FEF281A380AC301B2010E9470
:10DBF0005E0D609174027091750280917202909135
:10DC000073020E948E298C0183E02816310434F0BF
:10DC10008EE12816310444F4012B51F084E1480EC2
:10DC2000511C611C711CDECF0115110509F0A6C045
:10DC300080917202909173028B30910509F086C039
:10DC40008090E3129090E412A090E512B090E6125A
:10DC5000C090DF12D090E012E090E112F090E2125A
:10DC600064E670E080E090E00E945E0D6FE676E092
:10DC7000CE0101960E946284CE0101960E944A372D
:10DC8000CE0101960E94D58361E082E00E94847BF0
:10DC900021E0B501A401CE0101960E94DD83BE0101
:10DCA0006F5F7F4F83E693E10E948985CE010196E5
:10DCB0000E94D5836FED83E693E10E94390E6AE6F8
:10DCC00076E083E693E10E94A98520E0B701A601F2
:10DCD000CE0101960E94DD83BE016F5F7F4F83E618
:10DCE00093E10E948985CE0101960E94D58367E960
:10DCF00076E083E693E10E94818589829A82AB82F5
:10DD0000BC82CD82DE82EF82F88629813A814B8106
:10DD10005C816D817E818F81988528960FB6F894FD
:10DD2000DEBF0FBECDBFDF91CF911F910F91FF904E
:10DD3000EF90DF90CF90BF90AF909F908F907F90AB
:10DD40006F905F904F903F902F900895863191058E
:10DD500009F476CF0C9709F083CF80905809909002
:10DD60005909A0905A09B0905B09C0905409D0900D
:10DD70005509E0905609F090570972CF0F3F8FEF89
:10DD80001807CCF06CE576E0CE0101960E94628423
:10DD90004AE050E070E060E0CE0101960E947536E6
:10DDA000CE0101960E94D58369E376E085E091E19A
:10DDB0000E94608332C00E3F8FEF1807B9F16BE20B
:10DDC00076E0CE0101960E9462844AE050E070E065
:10DDD00060E0CE0101960E947536CE0101960E9448
:10DDE000D5836CE176E085E091E10E946083B80123
:10DDF000CE0101960E94CC81BE016F5F7F4F85E00E
:10DE000091E10E945983CE0101960E94D58366E07C
:10DE100076E085E091E10E94028319821A821B82DA
:10DE20001C821D821E821F8218866FCF6BEF75E0E9
:10DE3000CE0101960E9462844AE050E070E060E00A
:10DE4000CE0101960E947536CE0101960E94D583BF
:10DE50006BED75E0ABCF2F923F924F925F926F9236
:10DE60007F928F929F92AF92BF92CF92DF92EF926A
:10DE7000FF920F931F93CF93DF93CDB7DEB7AC978D
:10DE80000FB6F894DEBF0FBECDBF8C017B01809131
:10DE9000D00B9091D10B01969093D10B8093D00B26
:10DEA0002091EC0B222341F06AE070E00E9433B62F
:10DEB000181619060CF4C0C281E08093EC0B109286
:10DEC000D10B1092D00B50E040E069E374E0C80140
:10DED0000E94662D82E0E816F10409F4C6C26DE5E1
:10DEE00074E084E491E10E94C281609174027091B7
:10DEF000750280917202909173020E948E291C011A
:10DF00006AEB7DE0C8010E944D2D69E976E0C80109
:10DF10000E9481856DEE72E1CE0101960E946B84B4
:10DF2000BE016F5F7F4FC8010E948985CE010196B7
:10DF30000E94D58362EA76E0C8010E9481856FE580
:10DF400077E0C8010E94A98563EF72E1CE010196D6
:10DF50000E946B84BE016F5F7F4FC8010E9489855C
:10DF600065E577E0C8010E94A98562E072E1CE0113
:10DF700009960E947484BE01675F7F4FC8010E94AA
:10DF8000898568E477E0C8010E94A9856AE672E1A4
:10DF9000CE010F960E947484BE01615F7F4FC8015D
:10DFA0000E94898561E477E0C8010E94A985CE01BD
:10DFB0000F960E94D583CE0109960E94D583CE018B
:10DFC00001960E94D5830E94910D28EE33E040E037
:10DFD00050E00E94B1B429013A0167E377E0C8013B
:10DFE0000E94A985CE0101960E948E2FBE016F5F0F
:10DFF0007F4FC8010E948985CE0101960E94D5837A
:10E00000C301B20120E13EE040E050E00E94D3B401
:10E010004B015C01B901CE0187960E94B72D4CE3FC
:10E02000C42ED12CE12CF12CC501B401A70196011D
:10E030000E94D3B4B901CE0101960E94B72D6FE4BE
:10E0400076E0CE0109960E947484BE016F5F7F4F17
:10E05000CE0109960E94EF82BC01CE0187960E94F4
:10E060005983CE0109960E94D583CE0101960E9464
:10E07000D583C301B201A70196010E94D3B4CE019A
:10E0800001960E94B72D6FE476E0CE0109960E94BA
:10E090007484BE016F5F7F4FCE0109960E94EF82AC
:10E0A000BC01CE0187960E945983CE0109960E9439
:10E0B000D583CE0101960E94D58368EA76E0CE0131
:10E0C00009960E947484BE01695D7F4FCE01099656
:10E0D0000E94EF826BEA76E00E94D982BC01CE01F9
:10E0E00001960E946B84BE016F5F7F4FC8010E9442
:10E0F0008985CE0101960E94D583CE0109960E94A2
:10E10000D58369EB76E0C8010E948185CE01019636
:10E110000E94A328B801CE0101960E94218564EBDC
:10E1200076E0C8010E946F850E94C96D29833A83F9
:10E130004B835C836D837E838F83988749815A816B
:10E140006B817C8121E0CE010F960E94DD83BE01B0
:10E15000615F7F4FCE0109960E946B8461EC76E08F
:10E16000CE0109960E94D982BC0184E491E10E940B
:10E170008583CE0109960E94D583CE010F960E9419
:10E18000D58368EC76E0CE010F960E94748464E437
:10E1900071E1CE010F960E94EF82BC01CE0109967B
:10E1A0000E946B84BE01675F7F4FC8010E94898512
:10E1B000CE0109960E94D583CE010F960E94D58389
:10E1C0004D815E816F81788521E0CE0109960E94A4
:10E1D000DD83BE01675F7F4F84E491E10E949C83F1
:10E1E000CE0109960E94D5836AED76E0CE010F96A6
:10E1F0000E94748464E471E1CE010F960E94EF8264
:10E200006BEE76E00E94D982BC01CE0109960E9495
:10E210006B84BE01675F7F4FC8010E948985CE0174
:10E2200009960E94D583CE010F960E94D583409116
:10E23000D60B5091D70B6091D80B7091D90B22E07F
:10E24000CE010F960E94DD8362EF76E0CE01459607
:10E250000E947484BE01615F7F4FCE0145960E948B
:10E26000EF8264E077E00E94D982BC01CE0109967A
:10E270000E946B84BE01675F7F4FC8010E94898541
:10E28000CE0109960E94D583CE0145960E94D58382
:10E29000CE010F960E94D5834091D20B5091D30BA3
:10E2A0006091D40B7091D50B22E0CE010F960E94A5
:10E2B000DD836DE077E0CE0145960E947484BE0157
:10E2C000615F7F4FCE0145960E94EF8264E077E068
:10E2D0000E94D982BC01CE0109960E946B84BE01C6
:10E2E000675F7F4FC8010E948985CE0109960E9411
:10E2F000D583CE0145960E94D583CE010F960E940C
:10E30000D583E6EF2E16EFEF3E062CF465EB7EE0AC
:10E31000C8010E944D2D62E97DE0C8010E944D2D8B
:10E320009AEAE92E91E1F92E27EDA22E22E0B22EF3
:10E33000CC24C394D12C4701F8E08F0E911C82E0CD
:10E34000A80EB11C8091AA119091AB118C159D055E
:10E350000CF464C0B601CE010F960E94CC8165E832
:10E3600076E0CE0145960E947484BE01615F7F4FC6
:10E37000CE0145960E94EF826AEB75E00E94D98239
:10E38000BC01CE0109960E946B84BE01675F7F4F7E
:10E39000C8010E948985B701645E7F4FCE014B960C
:10E3A0000E947484BE01655E7F4FC8010E9489850A
:10E3B0006BE177E0C8010E948185F5016081718180
:10E3C000660F771F660F771F6A547E4ECE018196C7
:10E3D0000E947484BE016F5D7F4FC8010E948985D1
:10E3E00060E277E0C8010E948185CE0181960E949B
:10E3F000D583CE014B960E94D583CE0109960E940B
:10E40000D583CE0145960E94D583CE010F960E94FA
:10E41000D583FFEFCF1ADF0A74018DCFCE01879627
:10E420000E94D58381E08093480C63E77EE0C801B9
:10E430000E944D2D1092EC0BAC960FB6F894DEBFF7
:10E440000FBECDBFDF91CF911F910F91FF90EF9045
:10E45000DF90CF90BF90AF909F908F907F906F9004
:10E460005F904F903F902F90089565EB7EE0C8013C
:10E470000E944D2DDACF8F929F92AF92BF92CF9292
:10E48000DF92EF92FF920F931F93CF93DF93CDB75D
:10E49000DEB7A0970FB6F894DEBF0FBECDBF6DE517
:10E4A00074E08EE691E10E94C2816DE574E082E63F
:10E4B00091E10E94C28140E6842E42E0942E5AEA05
:10E4C000C52E51E1D52E61EDA62E62E0B62E77ED78
:10E4D000E72E72E0F72E01E010E0F40181919191B6
:10E4E000A191B1914F01892B8A2B8B2B89F5F701D3
:10E4F00082819381F501208131818217930741F157
:10E500000130110559F42091DD123091DE1237FFF0
:10E5100005C0823091050CF409C30197880F991F3B
:10E52000FC01EF5AF34FD801AA0FBB1FA75BB34FF3
:10E5300060818C910E94D486F70182819381F501DC
:10E540009183808364E670E080E090E00E945E0D3D
:10E55000F501619171915F018091AA119091AB11C8
:10E56000801791070CF4E7C2CE0145960E94CC813A
:10E57000B801CE010F960E94CC81B601645E7F4F38
:10E58000CE0109960E9474846AEB75E0CE01019673
:10E590000E947484BE01675F7F4FCE0101960E9486
:10E5A000EF8266E277E00E94D982BE01615F7F4F11
:10E5B0000E94EF826DEB75E00E94D982BE016B5E16
:10E5C0007F4F0E94EF82BC018EE691E10E94598349
:10E5D000CE0101960E94D583CE0109960E94D58373
:10E5E000CE010F960E94D583CE0145960E94D58319
:10E5F0000F5F1F4FF8E0CF0ED11C22E0E20EF11C9E
:10E600000430110509F069CFE091C412F091C512F0
:10E61000EE0FFF1FE153FD4F60817181CE01019626
:10E620000E94CC8146E050E0BE016F5F7F4FCE017B
:10E6300009960E943330BE01675F7F4F82E691E109
:10E640000E945983CE0109960E94D583CE0101967E
:10E650000E94D583E091C612F091C712EE0FFF1F02
:10E66000E153FD4F60817181CE0101960E94CC8102
:10E6700046E050E0BE016F5F7F4FCE0109960E94D9
:10E680003330BE01675F7F4F82E691E10E9459837C
:10E69000CE0109960E94D583CE0101960E94D583B2
:10E6A0006AEB75E0CE0145960E9474840E94910D3C
:10E6B00028EE33E040E050E00E94B1B469017A01F5
:10E6C0006DE574E0CE014B960E9474846DE574E0B4
:10E6D00084E791E10E94C281CE0101960E948E2FB3
:10E6E00044E150E0BE016F5F7F4FCE0109960E946A
:10E6F0003330BE01675F7F4F84E791E10E949C83C6
:10E70000CE0109960E94D583CE0101960E94D58341
:10E710002AE0B701A601CE0109960E94138448E0C1
:10E7200050E0BE01675F7F4FCE010F960E943330ED
:10E7300064E771E1CE0101960E946B84BE01615FC6
:10E740007F4FCE0101960E94EF82BC0188E691E1E5
:10E750000E948583CE0101960E94D583CE010F963B
:10E760000E94D583CE0109960E94D5832AE0B70185
:10E77000A601CE0109960E94138469E277E0CE01DA
:10E7800001960E947484BE01675F7F4FCE0101969F
:10E790000E94EF82BE016B5E7F4F0E94EF82BC0140
:10E7A00084E791E10E945983CE0101960E94D583AE
:10E7B000CE0109960E94D5834091D60B5091D70B7C
:10E7C0006091D80B7091D90B21E0CE0101960E9487
:10E7D000DD83BE016F5F7F4FCE014B960E949C830D
:10E7E000CE0101960E94D58360E377E0CE010196C9
:10E7F0000E947484BE01655E7F4FCE0101960E9427
:10E80000EF82BE016B5E7F4F0E94EF82BC0184E706
:10E8100091E10E945983CE0101960E94D583BE01E9
:10E82000655E7F4FCE0101960E946B8446E050E00A
:10E83000BE016F5F7F4FCE0109960E943330BE014B
:10E84000675F7F4F88E691E10E945983CE01099668
:10E850000E94D583CE0101960E94D5834091D20BB0
:10E860005091D30B6091D40B7091D50B21E0CE0168
:10E8700001960E94DD83BE016F5F7F4FCE014B96F4
:10E880000E949C83CE0101960E94D5836EE377E0BF
:10E89000CE0101960E947484BE01655E7F4FCE0159
:10E8A00001960E94EF82BE016B5E7F4F0E94EF8255
:10E8B000BC0184E791E10E945983CE0101960E9438
:10E8C000D583BE01655E7F4FCE0101960E946B84A9
:10E8D00046E050E0BE016F5F7F4FCE0109960E9477
:10E8E0003330BE01675F7F4F88E691E10E94598314
:10E8F000CE0109960E94D583CE0101960E94D58350
:10E90000609174027091750280917202909173020D
:10E910000E948E299093E30B8093E20B892B71F078
:10E9200060917402709175028091720290917302ED
:10E930000E948E299093E30B8093E20B8091E20B6F
:10E940009091E30B8C3F9F4F0CF415C10E94C96D51
:10E9500029833A834B835C836D837E838F8398877F
:10E9600049815A816B817C8121E0CE0109960E9408
:10E97000DD83BE01675F7F4FCE014B960E949C8373
:10E98000CE0109960E94D58368E477E0CE0109960E
:10E990000E947484BE01655E7F4FCE0109960E947D
:10E9A000EF82BE016B5E7F4F0E94EF82BC0184E765
:10E9B00091E10E945983CE0109960E94D583BE0140
:10E9C000655E7F4FCE0109960E946B8446E050E061
:10E9D000BE01675F7F4FCE010F960E943330BE01AC
:10E9E000615F7F4F88E691E10E945983CE010F96C7
:10E9F0000E94D583CE0109960E94D5834D815E8108
:10EA00006F81788521E0CE0109960E94DD83BE01E9
:10EA1000675F7F4FCE014B960E949C83CE01099683
:10EA20000E94D58363E577E0CE0109960E94748445
:10EA3000BE01655E7F4FCE0109960E94EF82BE0146
:10EA40006B5E7F4F0E94EF82BC0184E791E10E94E0
:10EA50005983CE0109960E94D583BE01655E7F4F22
:10EA6000CE0109960E946B8446E050E0BE01675FCC
:10EA70007F4FCE010F960E943330BE01615F7F4F02
:10EA800088E691E10E945983CE010F960E94D583BA
:10EA9000CE0109960E94D5836EE671E184E791E18B
:10EAA0000E9459836AEB75E0CE0101960E9474843E
:10EAB00062E671E1CE0101960E94EF82BC0188E618
:10EAC00091E10E945983CE0101960E94D58368E6A8
:10EAD00071E1CE0101960E946B84CE0101960E94E5
:10EAE0007A30CE0101960E94D5836AE070E080E022
:10EAF00090E00E945E0DCE014B960E94D583CE0120
:10EB000045960E94D583A0960FB6F894DEBF0FBE3F
:10EB1000CDBFDF91CF911F910F91FF90EF90DF90CC
:10EB2000CF90BF90AF909F908F9008959801281B31
:10EB3000390BC901F3CCCE0145960E94CC81B801B6
:10EB4000CE010F960E94CC81B6016C5E7F4FCE0144
:10EB500009960E9474846AEB75E0CE0101960E94CA
:10EB60007484BE01675F7F4FCE0101960E94EF82E1
:10EB700065E277E018CD69E577E084E791E10E94EE
:10EB80004F8368E677E088E691E10E944F836FE665
:10EB900077E084E791E10E944F8368E677E088E6BA
:10EBA00091E10E944F8378CFBF92CF92DF92EF9294
:10EBB000FF920F931F93CF93DF93CDB7DEB7C4556A
:10EBC000D1090FB6F894DEBF0FBECDBF6C018B012B
:10EBD00065965FAF4EAF65978091D00B9091D10B4A
:10EBE00001969093D10B8093D00B8091EC0B811107
:10EBF0003CC0BB24B394B092EC0B1092D10B10929A
:10EC0000D00B6DE574E0CE01895B9F4F0E94748448
:10EC10006DE574E0CE01835B9F4F0E94748450E0E9
:10EC200040E069E374E0C6010E94662D01301105E1
:10EC300009F0A6C06DE574E084E791E10E94C2810D
:10EC40006596EEADFFAD65978081811124C00E946D
:10EC50003B72B092480CCE01835B9F4F0E94D583DC
:10EC6000CE01895B9F4F0E94D5830FB6F894DEBF1B
:10EC70000FBECDBFCC5ADF4F0FB6F894DEBF0FBE2C
:10EC8000CDBFDF91CF911F910F91FF90EF90DF905B
:10EC9000CF90BF9008956596EEADFFAD65978081EA
:10ECA000882309F467C000E210E09E012F5F3F4F08
:10ECB00040E250E0BE016F5D7F4FCE018D5A9F4F05
:10ECC0000E94F57B049739F3BE016F5D7F4FCE0143
:10ECD0008F5B9F4F0E947484BE016F5B7F4FCE019C
:10ECE000895B9F4F0E949C83CE018F5B9F4F0E9448
:10ECF000D583BE016F5F7F4FCE018F5B9F4F0E9418
:10ED00007484BE016F5B7F4FCE01835B9F4F0E9477
:10ED10009C83CE018F5B9F4F0E94D583BE01695BB0
:10ED20007F4F84E791E10E94598363968EAD9FAD3A
:10ED30006397892B09F4AFCF6DEB75E0CE018F5B44
:10ED40009F4F0E947484BE01635B7F4FCE018F5B37
:10ED50009F4F0E94EF826AEB75E00E94D982BC014E
:10ED600084E791E10E945983CE018F5B9F4F0E94FF
:10ED7000D58391CF64E771E180E591E10E948583BD
:10ED80001092EC0B68CF0895AF92BF92CF92DF92B2
:10ED9000EF92FF920F931F93CF93DF936C017B0150
:10EDA0008B01040F151FEB015E01AE18BF08C017E1
:10EDB000D10759F06991D601ED91FC910190F08154
:10EDC000E02DC6011995892B79F7C501DF91CF9107
:10EDD0001F910F91FF90EF90DF90CF90BF90AF9079
:10EDE0000895FC01538D448D252F30E0842F90E051
:10EDF000821B930B541710F0CF9608950197089536
:10EE0000FC01918D828D981761F0A28DAE0FBF2FFE
:10EE1000B11D5D968C91928D9F5F9F73928F90E054
:10EE200008958FEF9FEF0895FC01918D828D9817C3
:10EE300031F0828DE80FF11D858D90E008958FEF00
:10EE40009FEF0895FC01918D228D892F90E0805CC9
:10EE50009F4F821B91098F73992708958AEA9EE03C
:10EE60000E94227721E0892B09F420E0822F089567
:10EE700087E49FE00E94227721E0892B09F420E0BB
:10EE8000822F0895FC01A48DA80FB92FB11DA35A9C
:10EE9000BF4F2C91848D90E001968F739927848FBA
:10EEA000A689B7892C93A089B1898C9183708064DD
:10EEB0008C93938D848D981306C00288F389E02D7E
:10EEC00080818F7D80830895EF92FF920F931F932F
:10EED000CF93DF93EC0181E0888F9B8D8C8D98130D
:10EEE0001AC0E889F989808185FF15C09FB7F89419
:10EEF000EE89FF896083E889F98980818370806465
:10EF000080839FBF81E090E0DF91CF911F910F91AF
:10EF1000FF90EF900895F62E0B8D10E00F5F1F4FBE
:10EF20000F731127E02E8C8D8E110CC00FB607FCCD
:10EF3000FACFE889F989808185FFF5CFCE010E945B
:10EF40004277F1CFEB8DEC0FFD2FF11DE35AFF4F10
:10EF5000F0829FB7F8940B8FEA89FB8980818062E9
:10EF6000CFCFCF93DF93EC01888D8823B9F0AA89A6
:10EF7000BB89E889F9898C9185FD03C0808186FD74
:10EF80000DC00FB607FCF7CF8C9185FFF2CF8081C3
:10EF900085FFEDCFCE010E944277E9CFDF91CF917F
:10EFA000089580E090E0892B29F00E943877811144
:10EFB0000E94000080E090E0892B49F080E090E022
:10EFC000892B29F00E94000081110E94000080E03E
:10EFD00090E0892B49F080E090E0892B29F00E9495
:10EFE000000081110E94000080E090E0892B29F050
:10EFF0000E942E7781110C9400000895CF92DF9229
:10F00000EF92FF92CF93DF9380915510883050F0AC
:10F01000CFEFDFEFCE01DF91CF91FF90EF90DF9048
:10F02000CF900895E0917A10E11142C00E94910DB5
:10F030006B017C0128EEC20E23E0D21EE11CF11C04
:10F0400089E490E10E942024882311F38091B0107C
:10F05000882331F080917B1090917C10892BC1F234
:10F0600089E490E10E948322EC01CF3FDC0771F03C
:10F070008091B010882371F280917B1090917C1068
:10F08000019790937C1080937B10C4CF0E94910DC8
:10F09000C616D706E806F90698F610927A1089E4A3
:10F0A00090E10E947B2489E490E10E944224B2CF47
:10F0B000E150E0937A10F0E0E15CFF4EC38DD0E0C8
:10F0C000A9CF0F931F93CF93DF93EC018C01F8012D
:10F0D00081918F018823A1F10E94FE77F80122918E
:10F0E000022E000C330B8217930789F38F3F98078A
:10F0F00081F0A0917A1091E09A0F90937A10B0E08D
:10F10000A15CBF4E5B968C93903219F48FE1809393
:10F110007A102FE1EC17FD07C9F092919F3FD1F3D0
:10F12000A0917A1081E08A0F80937A10B0E0A15C00
:10F13000BF4E5B969C93803269F720937A10EACF9A
:10F1400081E0DF91CF911F910F91089580E0F9CF79
:10F150008F929F92AF92BF92CF92DF92EF92FF92E7
:10F16000CF9320EF3FE030933C0C20933B0C88235F
:10F1700009F46DC040E060E070E0CB010E94D6125F
:10F1800081110BC080E0CF91FF90EF90DF90CF9086
:10F19000BF90AF909F908F9008958091130E8F77BE
:10F1A00089F780911F0E9091200EA091210EB091B1
:10F1B000220E84369105A105B10520F3C0901B0EE7
:10F1C000D0901C0EE0901D0EF0901E0EC114D104C4
:10F1D000E104F104B9F240E0C701B6010E94D61281
:10F1E000882381F28091600C9091610C811592408E
:10F1F00049F6A091650CAA2329F26091630C7091E5
:10F20000640C6115710509F4BDCF2091620C2223B5
:10F2100009F4B8CFA0930E102093001090E080E086
:10F2200030E0E1E0F0E0C82FAF01082E02C0440F4B
:10F23000551F0A94E2F72417350769F041E0480F9B
:10F2400001968930910579F7409309109BCFC12C25
:10F25000D12C7601C0CF8093091020916B0C309196
:10F260006C0C50E040E02115310541F42091790CFF
:10F2700030917A0C40917B0C50917C0C20930110C2
:10F28000309302104093031050930410460157012D
:10F29000860E971EA11CB11C80920F109092101028
:10F2A000A0921110B0921210E091660CF091670CD0
:10F2B000F0931510E0931410B0E00E94F2B4DC015A
:10F2C000CB01880D991DAA1DBB1D8093161090932C
:10F2D0001710A0931810B093191025E0EE0FFF1F20
:10F2E0002A95E1F7E150FE4FEF2FFF27E6958E0FAD
:10F2F0009F1FA11DB11D80930A1090930B10A09326
:10F300000C10B0930D108090680C9090690CB12C8B
:10F31000A12C8114910441F48090750C9090760C8E
:10F32000A090770CB090780CC81AD90AEA0AFB0AA8
:10F33000C80CD91CEA1CFB1C04C0F694E794D794B3
:10F34000C794CA95D2F7C0920510D0920610E092E9
:10F350000710F092081085EFC8168FE0D806E10478
:10F36000F10428F48CE08093131081E00CCF80E14D
:10F3700025EFC2162FEFD206E104F104A0F380912D
:10F38000810C9091820CA091830CB091840C80939D
:10F39000161090931710A0931810B093191080E2D4
:10F3A000E2CF10923A0C1092390C1092860E109205
:10F3B000A80E0E946C0F88EA9AE09093380C809314
:10F3C000370C89EA9AE09093360C8093350C0895B7
:10F3D000FB0101900020E9F73197AF01461B570B65
:10F3E000DC01ED91FC910280F381E02D19940E94E3
:10F3F00070B80F931F93CF93DF93EC0188819981AD
:10F40000009759F02A813B812617370730F081E0B9
:10F41000DF91CF911F910F9108958B016F5F7F4F07
:10F420000E948FB7009759F0998388831B830A83C2
:10F430002C813D81232B59F7FC011082E8CF80E01D
:10F44000E7CFEF92FF920F931F93CF93DF93611556
:10F45000710541F480E0DF91CF911F910F91FF90F2
:10F46000EF90089541155105B1F07B01EC010C813D
:10F470001D81040F151FB8010E94F979882351F3EB
:10F48000288139818C819D81B701820F931F0E9451
:10F49000C0B81D830C8381E0DECFCF93DF93EC01F6
:10F4A00088819981009711F00E9406B7198218820D
:10F4B0001D821C821B821A82DF91CF910895EF92E8
:10F4C000FF920F931F93CF93DF93EC017B018A018F
:10F4D000BA010E94F97981110BC0CE010E944D7AC8
:10F4E000CE01DF91CF911F910F91FF90EF90089582
:10F4F0001D830C83B701888199810E94C0B8F0CF29
:10F500008CBD9DBD08958F929F92AF92BF92CF9276
:10F51000DF92EF92FF920F931F93CF93DF93D091DF
:10F52000A80ED13208F0D7C0182FC091A70E0E94A4
:10F53000390D6B017C0180917F0E81116BC082E0DF
:10F5400080937F0E10937E0E8FEF80937D0E10922E
:10F550007C0ED0937B0EA7E8BEE0EBE5FEE080E0FA
:10F56000D81391C010925A0E80915A0ECC0FC82B0E
:10F57000C0935A0E8091590E813009F088C01092C4
:10F58000590E0E94390D6B017C0180915A0E8093B7
:10F59000BB008091810E9091820EA091830EB0915C
:10F5A000840E892B8A2B8B2BA1F00E94390D0091A0
:10F5B000810E1091820E2091830E3091840E6C1971
:10F5C0007D098E099F09061717072807390708F4D0
:10F5D00042C08091BC0083FDD8CF85EC8093BC00F5
:10F5E0000E94390D6B017C0180917F0E823009F4FD
:10F5F00050C080917D0E8F3F09F46FC080917D0EC9
:10F60000803209F46CC080917D0E803309F469C0AA
:10F6100084E026C08091810E9091820EA091830E8D
:10F62000B091840E892B8A2B8B2B09F484CF0E94F6
:10F63000390D8090810E9090820EA090830EB09034
:10F64000840E6C197D098E099F0986169706A806F7
:10F65000B90608F070CF8091800E0E948A0F85E075
:10F660001092860E1092A80E1092850EDF91CF9107
:10F670001F910F91FF90EF90DF90CF90BF90AF90D0
:10F680009F908F9008959D9191938F5F69CF85EEA4
:10F69000A5CF8091810E9091820EA091830EB091A2
:10F6A000840E892B8A2B8B2B09F49ECF0E94390D57
:10F6B0000091810E1091820E2091830E3091840E64
:10F6C0006C197D098E099F09061717072807390746
:10F6D00008F08ACFC0CF81E0C3CF80E0C1CF82E005
:10F6E000BFCF83E0BDCFCF93C82F682F607F83E665
:10F6F00093E10E94200E80E1C89FB001112483E6AF
:10F7000093E1CF910C94200ECF93DF9300D000D0E3
:10F710001F921F92CDB7DEB798E0E1E3F3E0DE0180
:10F72000119601900D929A95E1F790916C139617AE
:10F7300008F46FEF70E0660F771F21E030E02C0FC8
:10F740003D1F620F731FFB019081890F806828960F
:10F750000FB6F894DEBF0FBECDBFDF91CF910C94F2
:10F76000737BCF93DF93EC019A01AB01E889F989B0
:10F7700082E08083211581EE38074105510581F132
:10F7800060E079E08DE390E00E94B1B4215031094E
:10F79000410951095695479537952795EC85FD8583
:10F7A0001082EE85FF852083188EEC89FD8986E026
:10F7B0008083EA89FB89808180618083EA89FB8973
:10F7C000808188608083EA89FB898081806880836A
:10F7D000EA89FB8980818F7D8083DF91CF910895B5
:10F7E000E889F989108220E1D9CF2F923F924F9278
:10F7F0005F926F927F928F929F92AF92BF92CF92C1
:10F80000DF92EF92FF920F931F93CF93DF9300D07D
:10F81000CDB7DEB71C013B014A0129015801FC01AB
:10F82000C080D18070E060E0C3010E94A5B8A8014B
:10F8300070E060E0C2010E94A5B8F601808110E08E
:10F8400000E0811162C004E010E004C07601F10123
:10F85000F182E082C8010F900F900F90DF91CF915D
:10F860001F910F91FF90EF90DF90CF90BF90AF90DE
:10F870009F908F907F906F905F904F903F902F90D0
:10F8800008956B3209F482C06D3309F04EC0818156
:10F890008823E9F2F7018FEFE81AF80A60816532F0
:10F8A00009F452C00CF048C0662309F456C082E047
:10F8B000A816B1040CF061C0012B09F46BC003E081
:10F8C00010E0E8CF81818983882309F282818A83CD
:10F8D0007601811104C0F2E0EF0EF11CB8CF83E095
:10F8E000E80EF11C1B8240E150E070E060E0CE01C8
:10F8F00001960E942AAB19C0F3016083F1E08F1AD0
:10F900009108C30101963C0167017601FFEFEF1AF0
:10F91000FF0AF6016081663209F499CF0CF0B1CF8D
:10F92000662309F493CF653269F2F2E08F169104F1
:10F930001CF701E010E0E8CF663209F488CF6B32A3
:10F9400009F0B5CF60E2B3CF81818983882301F1CB
:10F9500082818A83811103C032967F0178CF7F0133
:10F9600093E0E90EF11C1B8240E150E070E060E0A2
:10F97000CE0101960E942AAB9ACFF2016083F1E09A
:10F98000AF1AB108C20101962C0184CF60E2CDCF3D
:10F99000F701E3CF02E010E07DCF0F931F93CF93E9
:10F9A000DF93EC010E94910D8B010E9430118F3F7B
:10F9B00069F00E94910D601B710B6C177D07A8F315
:10F9C00080E0DF91CF911F910F91089581E0F9CFF1
:10F9D000CF93DF93EC016E857F858889998941E01B
:10F9E0000E94D612882351F08A8920E2829FC001AA
:10F9F00011248B5A934FDF91CF91089590E080E0CE
:10FA0000FACF8F929F92AF92BF92CF92DF92EF92F6
:10FA1000FF920F931F93CF93DF9300D01F92CDB728
:10FA2000DEB7FC018581813091F080E00F900F906E
:10FA30000F900F90DF91CF911F910F91FF90EF905A
:10FA4000DF90CF90BF90AF909F908F90089584816A
:10FA500081FFEBCF83899489A589B689892B8A2B6D
:10FA60008B2B09F45EC07F0140E050E0BA01CF016A
:10FA70000E9419158823C9F2F701C38CD48C87889A
:10FA8000908CA18CB28C82E090E0A0E0B0E0F60116
:10FA900080839183A283B3839E012F5F3F4FB50183
:10FAA000A401C6010E94C113882309F4BECF00E05F
:10FAB00010E09801B501A401C6010E941F1388231C
:10FAC00009F4B3CF89809A80AB80BC80F601878926
:10FAD000803111F188EF9FEFAFEFBFE088169906F4
:10FAE000AA06BB06C8F2F701178A108E118E128E75
:10FAF000138A148A158A168A848180688483C701D0
:10FB00000E94F317882309F490CF40E050E0BA0137
:10FB1000C7010E9419158ACF88EF9FEFA0E0B0E0DF
:10FB2000DDCF81E083CF4F925F926F927F928F9271
:10FB30009F92AF92BF92CF92DF92EF92FF920F937C
:10FB40001F93CF93DF93CDB7DEB763970FB6F894CB
:10FB5000DEBF0FBECDBF7C016B013A01FB0120E08F
:10FB600090E080E06AE03191332309F461C040ED18
:10FB7000430F4A3008F04DC0689FA001699F500DA7
:10FB80001124CA01C097830F911D37FD9A958F3FAD
:10FB9000910549F340F3F7014281538164817581F6
:10FBA0008091101490911114A0911214B09113141B
:10FBB000481759076A077B0709F40DC28701085FD8
:10FBC0001F4F0E94910D6F7077277C5FC8010E94C4
:10FBD000D325813009F004C280E394E09A838983BD
:10FBE000F70182819381A481B5818B839C83AD834E
:10FBF000BE8345E350E0BE016F5F7F4FC8010E94A6
:10FC00005C26892BA9F5D12CC12CC8010E94FF22AA
:10FC100017C03E3209F0BFCF233009F4BCCFD30167
:10FC2000A20FB11D12968C932F5F90E080E09BCFC6
:10FC3000233009F0B0CFF3018583CC24C394D12CB9
:10FC4000C60163960FB6F894DEBF0FBECDBFDF913D
:10FC5000CF911F910F91FF90EF90DF90CF90BF90C9
:10FC6000AF909F908F907F906F905F904F9008958E
:10FC70000E94910DF7017783668342E050E0B7015F
:10FC80006A5F7F4FC8010E94F12581E090E09A836E
:10FC9000898342E050E0BE016F5F7F4FC8010E9440
:10FCA000F12580E091E09A83898342E050E0BE0133
:10FCB0006F5F7F4FC8010E94F1251A82198242E0CE
:10FCC00050E0BE016F5F7F4FC8010E94F12542E006
:10FCD00050E0BE016F5F7F4FC8010E94F12542E0F6
:10FCE00050E0BE016F5F7F4FC8010E94F1255601B1
:10FCF000F6018081882301F16501F60181912F01D0
:10FD0000882311F08E32B1F446018A189B0818142A
:10FD1000190474F48D8641E050E0BE01635F7F4FAB
:10FD2000C8010E94F125A401B501C8010E94F12576
:10FD30005201DECF6201E1CF1D8641E050E0BE01FD
:10FD4000635F7F4FC8010E94F125C12CDD24D3944D
:10FD5000DA82C98242E050E0BE016F5F7F4FC80186
:10FD60000E94F125DA82C98242E050E0BE016F5F55
:10FD70007F4FC8010E94F125C8010E942B26892BC4
:10FD800009F441CFF3E0AF2EB12C230122E0420E63
:10FD9000511CD4C0F7014281538164817581808DEB
:10FDA000918DA28DB38D481759076A077B0709F01B
:10FDB00008C1848D958DC59709F003C181A192A1D9
:10FDC0005DEFC52EDD24DA940C970CF4ADC04CE049
:10FDD00050E0BE016F5F7F4FC8010E94DE218B8122
:10FDE0009C819827892798279A8B898BF7014681D0
:10FDF000578129813A814217530709F0E7C097FFDD
:10FE0000E5C08F7092703BEFC32EDD24DA94892B0E
:10FE100009F08AC06F8078847624672476242AEFDC
:10FE2000C22EDD24DA946114710409F47DC0D12C52
:10FE3000C12C8D819E81982789279827C816D906BD
:10FE4000F8F441E050E0BE01635F7F4FC8010E94BB
:10FE5000DE214D85442331F050E070E060E0C801C0
:10FE60000E94DE218D858111ECCF44E050E070E0EE
:10FE700060E0C8010E94DE21FFEFCF1ADF0AD9CF70
:10FE8000912C812C41E050E0BE016D5E7F4FC80196
:10FE90000E94DE214B89842F807C09F06CC04423B2
:10FEA00031F050E070E060E0C8010E94DE218B89F3
:10FEB0008111E8CF42E050E0BE01615F7F4FC80191
:10FEC0000E94DE2142E050E0BE01635F7F4FC80127
:10FED0000E94DE2144E050E070E060E0C8010E9432
:10FEE000DE2142E050E0BE016F5E7F4FC8010E94FC
:10FEF000DE218F85988949895A898115914009F0B9
:10FF000043C0CD84DE84DC24CD24DC2481E0C8160B
:10FF1000D104D1F54115544009F04AC044E050E005
:10FF2000B201C8010E94DE2121E0A21AB10809F441
:10FF30006CCEFFEFCF16DF0609F067CE0E94910D61
:10FF40003B014C01C8010E942722181619060CF427
:10FF500021CF0E94910D661977098809990969389E
:10FF600073418105910548F562E370E080E090E01F
:10FF70000E945E0DE7CF41E050E070E060E0C80114
:10FF80000E94DE211B8A93CF54274527542770E017
:10FF900060E0C8010E94DE21FFEF8F1A9F0A6814FB
:10FFA000790409F06FCF96EFC92EDD24DA94BCCF27
:10FFB000E7EFCE2EDD24DA94B7CFCC24CA94DC2C24
:10FFC000B3CF6EEFC62EDD24DA94AECF4CEFC42E45
:10FFD000DD24DA94A9CF8EEFC82EDD24DA9430CE5A
:10FFE000D12CC12C2DCE0F931F93CF93DF934115AE
:10FFF000510541F0FC01048115810115110539F409
:020000021000EC
:10000000FB011082DF91CF911F910F910895415014
:1000100051094017510708F48A01EB01FC01608186
:100020007181A801CE010E94D5B8C00FD11F1882DE
:10003000E9CF20E3FC0120833296862F82958F70D2
:100040006F706A3030F4605D6293682F8111F5CF74
:100050000895695CF9CF5F926F927F928F929F9221
:10006000AF92BF92CF92DF92EF92FF920F931F93C6
:10007000CF93DF93CDB7DEB7C754D1090FB6F8944D
:10008000DEBF0FBECDBF5C013B0119A218A282E901
:1000900093E09F8F8E8F1BA21C821B829A83898381
:1000A0001E8210E000E06E018EE1C80ED11C8AE1D4
:1000B000E82E80E1F82EF501E00FF11F80818F32EC
:1000C00011F40F5F1F4FD501A00FB11FFE01FB966A
:1000D00090E080E04F012D912F3249F0222339F03A
:1000E0000F5F1F4F019621938C309105A1F7880D6A
:1000F000991DFC011082F501E00FF11F80818F3204
:1001000011F40F5F1F4FF501E00FF11F508041E028
:10011000511040E030E020E0B401C701F30119952F
:10012000811121C0FAE1EF16F0E1FF06C1F480E091
:10013000C95BDF4F0FB6F894DEBF0FBECDBFDF91B6
:10014000CF911F910F91FF90EF90DF90CF90BF90D4
:10015000AF909F908F907F906F905F900895C701B0
:100160000E942218E4CF552091F021E0A401B701AC
:10017000C6010E943618982E8AE1E81680E1F8063A
:1001800081F0C7010E942218911010C0D0CF9AE1CF
:10019000E91690E1F90619F0C7010E94221881E0E2
:1001A000C7CF992021F2FE0131967F019E2D8F2D20
:1001B0007601C92ED82E7FCF8F929F92AF92BF9299
:1001C000CF92DF92EF92FF920F931F93CF93DF9323
:1001D000CDB7DEB760970FB6F894DEBF0FBECDBFC8
:1001E0007C019091400C992351F108E0933309F47C
:1001F00004E06B0180E591E00E94807A9E012F5F10
:100200003F4F5901490110E0812F0E943F1EF40128
:1002100081934F018823D9F01F5F0113F5CF00E0D0
:10022000F50181915F018D3161F0883151F08A5182
:10023000823038F00F5F1013F3CF0E94BA1F18E01E
:100240008AC060E170E0802F0E949D1E102FA12EB9
:10025000B12CF501EE0FFF1FEB5DF34F1182108201
:1002600083EE93E00197F1F742E870E060E0812FC0
:100270000E94801E4FEF62E070E0812F0E94801E7E
:10028000B601C114D10491F4809190029091910231
:1002900001968115F0EC9F0708F471C090939102CC
:1002A000809390026091900270919102812F0E9440
:1002B0006A1E86E0E9E3F3E0DE01199601900D92F3
:1002C0008A95E1F7F70183818F778C8784818D8709
:1002D00085818E87A7014E5F5F4F24E030E06CE0A0
:1002E00070E0812F0E94431EB601812F0E94541E90
:1002F00026E030E0AE01475F5F4F66E070E0812F9F
:100300000E94431E61E070E0812F0E949D1E27E045
:100310002A9DC0012B9D900D11249C012351344F27
:100320007901F9011182108222E030E0AE01415FD3
:100330005F4F68E270E0812F0E94AD1E8F85988923
:10034000982789279827F70193838283168215823D
:1003500014820E94BA1F812F60960FB6F894DEBFF8
:100360000FBECDBFDF91CF911F910F91FF90EF9006
:10037000DF90CF90BF90AF909F908F90089580E0D6
:1003800090EC8CCFFB0101900020E9F73197AF0191
:10039000461B570B0C945F7A0F931F93CF93DF93F9
:1003A000CDB7DEB762970FB6F894DEBF0FBECDBFF4
:1003B0008C01CB01F8011182108213821282158206
:1003C00014824AE0BE016F5F7F4F0E9471ACBE0194
:1003D0006F5F7F4FC8010E94C28162960FB6F8948A
:1003E000DEBF0FBECDBFDF91CF911F910F9108955A
:1003F0000F931F93CF93DF93CDB7DEB7A1970FB6BF
:10040000F894DEBF0FBECDBF8C01CB01BA01F8015D
:100410001182108213821282158214822AE0AE01A8
:100420004F5F5F4F0E94ABACBE016F5F7F4FC80153
:100430000E94C281A1960FB6F894DEBF0FBECDBF59
:10044000DF91CF911F910F910895FC0180819181DF
:10045000009711F00C9431AC60E070E0CB0108958E
:10046000AF92BF92CF92DF92EF92FF920F931F93C2
:10047000CF93DF93DC01CD90DC901197C114D104B0
:1004800039F01496CD91DC918C017601209761F4BE
:10049000DF91CF911F910F91FF90EF90DF90CF9060
:1004A000BF90AF90089575015701BFEFAB1ABB0A1B
:1004B000F7018081082E000C990B0E9458AC892B03
:1004C00091F72197CC0DDD1D8881082E000C990B2A
:1004D0000E9458AC892B29F0CE15DF0510F021972A
:1004E000F3CFAE014F5F5F4F4E195F09D8011596EC
:1004F0005C934E931497CE14DF0420F4B701C60129
:100500000E948AB8D801ED91FC91119714968D91B3
:100510009C91E80FF91F1082BBCFFC01248135812B
:100520006217730748F480819181009729F0860F44
:10053000971FFC018081089580E00895FC012481CB
:100540003581FB014481558124173507A0F0FC015A
:1005500080819181009779F0FB0160817181611543
:10056000710549F0241B350B820F931F0E94B7B809
:1005700021E0892B09F020E0822F0895FB014481BE
:100580005581FC01248135812417350778F080815D
:100590009181009759F0FB016081718161157105AE
:1005A00029F00E94C7B821E0892B09F020E0822FB2
:1005B0000895CF93DF93EC01FB0101900020E9F750
:1005C0003197AF01461B570B0E94217A811103C05E
:1005D000CE010E944D7ACE01DF91CF910895CF9345
:1005E000DF93EC01FB0144815581608171810E94A0
:1005F000217A811103C0CE010E944D7ACE01DF9194
:10060000CF910895EF92FF920F931F93CF93DF93B3
:10061000EC017B01CB010E9468AC0097A9F00C8132
:100620001D81080F191FB801CE010E94F979882396
:1006300061F0288139818C819D81B701820F931FE0
:100640000E9461AC1D830C8381E0DF91CF911F91EB
:100650000F91FF90EF900895CF93DF931F921F9219
:10066000CDB7DEB769831A8241E050E0BE016F5F0B
:100670007F4F0E94217A0F900F90DF91CF910895C4
:10068000CF93DF93EC0160E00E942C83811103C0C3
:10069000CE010E944D7ACE01DF91CF910895FB01EA
:1006A00001900020E9F73197AF01461B570B0C94DE
:1006B000217AFB0144815581608171810C94217AFA
:1006C000EF92FF920F931F93CF93DF93EC018B0177
:1006D000CB010E9468AC7C01BC01CE010E94F9797B
:1006E00081110BC0CE010E944D7ACE01DF91CF91D6
:1006F0001F910F91FF90EF900895FD82EC82B80159
:10070000888199810E9461ACF0CFCF93DF93EC0197
:10071000FB018617970749F06081718161157105AA
:1007200041F0448155810E945F7ACE01DF91CF91E3
:1007300008950E944D7AF9CF0F931F93CF93DF93C3
:100740008C01EB01FC01808191810097E1F06881CF
:10075000798161157105A9F0428153812C813D8118
:100760004217530770F00E94C0B88C819D81F80138
:10077000958384831D821C82DF91CF911F910F91FD
:1007800008950E9406B788819981F801918380833A
:100790008A819B81938382838C819D8195838483CD
:1007A000198218821B821A82E5CFFC018081918117
:1007B000009711F00C9406B70895EF92FF920F93F3
:1007C0001F93CF93DF93CDB7DEB7A1970FB6F89401
:1007D000DEBF0FBECDBF7C01CB01BA01F701118294
:1007E0001082138212821582148242E0420F8E011F
:1007F0000F5F1F4F0E9468AA009789F0BC01C701D4
:100800000E94C281A1960FB6F894DEBF0FBECDBF85
:10081000DF91CF911F910F91FF90EF900895C70145
:100820000E944D7AEFCF0F931F93CF93DF93CDB7F5
:10083000DEB7A2970FB6F894DEBF0FBECDBF8C0116
:10084000CB01BA01F8011182108213821282158243
:10085000148230E0AE014F5F5F4F0E947CACBE015E
:100860006F5F7F4FC8010E94C281A2960FB6F894B5
:10087000DEBF0FBECDBFDF91CF911F910F910895C5
:10088000CF93DF931F921F92CDB7DEB7FC01118289
:100890001082138212821582148269831A82BE0129
:1008A0006F5F7F4F0E94C2810F900F90DF91CF91B9
:1008B0000895FC0111821082138212821582148223
:1008C0000C949C83FC011182108213821282158287
:1008D00014820C946083FC011182108213821282B4
:1008E000158214820C948583FC011182108213827C
:1008F0001282158214826115710551F0FB0101907D
:100900000020E9F73197AF01461B570B0C945F7A33
:100910000895AF92BF92CF92DF92EF92FF920F9322
:100920001F93CF93DF936C015B017A018901241738
:10093000350720F48F2D7901042F182F6DE574E011
:10094000C6010E947484D5011496CD91DC91EC16F9
:10095000FD06E0F40C171D0708F4E801D501ED9140
:10096000FC911197EC0FFD1F108110826D917C910D
:100970006E0D7F1DC60161157105A1F00E94C28137
:10098000F50180819181C80FD91F1883C601DF91BD
:10099000CF911F910F91FF90EF90DF90CF90BF907C
:1009A000AF9008950E944D7AEBCF8F929F92AF92B5
:1009B000BF92EF92FF920F931F93CF93DF93CDB728
:1009C000DEB7A1970FB6F894DEBF0FBECDBF7C0196
:1009D000FA01CB0119A2223008F42AE08E010F5D42
:1009E0001F4F822E912CB12CA12CBF01A501940187
:1009F0000E94B1B4F901CA016A300CF5605DD801FA
:100A00006E938D01232B242B252B79F790E080E02A
:100A1000109721F0BD01C7010E94E879A1960FB699
:100A2000F894DEBF0FBECDBFDF91CF911F910F9124
:100A3000FF90EF90BF90AF909F908F900895695C6A
:100A4000DECF8F929F92AF92BF92CF92DF92EF92C2
:100A5000FF920F931F93CF93DF937C01EB016C0107
:100A600082E0C80ED11C4701E5E08E0E911C10E01B
:100A700000E0F60141916F0150E070E060E02AE093
:100A8000CE010E94D5845C01E881F9810190F0815A
:100A9000E02D6EE2CE0119958A0D9B1D080F191FDE
:100AA000C814D90431F7F701458150E070E060E0E7
:100AB0002AE0CE010E94D584800F911FDF91CF9153
:100AC0001F910F91FF90EF90DF90CF90BF90AF906C
:100AD0009F908F9008956DE378E00C94E8790F93E0
:100AE0001F93CF93DF93EC010E94E8798C01CE0134
:100AF0000E946B85800F911FDF91CF911F910F9105
:100B000008956115710511F00C94E87990E080E08A
:100B10000895DB0114964D915C9115976D917C9130
:100B2000DC01ED91FC910280F381E02D19940F938B
:100B30001F93CF93DF93EC010E9489858C01CE0136
:100B40000E946B85800F911FDF91CF911F910F91B4
:100B50000895EF92FF920F931F93CF93DF938C0131
:100B60007B01D0E0C0E0F701EC0FFD1F649166232C
:100B700061F0D801ED91FC910190F081E02DC80168
:100B80001995892B11F02196EECFCE01DF91CF91EF
:100B90001F910F91FF90EF9008950F931F93CF93A4
:100BA000DF93EC010E94A9858C01CE010E946B8528
:100BB000800F911FDF91CF911F910F910895DC015C
:100BC00080E394E08D939D9384E0FB0101900D926E
:100BD0008A95E1F708951F920F920FB60F92112494
:100BE0000BB60F922F933F934F935F936F937F9327
:100BF0008F939F93AF93BF93EF93FF938AEA9EE007
:100C00000E944277FF91EF91BF91AF919F918F9199
:100C10007F916F915F914F913F912F910F900BBEFC
:100C20000F900FBE0F901F9018951F920F920FB646
:100C30000F9211240BB60F922F938F939F93EF93E4
:100C4000FF93E091BA0EF091BB0E8081E091C00E4F
:100C5000F091C10E82FD1DC090818091C30E8F5F07
:100C60008F732091C40E821741F0E091C30EF0E023
:100C7000E655F14F958F8093C30EFF91EF919F91B1
:100C80008F912F910F900BBE0F900FBE0F901F9062
:100C900018958081F2CF1F920F920FB60F921124F8
:100CA0000BB60F922F933F934F935F936F937F9366
:100CB0008F939F93AF93BF93EF93FF9387E49FE04E
:100CC0000E944277FF91EF91BF91AF919F918F91D9
:100CD0007F916F915F914F913F912F910F900BBE3C
:100CE0000F900FBE0F901F9018951F920F920FB686
:100CF0000F9211240BB60F922F938F939F93EF9324
:100D0000FF93E091570FF091580F8081E0915D0FB4
:100D1000F0915E0F82FD1DC090818091600F8F5F0A
:100D20008F732091610F821741F0E091600FF0E026
:100D3000E95BF04F958F8093600FFF91EF919F914A
:100D40008F912F910F900BBE0F900FBE0F901F90A1
:100D500018958081F2CFCF93DF93282F30E0F901EF
:100D6000EC50F14F8491F901E850FF4ED491F90114
:100D7000E25CFE4EC491CC23A1F081110E94A10C33
:100D8000EC2FF0E0EE0FFF1FE652F14FA591B4916A
:100D9000EC91ED2381E090E009F480E0DF91CF91C8
:100DA000089580E090E0FACF1F93CF93DF93282F30
:100DB00030E0F901EC50F14F8491F901E850FF4E19
:100DC000D491F901E25CFE4EC491CC23A9F0162F18
:100DD00081110E94A10CEC2FF0E0EE0FFF1FEC53ED
:100DE000FF4EA591B4918FB7F894EC91111108C002
:100DF000D095DE23DC938FBFDF91CF911F910895B3
:100E0000DE2BF8CFAF92BF92CF92DF92EF92FF929C
:100E10000F931F93CF93DF93C82FD62F1092E71213
:100E20001092E8121092E9121092EA121092EB124C
:100E300061E00E94080D60E08C2F0E94D4866D2F27
:100E400070E090E080E00E945E0D60E08C2F0E94D8
:100E5000080D8BE990E00197F1F700E911E08C2F84
:100E60000E94AB86892B81F401501109C1F78EEFE6
:100E70009FEFDF91CF911F910F91FF90EF90DF9047
:100E8000CF90BF90AF90089500E911E08C2F0E94A1
:100E9000AB86019721F401501109C1F7E8CF18E2A0
:100EA000D0E800E090E9E92EFF24F3948C2F0E9413
:100EB000AB86892B29F481E0E81AF108B9F7D7CF7E
:100EC0000E94390D6B017C0180E9A82EBB24B394EC
:100ED0008C2F0E94AB86019729F481E0A81AB108F3
:100EE000B9F7C5CF0E94390D6C197D098E099F098C
:100EF000693271058105910538F0E02FF0E0E1528B
:100F0000FD4E80858D2B8087D69511F40F5FD0E83C
:100F1000115041F690E080E0ACCFEF92FF920F933A
:100F20001F93CF93DF93EC010E94500E7E01EE0CD5
:100F3000FF1CEE0CFF1CF701E152FD4F6083718333
:100F400082839383CC0FDD1FFE01E952FD4F808128
:100F500091811816190644F4FE01E153FD4F80817A
:100F600091811816190654F1FE01E952FD4F01E076
:100F700010E011830083FE01E75BF34F6091530C97
:100F800080810E94D486C153DD4F19830883F70105
:100F9000E154FD4F88E097E0A0E0B0E080839183CA
:100FA000A283B38364EF71E080E090E0DF91CF91A2
:100FB0001F910F91FF90EF900C945E0DDF91CF91F8
:100FC0001F910F91FF90EF9008950F931F93CF9370
:100FD000DF9300D000D01F921F92CDB7DEB7809173
:100FE000E01381112AC01092C8131092C71388EE23
:100FF00093E0A0E0B0E08093C9139093CA13A0934C
:10100000CB13B093CC138AEB93E09093C6138093E9
:10101000C51380E394E09093D4138093D31310927C
:10102000D5131092D6131092D7131092D81388E0CC
:101030008093DD1381E08093E01382E893E1909345
:10104000430C8093420C8091811381119DC060E319
:1010500072E080E090E00E945E0D1FB7F8948091EE
:101060008013811127C0E3E7F1E18491EDE2F1E122
:101070009491E82FF0E0EE0FFF1FE252FF4EA59192
:10108000B491EC91E92321F461E085E30E94D486D8
:1010900061E085E30E94080D8CB580618CBD8CB544
:1010A00080648CBD61E084E30E94080D61E083E30D
:1010B0000E94080D809180138F5F809380131FBF63
:1010C000E8E4F1E1E491F0E0EE0FFF1FEC53FF4E96
:1010D0008591949190933F0C80933E0CE2E0F1E176
:1010E000E491E0933D0C61E08AE00E94080D0E94CB
:1010F000A31C80E591E00E94807A84E38093400CF9
:1011000080E80E942C1E0E94161E882309F4F5C058
:1011100088E00E942C1E0E94031E883009F0EDC05A
:1011200080E10E942C1E0E94031E803109F0E5C060
:1011300080E00E942C1E0E94031E182F8111DDC02A
:1011400041E050E0BE016F5F7F4F8FE190E00E9471
:10115000AD1C8981833009F0D0C080E48093410CBC
:1011600042E06EE170E0812F0E94801E42E06FE15C
:1011700070E0812F0E94801E1F5F183089F70E9447
:10118000BA1F81E08093811380E591E00E94807A0C
:1011900046E050E062E972E089E090E00E94551D6F
:1011A00080E394E09A8389831B821C821D821E82C5
:1011B000CE0103960E94B31F0E94BA1F8091420C79
:1011C0009091430CDC0192961D921D921D921C92EF
:1011D0009597FC0116A217A210A611A69A961D9229
:1011E0001D921D921C929D9740E65AEE60E070E0C1
:1011F00046AB57AB60AF71AF40EA5FE060E070E0D4
:10120000DA964D935D936D937C93DD973E9624E142
:10121000DF011D922A95E9F726E0E2E9F2E0DC0120
:10122000189601900D922A95E1F7FC01EE5BFF4FB5
:1012300010820E9459398C01019709F0CBC080E5DA
:1012400091E00E94807A6091420C7091430C625F41
:101250007F4FCE0101960E94DF85CE0103960E944A
:10126000B31F6091420C7091430C6A5E7F4FCE01B8
:1012700001960E94DF8544E050E0BE016D5F7F4F24
:1012800081E090E00E94551D6091420C7091430CEA
:101290006E5E7F4FCE0101960E94DF8544E050E0F4
:1012A000BE016D5F7F4F85E090E00E94551D0E945A
:1012B000BA1F6091420C7091430C625E7F4FCE0169
:1012C00001960E94DF858B819C81AD81BE818093D8
:1012D0003B1090933C10A0933D10B0933E100E94A1
:1012E000390D7F7380919002909191026827792740
:1012F00070939102609390026DC087E38093400CDD
:1013000080E80E942C1E0E94161E882329F188E086
:101310000E942C1E0E94031E8830F1F480E10E947E
:101320002C1E0E94031E182F8031B1F480E00E9411
:101330002C1E0E94031E81110FC041E050E0BE012F
:101340006F5F7F4F89E390E00E94AD1C89818430FC
:1013500019F41093410C13CF83E38093400C80E881
:101360000E942C1E0E94161E882371F180E10E94AB
:101370002C1E0E94031E803139F582E10E942C1E32
:101380000E94031E823101F580E00E942C1E0E9403
:10139000031E811119C084E08093410C15E5188764
:1013A00041E050E0BE01685F7F4F8BE190E00E941A
:1013B000551D1F8341E050E0BE01695F7F4F8AE108
:1013C00090E00E94551DDBCE1092400C0E94BA1F87
:1013D00010E000E0C80128960FB6F894DEBF0FBEFB
:1013E000CDBFDF91CF911F910F9108952F923F9222
:1013F0004F925F926F927F928F929F92AF92BF9225
:10140000CF92DF92EF92FF920F931F93CF93DF93D0
:10141000CDB7DEB7C756D1090FB6F894DEBF0FBE01
:10142000CDBF5C013B01A6964FAFA6974E018EE162
:10143000880E911C6AE170E1C4010E94001C1C82AC
:101440001B8282E993E09A8389831E8263018E0165
:101450000F5F1F4F240118016FE270E0C6010E9468
:10146000ACB8009709F459C0F60120812F3271F40D
:10147000FFEFCF1ADF0A902F812F8201492E582EBD
:10148000942D852D2801092F182FE6CF8C198D302A
:1014900008F08CE0E82EF12CA701B601CE01885AA5
:1014A0009F4F0E94D5B8E8E5F0E0EC0FFD1FEE0D70
:1014B000FF1D1082C8010E94221821E0AE01485A87
:1014C0005F4FB201C8010E943618811120C01EAEC4
:1014D0001DAE82E993E09CAF8BAF21961FAE2197A2
:1014E000A896EEADFFADA8976E0E7F1EF30180812A
:1014F000811120C0BE01655C7F4FC1010E94001CAC
:1015000046E854E0B101C5010E946E1C31C0CE0C0A
:10151000DF1CC2010E942218B3CFC60186199709A9
:10152000A8969FAF8EAFA897B201CE01CB960E942E
:10153000001CD6CF19A218A282E993E09F8F8E8F4C
:101540001BA221968FAD219781112DC0F501138229
:10155000128288EE93E0A0E0B0E084839583A683B6
:10156000B78382E194E091838083128E118E14867A
:10157000C501C959DF4F0FB6F894DEBF0FBECDBF0E
:10158000DF91CF911F910F91FF90EF90DF90CF905F
:10159000BF90AF909F908F907F906F905F904F9093
:1015A0003F902F9008958250A6962FADA697A30145
:1015B0008230C8F46AE170E1C4010E9436188823C1
:1015C00029F2A6968FADA697867039F049A95AA937
:1015D0006BA97CA9C4010E941915B401C1010E9424
:1015E000001CA3018FCFBE01655C7F4FC4010E9428
:1015F0003618882309F4AACFCE01CB960E94221870
:10160000E0CF0F931F93CF93DF93CDB7DEB7AD97A6
:101610000FB6F894DEBF0FBECDBF8091480C882373
:1016200031F08091781190917911892B11F40E94F9
:101630003B726DE574E0CE0188960E9474848091BF
:10164000470C8823E1F060EA71E1CE0101960E9427
:101650006284CE0101960E94C830CE0101960E949C
:10166000D58368E972E0CE0101960E947484CE01B0
:1016700001960E947A30CE0101960E94D583809116
:10168000480C81111BC08091460C81117CC0809157
:10169000450C882309F44CC10FE110E08091440C03
:1016A000882309F4BDC00150110909F45DC064E14B
:1016B00070E080E090E00E945E0DF0CF80917811A4
:1016C00090917911892BF9F264E170E080E090E06B
:1016D0000E945E0D62E971E1CE0188960E946083EE
:1016E00064E771E1CE0101960E946B84AE014F5F09
:1016F0005F4F63E070E088E992E00E94B83D8C01A2
:10170000CE0101960E94D5830130110539F1BE0149
:10171000685D7F4FCE014C960E946B8466E571E157
:10172000CE014C960E94EF82BC01CE0101960E9430
:101730006B84CE0101960E947A30CE0101960E9400
:10174000D583CE014C960E94D5838091E813909169
:10175000E91301969093E9138093E8131092480CD3
:101760008091460C81118FCFCE0188960E94D5833F
:10177000AD960FB6F894DEBF0FBECDBFDF91CF910F
:101780001F910F91089580916C1190916D11892B8B
:1017900009F47DCF64E871E1CE0188960E946083F0
:1017A00068E671E1CE0101960E946B84AE014F5F45
:1017B0005F4F62E070E082EB92E00E94B83D8C01E6
:1017C000CE0101960E94D5830130110509F45FCF47
:1017D000BE01685D7F4FCE014C960E946B8466E52A
:1017E00071E1CE014C960E94EF82BC01CE010196C0
:1017F0000E946B84CE0101960E947A30CE01019640
:101800000E94D583CE014C960E94D5838091E81327
:101810009091E91301969093E9138093E81337CFE1
:1018200043E165EA72E0CE0101960E94F689BE01AD
:101830006F5F7F4F87E493E10E94872C81E0809364
:10184000440C87E493E10E94501C8823E1F164E793
:1018500071E187E493E10E94978587E493E10E9418
:101860005C1C62E370E080E090E00E945E0D1092EC
:10187000440C8091470C882331F1CE014C960E9494
:101880008E2F6DE877E0CE0182960E947484BE01AF
:10189000645E7F4FCE0182960E94EF82BC01CE0132
:1018A00001960E946B84CE0101960E947A30CE018F
:1018B00001960E94D583CE0182960E94D583CE01E7
:1018C0004C960E94D58387E493E10E945C1C62E3FE
:1018D00070E080E090E00E945E0D1092440C43E1C5
:1018E00062EB72E0CE0101960E94F689BE016F5F45
:1018F0007F4F87E493E10E94872C81E08093440C22
:1019000087E493E10E94501C882331F068E671E17E
:1019100087E493E10E94978587E493E10E945C1C31
:1019200062E370E080E090E00E945E0D1092440C53
:101930006DE574E088E691E10E94C2816DE574E096
:1019400084E791E10E94C2810FCF89EF90E10E946C
:10195000D5838FEF90E10E94D58385E091E10E94CD
:10196000D5838BE091E10E94D58381E191E10E94D2
:10197000D58387E191E10E94D5838DE191E10E94B9
:10198000D58383E291E10E94D58384E491E10E94B2
:10199000D5838AE491E10E94D58380E591E10E949C
:1019A000D58386E591E10E94D5838CE591E10E9483
:1019B000D58382E691E10E94D58388E691E10E9479
:1019C000D5838EE691E10E94D58384E791E10E9460
:1019D000D5838DEE92E10E94D58383EF92E10E9440
:1019E000D58389EF92E10E94D5838FEF92E10E9427
:1019F000D58385E093E10E94D5838BE093E10C943D
:101A0000D5838091F002811110C081E08093F002B3
:101A10008093EF0280916913982F946090936913DB
:101A20008C600E94737B0C94F0288091EF028823D5
:101A3000D1F310926E1360E083E693E10E940C0EE6
:101A40001092EF02809169138B7F809369138860F5
:101A50000E94737B1092F0020895CF92DF92EF9272
:101A6000FF920F931F93CF93DF93CDB7DEB7AA9763
:101A70000FB6F894DEBF0FBECDBFBC01CE01859678
:101A80000E946B84CE0185960E943082BE016B5D00
:101A90007F4F8AEA9EE00E94978568EE73E080E0BF
:101AA00090E00E945E0D8AEA9EE00E94B17760EDB0
:101AB00077E080E090E00E945E0D83E290E09A8300
:101AC0008983FE0133968CE1DF011D928A95E9F747
:101AD000F12CE12C01E010E08AEA9EE00E942277DE
:101AE000892B09F449C08AEA9EE00E940077CC2441
:101AF000C394D12CCC0EDD1EC00ED11EF601808306
:101B000065E070E080E090E00E945E0DD6018C916F
:101B10008A3019F488ECE82EF12C0F5F1F4FB8ECD7
:101B2000EB16F10419F00F301105B1F6FE01E00FCC
:101B3000F11F1282BE016F5F7F4FCE014F960E9450
:101B40007484CE014F960E947A30CE014F960E9447
:101B5000D583CE0185960E94D583AA960FB6F894B8
:101B6000DEBF0FBECDBFDF91CF911F910F91FF90D0
:101B7000EF90DF90CF90089562E370E080E090E016
:101B80000E945E0DBFEFEB1AFB0AC9CFDF92EF9206
:101B9000FF920F931F93CF93DF93CDB7DEB72C97B0
:101BA0000FB6F894DEBF0FBECDBF8C0180915E0AE8
:101BB000882309F486C0109265096DE574E0CE01B2
:101BC00001960E947484F12CE12CDD24D3948AEADE
:101BD0009EE00E9422771816190694F480916509F8
:101BE00081110EC08AEA9EE00E9400778A30D1F50A
:101BF0008D819E81892B09F443C0D092650940C034
:101C000062E370E080E090E00E945E0DEF2851F00A
